:100000000C94EC230C941D240C941D240C941D249E
:100010000C941D240C941D240C941D240C941D245C
:100020000C941D240C941D240C941D240C941D244C
:100030000C941D240D94EF570C941D240C941D2436
:100040000C941D240C949DF60C941D240C941D24DA
:100050000C941D240C941D240C9464F30D94A5574A
:100060000C941D240C94495D0C943F5D0C941D244C
:100070000C941D240C941D240C941D240C941D24FC
:100080000C9415410C941D240C941D240C941D24D7
:100090000C941D240C941D240C941D240C941D24DC
:1000A0000C941D240C941D240C94E7400C941D24E6
:1000B0000C941D240C941D240C941D240C941D24BC
:1000C0000C941D240C941D240C941D240C941D24AC
:1000D0000C941D240C941D240C941D240C941D249C
:1000E0000C941D24084AD73B3BCE016E84BCBFFD57
:1000F000C12F3D6C74319ABD56833DDA3D00C77FF8
:1001000011BED9E4BB4C3E916BAAAABE0000008090
:100110003F05A84CCDB2D44EB93836A9020C50B91F
:10012000918688083CA6AAAA2ABE000000803F004B
:100130000C94B89B0C9471900C94249C0C94F2DE5B
:100140000C9447950C9443B00C94D5C90C94868CB0
:100150000D94D2510C94E9920D949D500D943461FC
:100160000C9439930C94E1C90C94B9B10D94DC5101
:100170000C9463D30C9438A10D94C8510C949093B3
:100180000C94B79A0C94E7970D9499500C942DA069
:100190000C94F9C90C94BF430C94D2D20D94C35063
:1001A0000C942AB30D94BF500D94AB500C94FACD1F
:1001B0000D949A510D94B1500C94B48C0C9447DE6C
:1001C0000D944A2F0C94DF910C94AF9B0C946E917C
:1001D0000C94CC400C94F3970C946C910C943F9C31
:1001E0000C9455C00C9425240D9416610C940EAFFC
:1001F0000D948C500C94EF970C94815D0C94799134
:100200000C94128D0D94A3500D94B8510C94E9B92F
:100210000C94A69A0C949D950C94E7C90C94EB97BA
:100220000C947B400D946D500C94FCA30D9488505D
:100230000C948A980C94C9C90D9409520C94579146
:100240000C9470A70C9496400C9475930C94AB98F6
:100250000D94F5510D948D510C94F8C70D94FF51E8
:100260000C948A930C94DB970C94C85D0C94E2DD9B
:100270000C94FBA60C94C98F0C9449900C94D9391A
:100280000D94EE500C94EE910D9427510C94199905
:100290000C94F3C90C94A7920D94B9500C941FB50B
:1002A0000C94E9DF0C9488900C947E910D94135279
:1002B0000C94A09A0C94DBC90C94608F0C94C59B91
:1002C0000D94A4510C9488910C944B910D941D5253
:1002D0000C94C89B0C94FA260C9483910C94219C4A
:1002E0000C94C29A0C942EAE0C94AE8F0C940D9676
:1002F0000C941FDF0C94AC9B0D9427520C948E939E
:100300000C940C8D0D9495510C94F5B70C9403DE60
:100310000C94F1D20C94C3D30C9422240D94D3509A
:100320000C9488930C94DB5D0C94518F0C94279063
:100330000C94D75D0C94AE9A0D942C510C94F38CC4
:100340000C9470CA0C9412920C9402940C94E3DAFC
:100350000C94E35D0C9432990C94589E0C9444D305
:100360000C9462DE0C940BCA0D94AE510C94E28F87
:100370000D9438510C94E2DA0C94DF5D0C94B39830
:100380000C94E3970C94A4AC0C94FFC90C94E75D17
:100390000C944B990C94AA5D0C9486930C94B69093
:1003A0000C94F7910C94A4D30C94CEDC0C94B29BD7
:1003B0000C94B95D0D94E6510C94A98C0C94CB9BD4
:1003C0000C946ADD0C94B59B0C94BB9B0D94A750C8
:1003D0000C94DF970C946F260D94B5500C94A99B48
:1003E0000C943B950C9436900C9495950C94E7984E
:1003F0000C9486C10C946A910C94FFB70C94DBC5E5
:100400000C94F95D0C9492930C94C5910C94EDD3DB
:100410000C9499950C9484930D943E510C948C9368
:100420000D9472500C94F1910C94F7970D94C46054
:100430000C94ECA60C941F240C94F6A60D948450F6
:100440000C94E0DE0C9462900C949B8F0C94B14061
:100450000C94DCB00C94F8920C9417B80D94535192
:100460000C94D7970C94C39B0C94EE5D0C94798FED
:100470000C9405CA0C9421270D94282F0C9453B684
:100480000C9442910C9433A90C94F58F0D94FB2E8F
:100490000C9400990C94D3970C94BE9B0C94D0BEF2
:1004A0000C94AACA0C94E8BC0C941F8F0D94935022
:1004B0000C949F900C94F1A60C948D910D949050F7
:1004C0000C947FAB0D94C0510C94CF5D0D944851AA
:1004D0000C9460DA0C94388F0C94A4AF0C94F491C3
:1004E0000C94015E0C94EDC90C944DDD0C94C3C9C1
:1004F0000C9498260C94D35D0C94888F0C94CFC9DF
:100500000C940E900C949E9B0C9456990C9436DC93
:100510004E414E494E495459494E46CDCCCC3D0AE8
:10052000D7233C17B7D13877CC2B329595E6241FCB
:10053000B14F0A000020410000C84200401C462084
:10054000BCBE4CCA1B0E5AAEC59D7400407A10F357
:100550005A00A0724E18090010A5D4E80000E876F1
:1005600048170000E40B54020000CA9A3B00000048
:10057000E1F505000080969800000040420F000061
:1005800000A08601000000102700000000E8030022
:100590000000006400000000000A000000000001EC
:1005A00000000000002C76D888DC674F0823DFC1EC
:1005B000DFAE59E1B1B796E5E3E453C63AE65199A7
:1005C0007696E8E6C28426EB898C9B62ED407C6FD0
:1005D000FCEFBC9C9F40F2BAA56FA5F490055A2A87
:1005E000F75C936B6CF9676DC11BFCE0E40D47FE93
:1005F000F520E6B500D0ED902E0300943577050088
:1006000080841E080000204E0A000000C80C33330E
:1006100033330F986E12831141EF8D2114893BE61D
:100620005516CFFEE6DB18D1844B381BF77C1D90A6
:100630001DA4BBE424203284725E228100C9F1240F
:10064000ECA1E53D27434F4D4D554E49434154499B
:100650004F4E0044525952554E004552524F52533C
:1006600000494E464F004543484F004572726F7235
:100670002077726974696E6720746F204545505207
:100680004F4D210A0053544F505045442E200050E6
:1006900072696E7465722073746F70706564206423
:1006A000756520746F206572726F72732E204669B3
:1006B0007820746865206572726F7220616E6420A4
:1006C000757365204D39393920746F2072657374E4
:1006D0006172742E202854656D7065726174757234
:1006E000652069732072657365742E2053657420CC
:1006F00069742061667465722072657374617274C6
:10070000696E67290A004E6F20436865636B7375D5
:100710006D2077697468206C696E65206E756D62F6
:1007200065722C204C617374204C696E653A200010
:100730004E6F20436865636B73756D2077697468CD
:10074000206C696E65206E756D6265722C204C613F
:100750007374204C696E653A2000636865636B733F
:10076000756D206D69736D617463682C204C6173C5
:1007700074204C696E653A20004C696E65204E7598
:100780006D626572206973206E6F74204C617374A2
:10079000204C696E65204E756D6265722B312C2080
:1007A0004C617374204C696E653A20004D313130D4
:1007B0000053657269616C20737461747573206D88
:1007C00069736D617463680A00776169740A005324
:1007D000442072656164206572726F720A00486F0E
:1007E00074656E642049646C652054696D656F752D
:1007F0007400486F74656E642049646C65205469A8
:100800006D656F75740A002121204B494C4C2063A3
:100810006175736564206279204B494C4C20627588
:1008200074746F6E2F70696E0A002121204B494C41
:100830004C2063617573656420627920746F6F204A
:100840006D75636820696E6163746976652074698B
:100850006D65202D2063757272656E7420636F6DF7
:100860006D616E643A20004D656469612052656D6A
:100870006F766564004D6564696120496E736572C9
:10088000746564004D313030305300627573793ACD
:100890002070617573656420666F7220696E707573
:1008A000740A00627573793A20706175736564200B
:1008B000666F7220757365720A00627573793A20EB
:1008C00070726F63657373696E670A00506C65615F
:1008D0007365205265736574005052494E544552F9
:1008E0002048414C5445440025533A20255300707C
:1008F0006F7765726F6666004B494C4C45442E20FD
:10090000005072696E7465722068616C7465642E43
:10091000206B696C6C28292063616C6C6564210A0A
:100920000053544F505045442E20005072696E744D
:1009300065722073746F70706564206475652074CF
:100940006F206572726F72732E204669782074680A
:1009500065206572726F7220616E64207573652008
:100960004D39393920746F20726573746172742E39
:10097000202854656D7065726174757265206973A5
:100980002072657365742E2053657420697420612C
:10099000667465722072657374617274696E67291A
:1009A0000A006563686F3A004572726F723A0042DE
:1009B000696C696E656172204C6576656C696E67FD
:1009C00020477269643A0A0021212053544F502075
:1009D00063616C6C65642062656361757365206F2B
:1009E0006620424C546F756368206572726F722086
:1009F0002D20726573746172742077697468204D5C
:100A00003939390A0021212053544F502063616C39
:100A10006C65642062656361757365206F66204252
:100A20004C546F756368206572726F72202D20724E
:100A30006573746172742077697468204D3939392F
:100A40000A005072696E74696E67204F626A65634E
:100A500074002553202569002F2F616374696F6E20
:100A60003A00737461727400656E6400486F746557
:100A70006E6420746F6F20636F6C640A0053656E40
:100A800064204D31303820746F20726573756D6548
:100A90000A00496E736572742066696C616D656EDB
:100AA0007420616E642073656E64204D3130380AA5
:100AB0000052656865617420446F6E650052656818
:100AC000656174696E672E2E2E00526568656174CB
:100AD000004865617465722054696D656F757400B6
:100AE00053656E64204D31303820746F2068656125
:100AF00074206E6F7A7A6C650A004E6F7A7A6C6534
:100B0000205061726B65640070617573656400509C
:100B10006175736500726573756D65640052657308
:100B2000756D696E67004732362043616E63656C90
:100B30006564004732362048656174696E67204EEF
:100B40006F7A7A6C65004732362048656174696E49
:100B500067204265640057616974696E6720666F3B
:100B600072206865617475702E0A00466978656444
:100B7000204C656E677468205072696D6500446F23
:100B80006E65205072696D696E67004D616E7561AA
:100B90006C207072696D696E672E2E2E004C656137
:100BA00076696E6720473236003F53706563696629
:100BB00069656420582C5920636F6F7264696E6197
:100BC0007465206F7574206F6620626F756E647334
:100BD0002E0A003F28522965706561742076616C89
:100BE0007565206E6F7420706C61757369626C65D9
:100BF0003B206D757374206265206174206C6561A3
:100C0000737420312E0A003F53706563696669650D
:100C100064206E6F7A7A6C652074656D70657261A0
:100C200074757265206E6F7420706C617573696283
:100C30006C652E0A003F53706563696669656420C0
:100C400066696C616D656E742073697A65206E6F7C
:100C50007420706C61757369626C652E0A003F5375
:100C60007065636966696564207072696D65206C82
:100C7000656E677468206E6F7420706C617573693F
:100C8000626C652E0A003F5370656369666965642E
:100C9000206E6F7A7A6C652073697A65206E6F7446
:100CA00020706C61757369626C652E0A003F526535
:100CB0007472616374696F6E204D756C7469706CC9
:100CC000696572206D757374206265207370656349
:100CD00069666965642E0A003F53706563696669D9
:100CE00065642052657472616374696F6E204D751E
:100CF0006C7469706C696572206E6F7420706C61C1
:100D0000757369626C652E0A003F5370656369668E
:100D1000696564206C6179657220686569676874CB
:100D2000206E6F7420706C61757369626C652E0A39
:100D30000043292E0A003F53706563696669656444
:100D4000206265642074656D70657261747572658A
:100D5000206E6F7420706C61757369626C652028F9
:100D600034302D00473236207374617274696E67B7
:100D70002E2E2E0A004F46460A0046616465204822
:100D800065696768742000426564204C6576656C0F
:100D9000696E6720004661696C656420746F206528
:100DA0006E61626C6520426564204C6576656C6995
:100DB0006E670A00496E76616C6964206D657368C0
:100DC0002E0A0050726F62696E6720506F696E74F0
:100DD0000025532025692F2569002E0A002F005079
:100DE000726F62696E67206D65736820706F696EDF
:100DF000742000202844525952554E290047323958
:100E0000204175746F20426564204C6576656C697D
:100E10006E67003F20284C2C522C462C4229206F14
:100E20007574206F6620626F756E64732E0A003FC2
:100E30002856296572626F7365206C6576656C2033
:100E4000696D706C61757369626C652028302D3432
:100E5000292E0A00426164205A2076616C75650A69
:100E6000004E6F2062696C696E65617220677269FD
:100E7000640A00446576696174696F6E0025533AAF
:100E80002025730046696E6973686564210A003A1B
:100E9000207A3A2000206F662000476F696E672035
:100EA000746F3A20580043570A00206469723A0070
:100EB00020616E676C653A005374617274207261D0
:100EC000646975733A004D343820506F696E740050
:100ED00025533A2025642F256400506F7369746987
:100EE0006F6E696E67207468652070726F62652E20
:100EF0002E2E0A003F4C656773206F66206D6F765B
:100F0000656D656E7420696D706C61757369626C76
:100F1000652028302D3135292E0A003F2028582CF5
:100F20005929206F7574206F6620626F756E647327
:100F30002E0A0050726F6265206F7574206F6620F4
:100F4000626F756E6473003F53616D706C652073E2
:100F5000697A65206E6F7420706C61757369626C5C
:100F6000652028342D3530292E0A004D3438205A7A
:100F70002D50726F6265205265706561746162699F
:100F80006C69747920546573740A003F285629658A
:100F900072626F7365206C6576656C20696D706C2C
:100FA00061757369626C652028302D34292E0A0022
:100FB0005374616E6461726420446576696174691A
:100FC0006F6E3A20002052616E67653A2000204D16
:100FD00061783A2000204D696E3A200020536967FD
:100FE0006D613A20004D65616E3A2000205200414B
:100FF0006363656C65726174696F6E3A2050005767
:1010000041524E494E4721204C6F77205A204A6565
:10101000726B206D6179206C65616420746F20753E
:101020006E77616E746564207061757365732E0AE6
:101030000020204D61783A2000200020204D696E6C
:101040003A2000536F667420656E6473746F70731A
:101050003A20004D32342053256C642054256C64B2
:10106000004739322E392045257300473120462567
:1010700064004739322E39205A2573004731205AEF
:101080003020463230300047312058257320592512
:1010900073204633303030004D34323020532569D0
:1010A000205A2573004D31303620502569205325B4
:1010B00069004D32303020442573004732385230B9
:1010C0005859004739322E39204530205A300A47C6
:1010D000315A2573004D31303920532569004D3187
:1010E000393020532569004D343230205330205A96
:1010F000300020496E76616C696420657874727581
:10110000646572200047322F47332062616420708B
:101110006172616D65746572730A00536C65657008
:101120002E2E2E005A2050726F626520506173740B
:10113000204265640A005A2050726F626520506137
:10114000737420426564004732384C30004D3131B1
:10115000372050726F6265206661696C65642E0A83
:101160004732380A0070726F62655F726577697026
:101170006500473239205265747279696E67005094
:10118000726F62696E67204661696C6564004D31FB
:10119000313720426564206C6576656C696E672026
:1011A0006661696C65642E0A4730205A31300A4DF9
:1011B0003330302050323520533838300A4D3330F8
:1011C00030205035302053300A4D333030205032EB
:1011D0003520533838300A4D3330302050353020E8
:1011E00053300A4D333030205032352053383830A8
:1011F0000A4D333030205035302053300A473420E8
:1012000053310070726F62655F6661696C6564007E
:101210004D31313720426564206C6576656C696EAE
:101220006720646F6E652E00205A3A200020593ADC
:10123000200042656420583A20004D657368207094
:101240006F696E74206F7574206F662072616E67AF
:10125000650A004D302053746F70004D3120537477
:101260006F7000436C69636B20746F2052657375F7
:101270006D652E2E2E004E6F204D6F76652E00452B
:101280006E642066696C65206C6973740A0042653F
:1012900067696E2066696C65206C6973740A004E1C
:1012A0006F206D656469610A00526573756D696EC2
:1012B0006720534400286E6F2066696C65290043DF
:1012C000757272656E742066696C653A20005072A2
:1012D000696E742074696D653A20000A53746174F4
:1012E000733A2046696C616D656E74207573656430
:1012F0003A20002C204C6F6E67657374206A6F6211
:101300003A2000546F74616C2074696D653A200056
:1013100053746174733A20002C204661696C6564D3
:101320003A20002C2046696E69736865643A200093
:101330005072696E74733A200053746174733A206A
:1013400000436F6F6C696E672E2E2E0048656174C6
:10135000696E672E2E2E0045202553006F6B006F9F
:10136000666600660661065A06530645064445420F
:1013700055473A004D3131332053004265642043D4
:101380006F6F6C696E672E2E2E0042656420486573
:101390006174696E672E2E2E00537550655220437E
:1013A000522D3230204F46462E002F2F004D313423
:1013B0003520533C696E6465783E206F7574206FEC
:1013C000662072616E67652028302D31290A004D34
:1013D00032303620580046523A0020466C6F773A39
:1013E00020003A200020536572766F2000206F7530
:1013F00074206F662072616E67650A0053657276AD
:101400006F200020643A0020693A0020703A0049B9
:101410006E76616C69642065787472756465720AB1
:101420000020643A0020693A0020703A004C43449E
:1014300020436F6E74726173743A200064697300A4
:10144000656E0043290A0061626C656420286D693D
:101450006E2074656D702000436F6C642065787435
:1014600072756465732061726520004D34323120DD
:10147000696E636F727265637420706172616D650D
:101480007465722075736167650A004D6573682025
:10149000706F696E74206F7574206F662072616E54
:1014A00067650A004F666673657473204170706CDF
:1014B000696564004572723A20546F6F20666172EC
:1014C0002100546F6F206661722066726F6D20720A
:1014D00065666572656E636520706F696E740A007B
:1014E000454550524F4D204F4B0A002E0A002028F0
:1014F000302D313029002076616C7565206F757450
:10150000206F662072616E676500416476616E636C
:1015100065204B3D004F4646004F4E00506F7765AB
:10152000722D6C6F7373207265636F7665727920AC
:10153000004D383400446F6E65207072696E7469B6
:101540006E672066696C650A004D3737004D333190
:10155000004361703A004D4541545041434B0043B4
:101560004F4F4C45525F54454D5045524154555292
:1015700045004348414D4245525F54454D50455208
:1015800041545552450042414259535445505049E7
:101590004E470041524353004D4F54494F4E5F4D0B
:1015A0004F44455300544845524D414C5F50524FB3
:1015B00054454354494F4E004C4F4E475F46494CAB
:1015C000454E414D45004155544F5245504F5254A0
:1015D0005F53445F5354415455530053445F575233
:1015E00049544500524550454154005344434152EB
:1015F000440050524F4D50545F535550504F525429
:1016000000454D455247454E43595F504152534561
:101610005200434153455F4C494748545F42524949
:101620004748544E45535300544F47474C455F4C31
:10163000494748545300534F4654574152455F5011
:101640004F574552004255494C445F50455243451F
:101650004E54004C4556454C494E475F4441544119
:10166000005A5F50524F42450052554E4F5554005C
:101670004155544F4C4556454C005052494E545FCD
:101680004A4F420050524F47524553530041555420
:101690004F5245504F52545F54454D5000564F4C99
:1016A000554D455452494300454550524F4D004217
:1016B000494E4152595F46494C455F5452414E5341
:1016C0004645520053455249414C5F584F4E5F5872
:1016D0004F4646004649524D574152455F4E414D97
:1016E000453A4D61726C696E20322E302E375F4460
:1016F00057372E332E3120544D33442032534D442E
:10170000424220284170722032392032303231205A
:1017100031343A30303A30342920534F5552434512
:101720005F434F44455F55524C3A68747470733A46
:101730002F2F6769746875622E636F6D2F496E7302
:10174000616E6974794175746F6D6174696F6E2F24
:101750004D61726C696E2F747265652F437265619D
:101760006C6974794477696E5F322E302050524F25
:10177000544F434F4C5F56455253494F4E3A312ECA
:1017800030204D414348494E455F545950453A53E6
:10179000755065522043522D3230204558545255D1
:1017A0004445525F434F554E543A312055554944B4
:1017B0003A63656465326132662D343161322D34AD
:1017C0003734382D396231322D6335356336326620
:1017D00033363766660A0050726F6265204F666660
:1017E000736574205A0050726F6265204F6666738D
:1017F0006574205A00290A0020746F20003F5A2087
:101800006F7574206F662072616E676520280029ED
:101810000A0020746F20003F59206F7574206F6696
:101820002072616E676520282D00290A0020746FE0
:1018300020003F58206F7574206F662072616E67BC
:101840006520282D0050726F6265204F66667365B3
:101850007420580043616E6E6F74206F70656E2047
:1018600073756264697220002569730025696D20B3
:10187000256973002569682025696D202569730035
:10188000256964202569682025696D202569730014
:1018900025697920256964202569682025696D20DE
:1018A0002569730023646566696E65204445464179
:1018B000554C545F00626564004B6420004B692006
:1018C000004B702000504944204175746F74756E50
:1018D000652066696E69736865642120507574209F
:1018E000746865206C617374204B702C204B6920E8
:1018F000616E64204B6420636F6E7374616E7473E9
:101900002066726F6D2062656C6F7720696E746FF0
:1019100020436F6E66696775726174696F6E2E68B9
:101920000A00504944204175746F74756E652066D5
:1019300061696C6564212074696D656F75740A0056
:10194000504944204175746F74756E6520666169F5
:101950006C6564212054656D706572617475726583
:1019600020746F6F20686967680A00204B643A2012
:1019700000204B693A2000204B703A200020436C35
:10198000617373696320504944200A00204E6F2020
:101990006F76657273686F6F740A002054753A2011
:1019A00000204B753A2000206D61783A2000206DB0
:1019B000696E3A200020643A200020626961733A1F
:1019C0002000504944204175746F74756E65207312
:1019D000746172740A00504944204175746F7475C3
:1019E0006E65206661696C6564212054656D706563
:1019F00072617475726520746F6F20686967680A18
:101A000000504944204175746F74756E65005049EB
:101A100044204175746F74756E65206661696C65EC
:101A20006421204261642068656174657220696484
:101A30000A004572723A207574663820666F6E74BB
:101A4000206E6F7420696E697469616C697A65646F
:101A50002E004572723A207574663820666F6E7477
:101A6000206E6F7420696E697469616C697A65644F
:101A70002E004572723A207574663820666F6E7457
:101A8000206E6F7420696E697469616C697A65642F
:101A90002E00FFE0FFD140A0C8A6A22FF80023AC83
:101AA00000AF10FFFEFF05FFD0FFE0FFC1FFD1E256
:101AB00040A0C8A6A22FF800238127AC00AFFFD01A
:101AC000FF64FFD1A5FFD0FF64FF64FFD1A4FFD066
:101AD000FF16FFFE000C0F00FE07022503BB017F6F
:101AE000FE08FE08FE05080806000040F0C88888C9
:101AF000987810050808060000C0F888888888884B
:101B0000F80505050600012030F830200508080614
:101B100000002070F820202020E00509090600FFC1
:101B20002070A8A8B888887020070505070001D88C
:101B30006C366CD80509090600FFF8A888888888E3
:101B400088A8F8050A0A0600FE205050505088A8C0
:101B5000A8887003030306000340A040FFFFFFFFB7
:101B6000FFFFFFFFFFFFFFFFFFFFFFFFFFFFFFFF85
:101B7000FFFF0000000605FF010707060200808046
:101B80008080800080030303060105A0A0A0050655
:101B90000606000050F85050F8500509090600FFED
:101BA0002070A8A07028A87020050707060000C8AC
:101BB000C8102040989805070706000040A0A040E4
:101BC000A8906801030306020580808003090906C6
:101BD00001FF204040808080404020030909060129
:101BE000FF8040402020204040800507070600007D
:101BF00020A8702070A8200505050600012020F807
:101C000020200203030601FFC040800501010600F9
:101C100003F8020202060100C0C005070706000023
:101C200008101020404080050707060000708898C3
:101C3000A8C8887003070706010040C04040404024
:101C4000E0050707060000708808102040F8050727
:101C500007060000F808103008887005070706001E
:101C60000010305090F81010050707060000F880AB
:101C7000F008088870050707060000304080F088EB
:101C80008870050707060000F808101020202005BE
:101C900007070600007088887088887005070706A7
:101CA000000070888878081060020505060100C0F1
:101CB000C000C0C00206060601FFC0C000C04080D0
:101CC00003050506010120408040200503030600AE
:101CD00002F800F803050506010180402040800558
:101CE000070706000070881020200020050707065F
:101CF00000007088B8A8B88070050707060000705B
:101D00008888F8888888050707060000F04848702A
:101D10004848F005070706000070888080808870BA
:101D2000050707060000F04848484848F00507073F
:101D3000060000F88080F08080F8050707060000A4
:101D4000F88080F08080800507070600007088809A
:101D500080988870050707060000888888F88888BA
:101D600088030707060100E04040404040E00507C7
:101D700007060000381010101090600507070600D5
:101D8000008890A0C0A0908805070706000080800A
:101D900080808080F805070706000088D8A888881A
:101DA00088880507070600008888C8A898888805DD
:101DB000070706000070888888888870050707066E
:101DC0000000F08888F0808080050707060000701A
:101DD000888888A89068050707060000F08888F0C2
:101DE000A09088050707060000708880700888703A
:101DF000050707060000F8202020202020050707FF
:101E00000600008888888888887005070706000013
:101E10008888888850502005070706000088888831
:101E200088A8A85005070706000088885020508819
:101E30008805070706000088885020202020050715
:101E400007060000F80810204080F8030909060181
:101E5000FFE080808080808080E00507070600002A
:101E6000804040201010080309090601FFE02020EF
:101E70002020202020E005030306000520508805CF
:101E800001010600FEF8030303060105804020055A
:101E90000505060000700878887805070706000029
:101EA0008080F0888888F005050506000070808035
:101EB0008870050707060000080878888888780574
:101EC00005050600007088F0807005070706000011
:101ED000304840E04040400507070600FE70888813
:101EE000887808700507070600008080F0888888D9
:101EF000880307070601004000C0404040E0040995
:101F0000090601FE10003010101010906005070740
:101F100006000080808890E0908803070706010093
:101F2000C04040404040E0050505060000D0A8A89C
:101F3000A8A8050505060000B0C88888880505051D
:101F400006000070888888700507070600FEF08884
:101F50008888F080800507070600FE7888888878E2
:101F60000808050505060000B0C880808005050545
:101F700006000078807008F00507070600002020A2
:101F8000F820202018050505060000888888986834
:101F9000050505060000888888502005050506000F
:101FA000008888A8A8500505050600008850205024
:101FB000880507070600FE888888502040800505B0
:101FC00005060000F8102040F80309090601FF206B
:101FD00040404080404040200109090602FF8080C7
:101FE000808080808080800309090601FF80404056
:101FF00040204040408005030306000248A890FFAF
:10200000554E4C4F41442046494C414D454E54009D
:102010004C4F41442046494C414D454E54004649A1
:102020004C414D454E54204348414E474500426582
:102030006400456E636C6F73757265002568753A50
:1020400025303268750025303268753A253032689F
:102050007500202020202020200020202020001F8C
:10206000E020102010201010201020201020103010
:10207000300840048003001FE03FF03FF03FF01FB6
:10208000E01FE03FF03FF03FF00FC0078003003F4C
:10209000FFF038007030FC3020FC10207810203029
:1020A000102C00D02E31D02F7BD02F7BD02E31D0D2
:1020B0002C00D020301020781020FC1030FC30385C
:1020C00000703FFFF03FFFF038007031863023870B
:1020D000102787902F87D02F03D020301020781022
:1020E0002078102030102F03D02F87D027879023FF
:1020F00087103186303800703FFFF01FFFF81FFF58
:10210000F804104002082002082004104008208033
:102110001041001041000820800410400000001F02
:10212000FFF81FFFF8FFFFFF8000018E00E19F0115
:10213000F19381399F81F99F81F99FB9F98F28F136
:102140008038018000019FFFF99174999B06A99B3B
:1021500054A99B56A99B54999FFFF9FFFFFF6E6FEF
:1021600074696669636174696F6E200063616E6390
:10217000656C005072696E742041626F72746564A0
:10218000004469736D6973730055492041626F7231
:10219000746564004D323520500A4D32340052656A
:1021A00073756D6500554920506175736500506108
:1021B0007573696E672E2E2E00726573756D6500DE
:1021C0004D32340000FE0003FF8007C7C00701E066
:1021D0000000E00000F00000700400700E00701FAE
:1021E00000703F80F00E00E00F01E007C7C003FF62
:1021F0008000FE0000FE0003FF8007C7C00F01E063
:102200000E00E03F80F01F00700E007004007000B0
:1022100000700000F00000E00701E007C7C003FF06
:102220008000FE000E000E000E000E000E000E00DC
:102230000E000E007FC03F801F000E00040004004F
:102240000E001F003F807FC00E000E000E000E002B
:102250000E000E000E000E00FFFFFF7F80FFC0FF8C
:10226000C0FFC07F807F80FFC0FFC0FFC03F001E57
:10227000000C0050726F6265205A204F66667365CD
:1022800074004C6F6164206D6D00556E6C6F6164FD
:10229000206D6D0046696C2E204469612E0045203A
:1022A000696E206D6D5E3300416476616E636520FA
:1022B0004B004D33303320553120452569205325BF
:1022C0006900504944204175746F74756E65202A09
:1022D000005049442D44202A005049442D49202AC9
:1022E000005049442D50202A002008204661637484
:1022F000002008204D6178002008204D696E004FB5
:102300006666004F6E004175746F74656D7000569F
:1023100054726176204D696E00566D696E00566D7F
:102320006178204500566D6178205A00566D6178BD
:10233000205900566D6178205800416D6178204524
:1023400000416D6178205A00416D6178205900414B
:102350006D6178205800412D54726176656C0041A2
:102360002D5265747261637400416363656C00563D
:10237000652D4A65726B00565A2D4A65726B005680
:10238000592D4A65726B0056582D4A65726B005084
:10239000726F6265205A204F6666736574005072D2
:1023A0006F62652059204F66667365740050726FC6
:1023B00062652058204F666673657400452073740B
:1023C0006570732F6D6D005A2053746570732F6D97
:1023D0006D00592053746570732F6D6D0058205334
:1023E000746570732F6D6D00416476616E63656412
:1023F0002053657474696E6773003F0043616E63B8
:10240000656C00496E6974004D34323800496E695C
:102410007469616C697A6520454550524F4D00469C
:10242000696C616D656E740054656D706572617480
:102430007572650053746570732F6D6D0050726F07
:102440006265204F666673657473004A65726B003F
:10245000416363656C65726174696F6E0056656C8B
:102460006F636974790053657420486F6D65204F00
:1024700066667365747300436F6E66696775726133
:1024800074696F6E003F004E65787420506F696EFE
:102490007400446F6E65004E65787400486F6D6916
:1024A0006E672058595A003F0043616E63656C2087
:1024B0004F626A656374004E4F0059455300436193
:1024C0006E63656C204F626A656374203D004D61E8
:1024D000696E0053572D4D6F64650053746F77001C
:1024E0004465706C6F790053656C662D5465737428
:1024F00000526573657400426564004E6F7A7A6CB1
:10250000650046616E20537065656400436F6E66BA
:10251000696775726174696F6E00526573746F726A
:10252000652044656661756C7473004C6F6164204E
:1025300053657474696E67730053746F72652053CA
:10254000657474696E6773005072656865617420A4
:102550002420436F6E66004F6666004F6E00506F1A
:10256000776572204F7574616765004C4344204362
:102570006F6E747261737400424C546F75636800BF
:1025800050726F6265205A204F6666736574004111
:102590006476616E6365642053657474696E6773F5
:1025A000004D61696E004D37303220542564004D76
:1025B00036303020423020542564004D37303220F0
:1025C0003B2564004D37303120542564004D3730B1
:1025D00032004D373031004D363030204230004D22
:1025E00061696E00436F6E74696E75650050757237
:1025F0006765206D6F726500524553554D45204FFC
:102600005054494F4E533A005052494E5420504175
:10261000555345440020204E6F7A7A6C653A20006D
:102620005061726B696E672E2E2E00000057616933
:102630007420666F720066696C616D656E742063EC
:1026400068616E676500746F2073746172740057FF
:1026500061697420666F720066696C616D656E7485
:1026600020756E6C6F616400004E6F7A7A6C652025
:1026700068656174696E6700506C65617365207789
:102680006169742E2E2E000050726573732062757E
:1026900074746F6E00746F2068656174206E6F7A59
:1026A0007A6C650000496E736572742066696C61AE
:1026B0006D656E7400616E64207072657373206264
:1026C0007574746F6E00746F20636F6E74696E75CD
:1026D00065005761697420666F720066696C616D90
:1026E000656E74206C6F61640000507265737320B6
:1026F000427574746F6E00746F20726573756D65CA
:10270000207072696E7400005761697420666F7280
:10271000207072696E7400746F20726573756D65D8
:102720002E2E2E00005761697420666F7200666954
:102730006C616D656E7420707572676500003E2077
:1027400000256C642E25696D00457874727564658A
:102750006420546F74616C003E20004C6F6E67659E
:102760007374204A6F622054696D65003E200054E6
:102770006F74616C205072696E742054696D6500CD
:10278000436F6D706C65746564003A200050726927
:102790006E7420436F756E74003A2000313530003E
:1027A00035004245443A20415443203130344754A7
:1027B0002D320052756E61776179205761746368BC
:1027C0003A204F4E004D61782054656D70003331D2
:1027D00035004D696E2054656D7000350045313A05
:1027E000204550434F53203130304B00505355005B
:1027F00047656E657269630050726F746F636F6CCA
:1028000000312E3000426175640032353030303096
:1028100000437265616C69747933442052414D50B4
:10282000530042696C696E656172204C6576656C17
:10283000696E670045787472756465727300310063
:1028400074696E796D616368696E657333642E6354
:102850006F6D0053755065522043522D3230003257
:102860003032312D30342D313800322E302E375F5A
:102870004457372E332E31004D61726C696E005013
:1028800072696E7465722053746174730054686564
:10289000726D6973746F727300426F617264204964
:1028A0006E666F005072696E74657220496E666F55
:1028B000004D61696E004D313030300053746F70DF
:1028C000205072696E7400526573756D6520507288
:1028D000696E7400506F776572204F75746167651B
:1028E000004D3139305335350A4732380A473239CD
:1028F0000A4D3430300A4D313034533231350A47C5
:1029000032380A4D313039533231350A4D34323094
:1029100053310A4731583130305931303046353033
:1029200030300A47315A300A4D3530300A4D313196
:102930003720536574205A204F6666736574004DC6
:10294000313036533132380A4D3330334338533215
:1029500031354530550A4D3530300A4D313137204B
:102960005049442054756E6520446F6E65004D31AA
:1029700039305335350A4D313034533231350A4709
:1029800032380A4732394C310A4731205831303019
:102990005931303046353030300A47315A30004DE9
:1029A0003530300A4D3131372053657474696E67A4
:1029B000732053746F726564005072657020666F87
:1029C00072205A2041646A7573740050494420543F
:1029D000756E650053746F72652053657474696E0B
:1029E0006773005365747570004D61696E003F0038
:1029F0004261636B0053746F70005072696E742093
:102A000066726F6D204D65646961004368616E6731
:102A100065204D65646961004D32310041626F751A
:102A200074205072696E746572004368616E6765E8
:102A30002046696C616D656E74004C6576656C69E5
:102A40006E6720546F6F6C7300436F6E66696775B5
:102A5000726174696F6E0054656D70657261747532
:102A60007265004D6F74696F6E00486F7374205308
:102A70007461727400526573756D65205072696E71
:102A800074004E6F204D656469610043616E63653B
:102A90006C204F626A6563740054756E65005374F0
:102AA0006F70205072696E740050617573652050AC
:102AB00072696E7400496E666F2053637265656E4D
:102AC000003F005374617274205072696E74004349
:102AD000616E63656C005072696E740043616E6E66
:102AE0006F7420656E746572207375626469723AE2
:102AF0002000022E2E004D61696E002100486F7487
:102B0000656E6420746F6F20636F6C640042616354
:102B10006B0050726F6365656400536F6674204587
:102B20006E6473746F7073004D6F74696F6E0044E0
:102B3000697361626C6520537465707065727300AF
:102B40004D3834004D34382050726F626520546522
:102B50007374004732384F0A4D34382050313000FA
:102B60004C6576656C20436F726E657273004661CA
:102B7000646520486569676874004F6666004F6E3B
:102B800000426564204C6576656C696E67004C6533
:102B900076656C20426564004732394E00486F6D9F
:102BA00065205A004732385A00486F6D6520590039
:102BB0004732385900486F6D652058004732385801
:102BC000004175746F20486F6D6500473238004DC5
:102BD00061696E0050726568656174202420456EDD
:102BE0006400507265686561742024204265640049
:102BF00054656D706572617475726500436F6F6CBA
:102C0000646F776E005072656865617420240046B9
:102C1000616E205370656564207E00426564004EDD
:102C20006F7A7A6C65004D61696E0050726F6265F3
:102C3000205A204F666673657400416476616E6346
:102C400065204B00466C6F770046616E20537065BF
:102C50006564207E00426564004E6F7A7A6C650080
:102C60005370656564004D61696E00486F6D696EF3
:102C700067204661696C6564006F70656E00545230
:102C800049474745524544003A20007A5F6D696ED6
:102C900000795F6D696E00785F6D696E00526570D6
:102CA0006F7274696E6720656E6473746F702073E1
:102CB00074617475730A0020746F6F206C6F6E6797
:102CC00020657874727573696F6E207072657665B1
:102CD0006E7465640A0020636F6C6420657874729A
:102CE0007573696F6E2070726576656E7465640ABF
:102CF00000486F6D65202573257325732046697222
:102D00007374005761726E696E673A20486F6D691F
:102D10006E672042756D702044697669736F72200A
:102D20003C20310A00020204000000000000000004
:102D300000000000000070430000704300007A4370
:102D4000000000410000004100000040FFFFFF00C4
:102D500000000100000001000080005555550000F2
:102D600000400033333300AAAA2A0049922400000D
:102D7000002000C7711C0099991900D14517005512
:102D80005515003BB1130024491200111111000028
:102D90000010000F0F0F00E3380E0043790D00CC38
:102DA000CC0C00C3300C00E8A20B0064210B00AA7D
:102DB000AA0A00703D0A009DD80900427B090092D2
:102DC000240900DCD30800888808001042080000AD
:102DD000000800F0C10700878707007550070071E1
:102DE0001C07003EEB0600A1BC06006990060066C9
:102DF000660600703E06006118060017F4050074B0
:102E0000D105005BB00500B2900500627205005567
:102E100055050078390500B81E0500050505004E6A
:102E2000EC040087D40400A1BD040090A70400496D
:102E3000920400C17D0400EE690400C756040044FA
:102E40004404005C32040008210400411004000026
:102E50000004003FF00300F8E0030026D20300C3A3
:102E6000C30300CCB503003AA803000A9B03003853
:102E70008E0300C08103009F750300D069030050DA
:102E80005E03001D53030034480300913D030033EB
:102E900033030016290300381F0300971503003081
:102EA0000C0300030303000BFA020049F10200BA0D
:102EB000E802005CE002002DD802002DD00200598B
:102EC000C80200B0C0020031B90200DAB10200AAA3
:102ED000AA0200A0A30200BC9C0200FA9502005CBA
:102EE0008F0200DF88020082820200457C020027F8
:102EF00076020027700200436A02007C640200D060
:102F00005E02003F590200C8530200FFFDFCFAF8C0
:102F1000F6F4F2F0EEECEAE9E7E5E3E1E0DEDCDA34
:102F2000D9D7D5D4D2D0CFCDCBCAC8C7C5C3C2C0DC
:102F3000BFBDBCBAB9B7B6B4B3B2B0AFADACAAA955
:102F4000A8A6A5A4A2A1A09E9D9C9A9998979594A5
:102F50009392908F8E8D8B8A8988878684838281D5
:102F6000807F7E7D7B7A79787776757473727170E5
:102F70006F6E6D6C6B6A69686766656463626160D9
:102F80005F5E5D5C5B5A59585857565554535251C1
:102F900050504F4E4D4C4B4A4A494847464645448F
:102FA00043424241403F3E3E3D3C3B3B3A3938384C
:102FB00037363535343332323130302F2E2E2D2CFA
:102FC0002B2B2A292928272726252524232322219C
:102FD0002120201F1E1E1D1C1C1B1B1A191918182E
:102FE000171616151514131312121111100F0F0EB8
:102FF0000E0D0D0C0C0B0A0A090908080707060636
:1030000005050404030302020100000000704300F0
:1030100000704300007A4300000000000000000040
:1030200000000053657474696E67732053746F7287
:10303000656400454550524F4D20496E6974696181
:103040006C697A65640A003B20003A0A0020204D32
:1030500036303320002055004C0046696C616D65A8
:103060006E74206C6F61642F756E6C6F6164206C80
:10307000656E677468733A0020204D393030204BFC
:10308000004C696E65617220416476616E63653AD9
:103090000020204D3835312058005A2D50726F6273
:1030A00065204F66667365740020204D34313320EF
:1030B0005300506F7765722D4C6F737320526563A8
:1030C0006F766572793A0020204D3235302043000A
:1030D0004C434420436F6E74726173743A00204411
:1030E0000020490020204D3330342050002044007F
:1030F00020490020204D33303120500050494420D9
:1031000073657474696E67733A0020460020480046
:1031100020204D3134352053004D61746572696152
:103120006C2068656174757020706172616D657482
:103130006572733A00204A00202047323920572018
:10314000490020204D3432302053004175746F20E7
:10315000426564204C6576656C696E673A00202094
:103160004D323036205800486F6D65206F666673AB
:1031700065743A0020580020530020204D3230352D
:10318000204200416476616E6365643A20423C6D82
:10319000696E5F7365676D656E745F74696D655F99
:1031A00075733E20533C6D696E5F66656564726140
:1031B00074653E20543C6D696E5F74726176656C17
:1031C0005F66656564726174653E20583C6D617828
:1031D0005F785F6A65726B3E20593C6D61785F79FC
:1031E0005F6A65726B3E205A3C6D61785F7A5F6AF8
:1031F00065726B3E20453C6D61785F655F6A657204
:103200006B3E0020540020520020204D32303420EC
:103210005000416363656C65726174696F6E20284C
:10322000756E6974732F7332293A20503C7072693D
:103230006E745F616363656C3E20523C72657472AC
:103240006163745F616363656C3E20543C747261BA
:1032500076656C5F616363656C3E0020204D3230A3
:10326000312058004D6178696D756D20416363654B
:103270006C65726174696F6E2028756E6974732F46
:103280007332293A0020204D3230332058004D61EE
:1032900078696D756D20666565647261746573200B
:1032A00028756E6974732F73293A005374657073AF
:1032B0002070657220756E69743A002044002020E9
:1032C0004D3230302053002044697361626C656474
:1032D0000A0046696C616D656E742073657474696B
:1032E0006E67733A0020204D3134392043203B2053
:1032F000556E69747320696E2043656C73697573CC
:103300000A0020286D6D290020204732312020201E
:10331000203B20556E69747320696E206D6D00002E
:10332000803B4400803B4400002041000096420066
:1033300000A0420000A0420000C8430000BE42D0EE
:10334000070000D0070000640000004B00000024CC
:10335000F4D43050C38E20C2A24017828B70111259
:103360007A910D816CD90AA861E108C75866076196
:103370005143061E4B5D05C145A7041A41110409BE
:103380003D9803713931034036DB0265339102D435
:10339000305402802E1D02632CEE01752AC501B047
:1033A00028A001102781018F2564012B244B01E007
:1033B000223401AC211F018D200D01801FFC0084EF
:1033C0001EED00971DDF00B81CD200E61BC60020D2
:1033D0001BBC00641AB200B219A8000A19A0006A46
:1033E000189900D117910040178B00B51684003151
:1033F000167E00B31579003A157300C7146F005894
:10340000146A00EE1366008813630025135E00C77C
:10341000125B006C12570015125400C1115100705C
:10342000114F0021114B00D61049008D1047004666
:1034300010440002104200C00F4000800F3E0042C6
:103440000F3C00060F3B00CB0E3800930E37005C9C
:103450000E3500270E3400F30D3200C10D310090FF
:103460000D3000600D2E00320D2D00050D2C00D901
:103470000C2B00AE0C2900850C29005C0C270035B4
:103480000C27000E0C2600E80B2400C40B2400A01F
:103490000B23007D0B23005A0B2100390B21001850
:1034A0000B2000F80A1F00D90A1E00BB0A1E009D4F
:1034B0000A1D00800A1D00630A1C00470A1B002C1D
:1034C0000A1B00110A1A00F7091A00DD091900C4C5
:1034D000091900AB091900920917007B091800634C
:1034E0000917004C09160036091600200916000AB3
:1034F000091500F5081500E0081400CC081400B800
:10350000081400A4081400900813007D0812006B32
:10351000081300580812004608120034081100234E
:103520000811001208110001081100F0071000E056
:10353000071000D0071000C0071000B0070F00A14F
:1035400007100091070E0083070F0074070F006536
:10355000070E0057070E0049070E003B070D002E0F
:10356000070E0020070D0013070D0006070D00F9D8
:10357000060C00ED060D00E0060C00D4060C00C899
:10358000060C00BC060C00B0060C00A4060B00994B
:10359000060C008D060B0082060B0077060B006CF4
:1035A000060B0061060A0057060B004C060A004293
:1035B000060A0038060A002E060A0024060A001A27
:1035C000060A001006090007060A00FD050900F4B6
:1035D000050900EB050900E2050900D9050900D03D
:1035E000050900C7050900BE050900B5050800ADBD
:1035F000050800A50509009C050800940508008C35
:10360000050800840508007C050800740508006CA6
:10361000050700650508005D050700560508004E12
:103620000507004705070040050800380507003179
:103630000507002A050700230507001C05060016DC
:103640000507000F0507000805060002050700FB37
:10365000040600F5040700EE040600E8040600E294
:10366000040700DB040600D5040600CF040600C9E9
:10367000040600C3040600BD040600B7040600B13A
:10368000040500AC040600A6040600A00405009B87
:1036900004060095040500900406008A04050085D0
:1036A000040500800406007A040500750405007016
:1036B0000405006B04050066040500610405005C58
:1036C00004050057040500520405004D0405004898
:1036D000040500430405003E0404003A04050035D7
:1036E000040500300404002C040500270404002312
:1036F0000405001E0404001A040400160405001149
:103700000404000D0404000904050004040400007E
:10371000040400FC030400F8030400F4030400F0B4
:10372000030400EC030400E8030400E4030400E0E5
:10373000030400DC030400D8030400D4030400D015
:10374000030400CC030400C8030300C503030024E2
:10375000F404D9201BC40C5C0E9804C4095F0265F4
:10376000077101F405F900FB04B30048048700C1A8
:103770000369005803550003034500BE023A008464
:1037800002310053022A002902250004022000E42D
:10379000011C00C8011900AF011700980114008432
:1037A000011300710110006101100051010E00436E
:1037B000010D0036010B002B010B0020010B001541
:1037C0000109000C01090003010800FB000800F3D7
:1037D000000800EB000700E4000600DE000600D849
:1037E000000600D2000600CC000500C7000500C29C
:1037F000000500BD000400B9000400B5000400B1DC
:10380000000400AD000400A9000400A5000300A20C
:103810000003009F0004009B000300980003009534
:1038200000020093000300900003008D0002008B53
:10383000000300880002008600020084000300816B
:103840000002007F0002007D0002007B0002007980
:10385000000200770001007600020074000200728E
:10386000000100710002006F0002006D0001006C99
:103870000002006A000100690002006700010066A2
:1038800000010065000100640002006200010061A7
:10389000000100600001005F0002005D0001005CAB
:1038A0000001005B0001005A0001005900010058AE
:1038B00000010057000100560001005500010054AE
:1038C00000010053000000530001005200010051AC
:1038D000000100500001004F0001004E0000004EAA
:1038E0000001004D0001004C0001004B0000004BA6
:1038F0000001004A000100490001004800000048A2
:10390000000100470001004600000046000100459C
:103910000000004500010044000100430000004396
:10392000000100420000004200010041000000418F
:10393000000100400001003F0000003F0001003E88
:103940000000003E0001003D0000003D0001003C81
:103950000000003C0000003C0001003B0000003B78
:103960000001003A0000003A00010039000000396F
:103970000001003800000038000000380001003766
:10398000000000370001003600000036000000365D
:103990000001003500000035000000350001003452
:1039A0000000003400000034000100330000003348
:1039B000000000330001003200000032000000323D
:1039C0000001003100000031000000310001003032
:1039D00000000030000000300001002F0000002F28
:1039E0000000002F0000002F0001002E0000002E1C
:1039F0000000002E0001002D0000002D0000002D11
:103A00000000002D0001002C0000002C0000002C04
:103A10000000002C0001002B0000002B0000002BF8
:103A20000000002B0001002A0000002A0000002AEC
:103A30000000002A000100290000002900000029E0
:103A400000000029000000290001002800000028D3
:103A500000000028000000280000002800010027C6
:103A600000000027000000270000002700000027BA
:103A700000010026000000260000002600000026AD
:103A800000000026000100250000002500000025A0
:103A90000000002500000025000000250001002492
:103AA0000000002400000024000000240000002486
:103AB0000001002300000023000000230000002379
:103AC000000000230000002300000023000100226A
:103AD000000000220000002200000022000000225E
:103AE0000000002200010021000000210000002150
:103AF0000000002100000021000000210000002142
:103B00000001002000000020000000200000002034
:103B10000000002000000020000000200000002025
:103B20000001001F0000001F0000001F0000001F18
:103B30000000001F0000001F0000001F0001001E09
:103B40000000001E0000001E0000001E00000023F8
:103B50002C0000B8220000561800003A0F0000B8F0
:103B6000080000B1040000710200003E01000020C6
:103B7000436F756E7420583A004265640045310009
:103B8000626564002C2073797374656D2073746FA3
:103B90007070656421204865617465725F49443ABC
:103BA000200048656174696E67204661696C6564D0
:103BB0000048656174696E67206661696C656400C0
:103BC0004D3131322053687574646F776E00100088
:103BD000C90210012C014001220170011801B0013D
:103BE0000E01F00104015002FA00B002F0003003AF
:103BF000E600D003DC009004D2007005C800A006E7
:103C0000BE000008B400B009AA00D00BA000600EEE
:103C1000960060118C000015820020197800C01DEC
:103C20006E00A0226400B0275A00902C5000003192
:103C30004600E0343C0010383200903A2800603CE6
:103C40001E00A03D1400803E0A00203F00005448A2
:103C500045524D414C2052554E41574159005468F0
:103C600065726D616C2052756E6177617900457285
:103C7000723A204D415854454D50004D41585445DD
:103C80004D50207472696767657265640045727291
:103C90003A204D494E54454D50004D494E54454DE6
:103CA000502074726967676572656400202F002078
:103CB00042403A0020403A0020573A0020573A004C
:103CC000496E76616C69642065787472756465729A
:103CD0000A007C3C3E5E2B3D3F2F5B5D3B2C2A2245
:103CE0005C0043616E6E6F74206F70656E2073753B
:103CF000626469722000534420496E6974204661F1
:103D0000696C0053442063617264206F6B0A006F1A
:103D100070656E526F6F74206661696C65640A002D
:103D2000766F6C756D652E696E6974206661696C5D
:103D300065640A004E6F20534420636172640A0078
:103D40000A4D3234004D3233202573002E0A006FA5
:103D500070656E206661696C65642C2046696C65CF
:103D60003A200046696C652073656C656374656410
:103D70000A002053697A653A200046696C65206F15
:103D800070656E65643A2000454E4420535542529A
:103D90004F5554494E450A002220706F730022206F
:103DA000706172656E743A2200535542524F5554F9
:103DB000494E452043414C4C207461726765743A0A
:103DC000220053756263616C6C204F766572666C7D
:103DD0006F77004578636565646564206D61782060
:103DE000535542524F5554494E452064657074688E
:103DF0003A002E0A0044656C6574696F6E20666136
:103E0000696C65642C2046696C653A200046696CD3
:103E1000652064656C657465643A00534420707273
:103E2000696E74696E67206279746520004E6F74E4
:103E3000205344207072696E74696E670A004142B3
:103E40005300504C41002F6175746F25632E67003D
:103E500057726974696E6720746F2066696C653A81
:103E60002000667265736800646F696E6700206683
:103E7000696C653A20004E6F77200002FD5555555C
:103E800055555FFFFFFFFFFFFFFFFFFFFE00000034
:103E900000003FFFFFFFFFFFFFFFFFFFFD000007E8
:103EA000FFFFFFFFFFFFFFFFFFFFFFFFFE07C00554
:103EB00055555555555FFFFFFFFFFFFFFC0A2006D4
:103EC00000000000003FFFFFFFFFFFFFFE14100592
:103ED000000007FFFFFFFFFFFFFFFFFFFC280806B2
:103EE00007C00555555555555FFFFFFFFE540404A7
:103EF0000A200600000000003FFFFFFFFC600406F0
:103F0000141005000007FFFFFFFFFFFFFE50040431
:103F100028080607C00555555555555FFC60040631
:103F20005404040A200600000000003FFE54041C54
:103F300060040614100500000000001FFC28082E75
:103F400050040428080607C00001F03FFE14105476
:103F50006004065404040A200002081FFC0A2066BC
:103F600054041C60040614100005043FFE07C054EE
:103F700028082E5004042808000A021FFC00002E06
:103F800014105460040654040015013FFE00001C88
:103F90000A206654041C60040018011FFC0000067F
:103FA00007C05428082E50040014013FFE000004EE
:103FB00000002E14105460040018011FFCFFFFFEC7
:103FC00000001C0A206654041C15013FFED5555400
:103FD00000000607C05428082A0A021FFC84104665
:103FE00000000400002E14105105043FFEC41044CC
:103FF000FFFFFE00001C0A206102881FFC8410469F
:10400000D5555400000607C05101F03FFE8410440E
:1040100084104600000400002A00001FFCC4104663
:10402000C41044FFFFFE00001C00003FFE8410444B
:10403000841046D5555400000000001FFCD555568D
:1040400084104484104600000000003FFCFFFFFC89
:10405000C41046C41044FFFFFFFFFF9FFE00000690
:10406000841044841046D555555555BFFD555554BB
:10407000D5555684104484104104109FFFFFFFFC67
:10408000FFFFFCC41046C410410411BFFFFFFFFE38
:1040900000000684104484104104109FFFFFFFFDC0
:1040A000555554D5555684104104109FFFFFFFFF0E
:1040B000FFFFFCFFFFFCC410410411BFFFFFFFFF27
:1040C000FFFFFE00000684104104109FFFFFFFFF6A
:1040D000FFFFFD555554D555555555BFFFFFFFFF03
:1040E000FFFFFFFFFFFCFFFFFFFFFF9FFFFFFFFF43
:1040F000FFFFFFFFFFFE00000000003FFFFFFFFF8C
:10410000FFFFFFFFFFFD55555555555FFFFFFFFFB3
:10411000FFFFFFFFFFFFFFFFFFFFFFFFFFFFFFFFAF
:10412000FFFFFFFFFFFFFFFFFFFFFFFFFFFFFFFF9F
:10413000FFFFFFFFFFFFFFFFFFFFFFFFFFFFFFFF8F
:10414000FFFFFFFFFFFFFFFFFFFFFFFFE02EFB7DF5
:10415000FBFBCFC1DFBB3EC0E1FE3C1FFDEE7B3968
:10416000F9F3CF9EDFBB3EDFDEFCDDE7FDEE3BBBC0
:10417000F9EBD7BF5FBB5EDFDEFDEDF7FDEEBBD336
:10418000FAEBB73FDFBB4EDFDFFFCDF3FDEEDBC762
:10419000FAEBBB7FC03B6EC0E3FF1DF3FDEECBEF40
:1041A000FADBBB7FDFBB66DFF8FFCDF3FDEEEBEFA5
:1041B000FB5B033F5FBB76DFFE7FEDF3FDEEF3EFCE
:1041C000FB5B79BEDFBB7ADFDE7DEDF7FDEEF3EF63
:1041D000FBBAFD9EDFBB7CDFDEFDCDE7FDEEFBEF36
:1041E000FBBAFDC1DFBB7EC0E0FE1C1F6D61726CBF
:1041F000696E66772E6F726700322E302E375F44FD
:1042000057372E332E31001FFFFFFFFFFFFF6000E7
:1042100000000001FF400000000000FF80000000DF
:1042200000007F83CF00000C303F87FF80000C3000
:104230001F867980000C000F8C30C7838C30E78C90
:1042400030CFC7CC31F38C30DCECEC33B98C30D8C8
:104250006C6C33198C30D06C0C33198C30D86C0CDE
:1042600033198C30DC6C0E3B198C30CF7C079F19D6
:104270008C30C77C038F19400000000000026000F2
:1042800000000000061FFFFFFFFFFFF870012C0178
:1042900090012701B0012201C0011D01F0011801A8
:1042A0001002130130020E016002090190020401A4
:1042B000C002FF000003FA004003F5008003F00095
:1042C000D003EB002004E6007004E100E004DC0011
:1042D0004005D700C005D2004006CD00D006C8007A
:1042E0008007C3003008BE00F008B900C009B40060
:1042F000B00AAF00B00BAA00D00CA500000EA000C1
:10430000500F9B00C01096005012910000148C00BA
:10431000C0158700B0178200B0197D00D01B78004F
:10432000001E730040206E0090226900F02464009B
:1043300040275F0090295A00E02B5500102E5000B6
:1043400020304B0010324600E033410090353C00F5
:104350001037370070383200A0392D00B03A2800ED
:10436000A03B2300603C1E00103D1900903D14004E
:10437000103E0F00703E0A00C03E0500003F0000E6
:10438000403FFBFF803FF6FFC03FF1FF2020506C15
:10439000616E6E65724275666665724279746573A8
:1043A0003A20002046726565204D656D6F72793A3E
:1043B0002000436F6D70696C65643A204170722013
:1043C000323920323032310A00204C61737420556A
:1043D0007064617465643A20323032312D30342D8E
:1043E0003138207C20417574686F723A2054696EB0
:1043F000794D616368696E657333440A00322E300B
:104400002E375F4457372E332E310A004D61726CC0
:10441000696E0020536F6674776172652052657310
:1044200065740A00205761746368646F6720526581
:104430007365740A002042726F776E206F75742066
:1044400052657365740A002045787465726E616CFC
:104450002052657365740A00506F77657255700A53
:104460000073746172740A004739310A47315A3552
:104470000A4739300A4D38340A4D31303453300A46
:104480004D3134305330004D31303031006572726F
:104490006F722077726974696E6720746F20666925
:1044A0006C650A00446F6E6520736176696E6720E3
:1044B00066696C652E0A004D323900456E6473746E
:1044C0006F7073002553202563202563202563200A
:1044D000256300205A3A0020593A0020583A0065D6
:1044E0006E6473746F7073206869743A2000000002
:1044F0000A0B02090C0D0E0807030401000000005E
:1045000000000000000000000000000000000000AB
:104510000000000000000000000012111000000068
:10452000000000000000000000000000000000008B
:1045300000000000004D6F76652025736D6D004D05
:104540006F766520302E316D6D004D6F76652031B0
:104550006D6D004D6F76652031306D6D004D6F765D
:1045600065204178697300457874727564657200DE
:104570004D6F7665205A004D6F76652059004D6F5E
:104580007665205800423E3E3E4368616E67652076
:1045900046696C616D656E7400556E6C6F61642068
:1045A00046696C616D656E74004C6F61642046698C
:1045B0006C616D656E74005072656865617420434E
:1045C0007573746F6D0050726568656174202400A6
:1045D0004261636B0050726F62696E672046616969
:1045E0006C656400205A3A200020593A2000426548
:1045F0006420583A200070726F6D70745F007368A9
:104600006F7700627574746F6E00626567696E0023
:1046100050757267654D6F726500506175736564A2
:1046200000436F6E74696E7565004C6F616420465F
:10463000696C616D656E74205400496E73657274A7
:104640002066696C616D656E7420616E64207365AF
:104650006E64204D3130380A00220A00556E6B6EB0
:104660006F776E20636F6D6D616E643A202200205B
:1046700042002050006F6B0053755065522043522A
:104680002D32302052656164792E005072696E744B
:10469000696E672E2E2E005072696E7420506175FF
:1046A00073656400204500205A00205900204D39D0
:1046B0003220580020453A00205A3A0020593A004A
:1046C000583A0020746F6F206C6F6E6720657874A5
:1046D000727573696F6E2070726576656E7465644D
:1046E0000A0020636F6C6420657874727573696F5B
:1046F0006E2070726576656E7465640A005265732B
:10470000656E643A20006E6F7469666963617469EE
:104710006F6E200000002200250028002B002E00D4
:104720003100340002010000050108010B01000006
:104730002100240027002A002D0030003300010151
:104740000000040107010A01050505050705080821
:104750000808020202020A0A08080404040401010B
:104760000101010101010303030303030303040720
:1047700007070C0C0C0C0C0C0C0C020202020606B7
:104780000606060606060B0B0B0B0B0B0B0B0102AA
:104790001020200808102040102040800201020153
:1047A000080402010102040810204080804020100B
:1047B0000804020180040201804020100804020164
:1047C00008040201010204081020408001020408CC
:1047D00010204080AE00F40011241FBECFEFD1E2C4
:1047E000DEBFCDBF00E00CBF13E0A0E0B2E0E8E91F
:1047F000FFEE02E00BBF02C007900D92AC39B1078B
:10480000D9F729E1ACE9B3E001C01D92A537B207A1
:10481000E1F713E2CBEED3E200E006C021970109F5
:10482000802FFE010F942974CA3ED10780E008074B
:10483000A9F70F945B620D94BA770C940000FC0109
:1048400084910895FC018081089590E080E00895AE
:10485000CF93DF93DB01F9019C919130C1F094304B
:1048600080F094509C938830D1F48081918100979E
:1048700071F0019791838083480F591FEA011882D4
:1048800006C08C3539F49C5F9C93943041F4DF91E1
:10489000CF9108958B3339F781E08C93F8CF208145
:1048A0003181B9016F5F7F4F71836083420F531F66
:1048B000EA018883808191818F3591056CF7E7CF7C
:1048C0000F931F9381E00091661710916717209155
:1048D0006817309169174091621750916317609182
:1048E000641770916517041715072607370708F432
:1048F00080E01F910F91089590E080E00895282FA7
:104900009091DD08833021F495FD0FC094FD0FC018
:10491000892F90E0B0E0A0E004C0B695A7959795E8
:1049200087952A95D2F78170089581E0089580E0F7
:104930000895CF92DF92EF92FF92CF93DF93EC0135
:10494000CC80DD80EE80FF8027E137EB41ED58EB36
:10495000C701B6010F94927687FD23C027E030E0AF
:1049600040E753E4C701B6010F94406D1816CCF030
:10497000C880D980EA80FB8027E137EB41ED58EB16
:10498000C701B6010F94927687FD0BC0C1E027E006
:1049900030E040E753E4C701B6010F94406D1816AC
:1049A0000CF4C0E08C2FDF91CF91FF90EF90DF905F
:1049B000CF9008952F923F924F925F926F927F9285
:1049C0008F929F92AF92BF92CF92DF92EF92FF921F
:1049D0000F931F93CF93DF93CDB7DEB72E970FB60C
:1049E000F894DEBF0FBECDBFE82ED62E042F122FB7
:1049F000282F30E03C872B87462F50E05A87498785
:104A000065E0F62EF29EC001F39E900D11249E8764
:104A10008D87FA01E80FF91FEE0FFF1FEE0FFF1F42
:104A2000E35EF94F60817181828193819B01AC01CA
:104A30000F942477882309F434C1E00E612F6D0DA3
:104A4000FE9CF0011124A985BA85AE0FBF1FAA0FE5
:104A5000BB1FAA0FBB1FA35EB94FAC901196BC90B1
:104A600011971296CC9012971396DC90E00EFE9C54
:104A7000A0011124A985BA85A40FB51FAA0FBB1FD9
:104A8000AA0FBB1FA35EB94FEC901196FC90119733
:104A900012960C91129713969C90862F90E0AD85FC
:104AA000BE85A80FB91FAA0FBB1FAA0FBB1FA35E0D
:104AB000B94F8C9011967C90119712966C9012972A
:104AC00013965C90610F70E0AD85BE85A60FB71F91
:104AD000AA0FBB1FAA0FBB1FA35EB94F4C90119624
:104AE0003C90119712961C91129713962C90E80FF8
:104AF000F91FEE0FFF1FEE0FFF1FE35EF94FB081AE
:104B0000B98321812A8332813B8383818C83FA019B
:104B1000E60FF71FEE0FFF1FEE0FFF1FE35EF94FCB
:104B200090819D83A181AE83B281BF832381288739
:104B30009701402F592DB701802F992D0F9424777D
:104B4000882321F0E12CF12C00E0912C9501A601A5
:104B5000B501C6010F942477882319F05701C02EA0
:104B6000D92C242D332D412F522D642D732D812FBF
:104B7000922D0F942477882321F0412C312C10E0C2
:104B8000212C282D372D462D552D682D772D862D3E
:104B9000952D0F942477882321F0842C732C612E7B
:104BA000522C2D813E814F8158856D817E818F8170
:104BB00098850F942477882321F01D821E821F82FE
:104BC000188629813A814B815C8169817A818B8148
:104BD0009C810F942477882341F03D8139834E8155
:104BE0004A835F815B8388858C8385E0EB85FC85C8
:104BF0008E9FD0018F9FB00D112429853A85A20F79
:104C0000B31FAA0FBB1FAA0FBB1FA35EB94FBA8762
:104C1000A9879501A601B501C6010F9432749701C9
:104C2000402F592D0F9431746B017C01282D372DA5
:104C3000462D552D682D772D862D952D0F94327488
:104C4000242D332D412F522D0F9431749B01AC0133
:104C5000C701B6010F9432746B017C0129813A813E
:104C60004B815C8169817A818B819C810F94327444
:104C70002D813E814F8158850F9431749B01AC0189
:104C8000C701B6010F94327420E030E040E450E4F4
:104C90000F942C75A985BA856D937D938D939C9304
:104CA00013972E960FB6F894DEBF0FBECDBFDF91DF
:104CB000CF911F910F91FF90EF90DF90CF90BF9019
:104CC000AF909F908F907F906F905F904F903F90AC
:104CD0002F900895129A0895269A2E9A0895EF9289
:104CE000FF920F931F93CF93DF93EC018B017A0117
:104CF0008A859B858617970731F0888199810F9463
:104D0000845A1B870A87B701888199810F94AE4B1B
:104D10002E813F81820F932F911D9F838E8390E080
:104D200080E0DF91CF911F910F91FF90EF90089558
:104D30009F92AF92BF92CF92DF92EF92FF920F932A
:104D40001F93CF93DF93EC018B01942EA52E8A85C0
:104D50009B858617970731F0888199810F94845A33
:104D60001B870A8788859985019649F5BC800A8149
:104D70008E81080FC880D980D6015596ED91FC919F
:104D8000C6011995B80EE92CFA2C10E0F701219113
:104D90007F01211127C08E819F81810F911D9F83EB
:104DA0008E8390E080E0DF91CF911F910F91FF9073
:104DB000EF90DF90CF90BF90AF909F9008950E81BD
:104DC0001F81692D7A2D888199810F94AE4B800FB8
:104DD000912F911D288539852817390738F681E0EC
:104DE00090E0E1CF4B2D602FC6010F94DC5A080FE5
:104DF000180FCCCFDF92EF92FF920F931F93CF93B8
:104E0000DF93EC01D62E1CAD0BAD7C0184E0E80EE7
:104E1000F11CE98DFA8DC7011995412F480F2D2DF1
:104E2000602FC7010F94DC5A9BAD890F8BAF81E0D7
:104E300090E0DF91CF911F910F91FF90EF90DF9065
:104E40000895AF92BF92DF92EF92FF920F931F935C
:104E5000CF93DF938C01EB01D42E79018FE04817BB
:104E600009F486C0A5E14A17B1F1BAE04B130EC0B0
:104E7000EC81FD8130E020E042E061E0C80119955D
:104E800047EA5AE1BE01C8010F94875B0A80DB81C3
:104E9000C02DF2E3DF1609F4E2C0FD1508F491C05D
:104EA00085E1D81609F4E0C0A7E1DA1609F4EFC0ED
:104EB000B4E1DB127BC0EE81FF818D8190E0880F31
:104EC000991F8E0F9F1F11928E179F07E1F7CE013A
:104ED0000F94A4586BC0AA80BB8042E95AE1C80174
:104EE0000F94875BF5014481440F406BBE01C801FC
:104EF0000F946F5B41E0BE01C8010F94775BD50151
:104F000016962D913C911797EC81FD8115964C9149
:104F100066E0C801199540E0BE01C8010F947F5BAF
:104F200042E95AE1BE01C8010F94875BF501448153
:104F3000440F4F5F406BBE01C8010F946F5B41E0AF
:104F4000BE01C8010F94775BD50115964C9115975A
:104F500016962D913C91240F311DEC81FD8166E068
:104F6000C801199540E0BE01C8010F947F5B8ECF48
:104F700041E0C8010F947F5B40E0BE01C8010F947F
:104F8000775B41E8BE01C8010F946F5BF701408178
:104F900050E05595479555954795BE01C8010F942A
:104FA0006F5B40E0BE01C8010F947F5B81E0DF9141
:104FB000CF911F910F91FF90EF90DF90BF90AF9036
:104FC0000895E6E4DE1609F471C0F7E4DF1609F48B
:104FD00071C08BE3D812EACFD70111969C9111973B
:104FE00013968C9138E0390F813031F0833011F015
:104FF000392F02C0392F985021E04B81491708F40E
:1050000020E041E0391708F040E091E05A8135177F
:1050100008F490E0322F342B932311F4242331F23F
:10502000F701128100E0D12C843048F490E0FC01BB
:10503000E054FD4FD08084549D4FDC010C9117FF4C
:1050400004C0B701CE010F94AB58F70180818D0DDC
:1050500080838181800F8183110F89F7A7CFB701EA
:10506000CE010F94AB58A2CFCE010F948E58882357
:1050700009F49DCFEE81FF818D8190E0880F991F0B
:105080008E0F9F1F11928E179F07E1F78FCFD701C9
:105090001C928A8111968C9311978D818150129662
:1050A0008C9312978B8113968C9380CF8D81F7010F
:1050B00080837CCF8981D7018C9378CFAB01BC01F1
:1050C000409366175093671760936817709369173A
:1050D0008FEC98E10C947FE580932F028032B8F535
:1050E00090916305891724F091E0980F90936305E0
:1050F00040915F0550916005609161057091620576
:10510000082E04C076956795579547950A94D2F76F
:1051100041704093DA1087FD1DC0282F082E000C27
:10512000330B3F938F9382E49AE09F938F9382E5B2
:105130009AE09F938F931F920E9411CA8DB79EB7DA
:1051400007960FB6F8949EBF0FBE8DBF08951092BC
:10515000DA10E1CF0D9477470F931F93CF93DF932E
:1051600000D01F92CDB7DEB79C0108EA18E090E1AD
:10517000E3EDF9E0D80101900D929A95E1F7F9017C
:105180002081318142815381F8016085718582855A
:1051900093850F943274F8016087718782879387B3
:1051A00080E090E0A0EAB0E489839A83AB83BC837B
:1051B000CE0101960F94FB180F900F900F900F9057
:1051C000DF91CF911F910F9108952F923F924F92AF
:1051D0005F926F927F928F929F92AF92BF92CF9287
:1051E000DF92EF92FF921F93CF93DF93CDB7DEB79D
:1051F0002C970FB6F894DEBF0FBECDBF7A01190110
:10520000DC012D913D914D915C912D833E834F8327
:105210005887FB0140805180628073808090D30961
:105220009090D409A090D509B090D609A501940119
:105230006D817E818F8198850F94406D81110EC0A4
:1052400011E0A30192016091D7097091D809809172
:10525000D9099091DA090F94406D811110E0D101C4
:105260002D913D914D915C9129873A874B875C87C1
:10527000F701C080D180E280F38020911302309149
:1052800014024091150250911602C701B6010F9405
:10529000406D882309F44EC0C0921302D0921402CC
:1052A000E0921502F09216028091DF099091E009D8
:1052B000A091E109B091E2094091D7095091D80934
:1052C0006091D9097091DA098092A8089092A90892
:1052D000A092AA08B092AB084093AC085093AD08D6
:1052E0006093AE087093AF08C092B008D092B10836
:1052F000E092B208F092B3088093B4089093B50896
:10530000A093B608B093B70820E030E040E05FE338
:10531000609108117091091180910A1190910B11FF
:105320000F94A66D69837A838B839C83CE0101964B
:105330000F94FB182D813E814F8158852093A8083A
:105340003093A9084093AA085093AB084092AC0848
:105350005092AD086092AE087092AF08D1012D91C5
:105360003D914D915C916091B4087091B508809128
:10537000B6089091B7080F9432746093B408709394
:10538000B5088093B6089093B70811112FC020E09C
:1053900030E0A90169857A858B859C850F94406DE5
:1053A000811133C060E070E088EC92E469837A8315
:1053B0008B839C83CE0101960F94FB182C960FB61D
:1053C000F894DEBF0FBECDBFDF91CF911F91FF904C
:1053D000EF90DF90CF90BF90AF909F908F907F9095
:1053E0006F905F904F903F902F9008952AEF3EE787
:1053F0004AE25FE360910C1170910D1180910E11E2
:1054000090910F110F94A66DD1CF60E070E080EA0B
:1054100091E4CCCFCF93DF9300D01F92CDB7DEB70E
:1054200080E090E0A0EAB0E489839A83AB83BC83F8
:1054300061E0CE0101960F9405110F900F900F902F
:105440000F90DF91CF9108958091220590912305CF
:10545000009731F04AE050E070E060E00D945B6B43
:1054600060E070E0CB0108958091E70982FF0BC0F6
:1054700063E686E29BE00E942CCA0F9498520E9439
:1054800026D181E0089580E00895809122059091D1
:105490002305009731F04AE050E070E060E00D94A1
:1054A0002D6A60E070E0CB0108950E94452A97FDC7
:1054B0000CC00E94452A6F3F71058105910509F0D6
:1054C00034F40E94452A862F089580E008958FEFD6
:1054D00008958091220590912305892B41F00E9427
:1054E000552A91E0811101C090E0892F089591E043
:1054F000FCCFCF92DF92EF92FF920F931F93CF9347
:10550000DF936B017A01EC01C255DB4F28813CE04F
:10551000389F8001399F100D112427FF24C0FB0103
:105520001182108288818F5F888388819801280F7B
:10553000311D87FD3A95C9012091D316F601281730
:10554000190629F024F088818C300CF43CC080814D
:105550009181049680349C4908F475C0F6018081DD
:105560009181049672C088819801280F311D87FDB2
:105570003A95C9012091D3162817190699F294F289
:105580008881A801480F511D87FD5A95FA01EE0F39
:10559000FF1FE40FF51FE557F94E808187FFC2CF4B
:1055A0008881F801E80FF11D87FDFA95CF01EE0F14
:1055B000FF1FE80FF91FE557F94E808160E08F77F4
:1055C0000F943D50AFCF808191812881A801420F77
:1055D000511D27FD5A959A01FA01EE0FFF1FE20FA8
:1055E000F31FE557F94E21813281820F931FF70196
:1055F0009183808388819801280F311D87FD3A951A
:10560000F901EE0FFF1FE20FF31FE557F94E8081FE
:1056100087FF20C08881080F111D87FD1A95F801AA
:10562000EE0FFF1FE00FF11FE557F94E808161E09B
:105630008F77DF91CF911F910F91FF90EF90DF90C7
:10564000CF900D943D5080E49CE9F70191838083D5
:105650008FEF8883DF91CF911F910F91FF90EF9093
:10566000DF90CF900895AF92BF92CF92DF92EF92EA
:10567000FF920F931F93CF93DF93EC015B018A019D
:10568000FB01199587FD16C0C82ED12CF12CE12CF9
:105690002196F801C082D182E282F382CE01DF91AD
:1056A000CF911F910F91FF90EF90DF90CF90BF901F
:1056B000AF900895982F907E903CA9F48F7190E060
:1056C000B0E0A0E06C017D0156E0CC0CDD1CEE1CCE
:1056D000FF1C5A95D1F7CE010196F50119958F73EC
:1056E000C82A2296D6CF982F907F903E11F58F70C2
:1056F00090E0B0E0A0E06C017D0136E0CC0CDD1C58
:10570000EE1CFF1C3A95D1F7CE010196F5011995D3
:105710008F73C82A46E0CC0CDD1CEE1CFF1C4A959A
:10572000D1F7CE010296F50119958F73C82A2396F9
:10573000B0CF982F987F903F79F5877090E0B0E0D8
:10574000A0E06C017D0186E0CC0CDD1CEE1CFF1C92
:105750008A95D1F7CE010196F50119958F73C82A64
:1057600096E0CC0CDD1CEE1CFF1C9A95D1F7CE0107
:105770000296F50119958F73C82A26E0CC0CDD1C22
:10578000EE1CFF1C2A95D1F7CE010396F501199561
:105790008F73C82A24967DCF982F907C903841F43F
:1057A000807C803869F42196CE01F5011995F8CFF7
:1057B0008E7F8D3F28F02196CE01F5011995F8CF07
:1057C000C12CD12C760165CF9CE0899F802D1124BE
:1057D00091E0980F909364052CE0280F2093A20885
:1057E00030E02E5F3F4F409158174217130619F0D3
:1057F00014F080E0089520915A179217D0F766238D
:1058000041F08E5F0F949E598091A2088E5F0F9495
:105810009E598091A20890915817891750F32091B2
:105820005A1790916405291720F310925B17809303
:105830005C1781E0089520915605022E000C330B71
:105840008217130641F08093560564ED7AE184E2F5
:1058500097E10D94845A08951F93CF93DF931F927D
:10586000CDB7DEB78F3F910519F014F08FEF90E0C0
:105870008837910514F488E790E090935A0280935A
:105880005902182F80915D17811105C081E0809326
:105890005D170F94C55860912617709127171983CB
:1058A0009E012F5F3F4F4FE084E297E10F94C15874
:1058B0000F90DF91CF911F910895CF93809157055D
:1058C00081114FC010925B1710925C1710925D17F8
:1058D000109229171092281710922B1710922A173E
:1058E00010922D1781E080932C1782E280932E175F
:1058F0001092331710923217E7E4F7E125E537E10C
:105900008FEF81932E173F07E1F7C1E0C093441753
:1059100020EE30E030933A1720933917C0933B17AD
:1059200010923C1710923D1790E490933E171092FE
:105930003F172CE332E0309356172093551722E29D
:1059400032E0309327172093261799E19093491757
:105950009BE190934817809347170F94C558C093C5
:1059600057058091590290915A020E942C2C81E097
:105970008093580582E99AE190933D1680933C16F6
:1059800010923F1610923E16CF910895CF92DF925B
:10599000EF92FF920F931F93CF93DF93CDB7DEB7B4
:1059A0002C970FB6F894DEBF0FBECDBF6F3F7105C9
:1059B0008105910509F0D0F480E297E10E94FA2672
:1059C000E0912817F09129173196849190E02C9658
:1059D0000FB6F894DEBF0FBECDBFDF91CF911F9100
:1059E0000F91FF90EF90DF90CF900895F0905B17AC
:1059F000E0905C172091580521110FC042E75AE151
:105A00006E2D8F2D0F94485B90E080E0F80EF092A1
:105A10005B17E0925C179927DACFC0902817D090D7
:105A2000291724E237E13A8329832F2D30E03C8384
:105A30002B832E2D30E03E832D8318861F822FEF7F
:105A40003FEF3A8729871C861B8608E916E29E01EC
:105A50002F5F3F4FAB01BC01C6010F948930B601E7
:105A600084E297E10F94845A8F819885CFCFCF93AA
:105A7000DF93FC0125AD211104C021E025AF0F9477
:105A8000C558C0912617D0912717E0915517F0916E
:105A9000561782E01995E0915517F091561781E05D
:105AA000199530E020E044E1BE0184E297E10F94D3
:105AB000C15827E537E147E1BE0184E297E10F9441
:105AC000C158E0915517F091561780E0DF91CF91C2
:105AD0001994CF92DF92EF92FF920F931F93CF937F
:105AE000DF93CDB7DEB72C970FB6F894DEBF0FBEAD
:105AF000CDBFF0905B17E0905C1720915805211105
:105B00001DC042E55AE16E2D8F2D0F94485B90E049
:105B100080E0F80EF0925B17E0925C1799272C96C4
:105B20000FB6F894DEBF0FBECDBFDF91CF911F91AE
:105B30000F91FF90EF90DF90CF900895C0902817BD
:105B4000D090291724E237E13A8329832F2D30E0C2
:105B50003C832B832E2D30E03E832D8318861F82BD
:105B60007A8769871C861B8608E916E29E012F5FEB
:105B70003F4F4FE154E2BC01C6010F944D31B601D5
:105B800084E297E10F94845A8F819885C2CF6FEF9A
:105B90007FEF0C94692DCF92DF92EF92FF920F93DB
:105BA0001F93CF93DF93CDB7DEB72C970FB6F89442
:105BB000DEBF0FBECDBFF0905B17E0905C17209169
:105BC000580521111DC042E35AE16E2D8F2D0F940F
:105BD000485B90E080E0F80EF0925B17E0925C1773
:105BE00099272C960FB6F894DEBF0FBECDBFDF917C
:105BF000CF911F910F91FF90EF90DF90CF9008957C
:105C0000C0902817D090291724E237E13A832983DE
:105C10002F2D30E03C832B832E2D30E03E832D83CF
:105C200018861F827A8769871C861B8608E916E218
:105C30009E012F5F3F4F42E254E2BC01C6010F9428
:105C40004D31B60184E297E10F94845A8F81988593
:105C5000C2CFBF92CF92DF92EF92FF920F931F932A
:105C6000CF93DF938B01F42EE90141FB662760F9A6
:105C70000E94E42B882309F45AC0B12C01151105A8
:105C800021F0C8010E94F7D1B82EE12C209721F015
:105C9000CE010E94E2D3E82E80E8C82ED12CF0FE7F
:105CA0001EC085E190E08B199109B7FC93958E1980
:105CB0009109E7FC939597FD019695958795F82EA8
:105CC00030E8C32ED12CFA94F7FC09C060E270E0F2
:105CD00080E090E00E94C62CC81AD90AF4CFBB20FD
:105CE00099F0C60166E070E00F940174262F409190
:105CF000A4085091A5086091A308C8010E9437D15B
:105D000096E0899F60011124EE2031F0B601CE01AA
:105D10000E94CB2DC81AD90A87E0C816D10438F0E2
:105D200060E270E080E090E00E94C62CF3CFDF914B
:105D3000CF911F910F91FF90EF90DF90CF90BF9088
:105D400008956FEF7FEF0C94CB2DAF92BF92CF925F
:105D5000DF92EF92FF920F931F93CF93DF935C013B
:105D60006B010E94F7D1E82EC6010E94E2D3F12C0C
:105D700003E110E0081B1109C5E20E151F050CF424
:105D8000CFE18C2F90E09C012E5F3F4F4091581740
:105D90004217130609F0CCF5099720915A172817D6
:105DA00019069CF14091A4085091A5086091A308A0
:105DB00010925B17C0935C1725E1C5010E9437D193
:105DC000D1E0C114D104B1F06AE370E080E090E06A
:105DD0000E94C62C0E151F05D4F4C45F809158177D
:105DE000C81740F020915A174C2F4950550B2417D3
:105DF00015067CF4DF91CF911F910F91FF90EF90EA
:105E0000DF90CF90BF90AF900895D0E0DACFDD2340
:105E100089F3802F880F080F000F00935B17C09342
:105E20005C1760E270E080E090E00E94C62CC60142
:105E3000DF91CF911F910F91FF90EF90DF90CF9066
:105E4000BF90AF900C94A12E8F929F92AF92BF9271
:105E5000CF92DF92EF92FF920F931F93CF93DF9336
:105E6000CDB7DEB72C970FB6F894DEBF0FBECDBF0F
:105E7000982F862F5A017901D02E692F0E94E42B8A
:105E8000882309F489C0C701002391F10E94F7D14A
:105E9000C82E80902817909029178091580581115D
:105EA00045C01FEF23E12C194091A4085091A5088B
:105EB0006091A308C5010E9437D1CC2009F46CC0C1
:105EC000B6E08B9F500111246AE370E080E090E01F
:105ED0000E94C62C57E0A516B10408F444C060E245
:105EE00070E080E090E00E94C62CA81AB90AF2CFB8
:105EF0000E94E2D3C82E8090281790902917809195
:105F00005805882371F2FE0133968AE0DF011D9265
:105F10008A95E9F784E297E19A8389830FE616E28E
:105F20009E012F5F3F4F42E254E212C0FE013396C2
:105F30008AE0DF011D928A95E9F784E297E19A836E
:105F400089830FE616E29E012F5F3F4F4FE154E237
:105F5000B701C4010F944D31B40184E297E10F946D
:105F6000845A1F819FCF4091A208212F30E0A6E0E4
:105F7000CA9EC00111242E5F3F4F281739070CF429
:105F80009C0180E8821B80935B1740935C17C701DC
:105F9000DD20A9F00E94C72D2C960FB6F894DEBF25
:105FA0000FBECDBFDF91CF911F910F91FF90EF906A
:105FB000DF90CF90BF90AF909F908F9008950E94F8
:105FC000A12EEACFE0E2F7E183AF64AFCA010C94FF
:105FD000A12E2F923F924F925F926F927F928F925B
:105FE0009F92AF92BF92CF92DF92EF92FF920F9368
:105FF0001F93CF93DF93D62FC72FFC018080918012
:10600000A280B380C501B40120E831E541E050E051
:106010000F948473C9016DE671E00F9401746B01F4
:106020007C01C501B40120E13EE040E050E00F9466
:106030008473CA01B90128E130E040E050E00F94D8
:106040008473362E272E062F172F8CE3482E512CC3
:10605000612C712CC501B401A30192010F948473CA
:10606000B62EA72ECA01B901A30192010F94847321
:10607000CB01C114D10479F1AF92BF927F936F939A
:106080002F923F92FF92EF92DF92CF9280E998E1B8
:106090009F938F93CF93DF930F94D76C8DB79EB759
:1060A0000E960FB6F8949EBF0FBE8DBF8D2F9C2FFE
:1060B000DF91CF911F910F91FF90EF90DF90CF90E4
:1060C000BF90AF909F908F907F906F905F904F9018
:1060D0003F902F900895E114F104C9F0AF92BF9260
:1060E0007F936F932F923F92FF92EF9280E898E117
:1060F0009F938F93CF93DF930F94D76CEDB7FEB739
:106100003C960FB6F894FEBF0FBEEDBFCFCF012B6C
:10611000B9F0AF92BF927F936F932F923F9284E733
:1061200098E19F938F93CF93DF930F94D76C8DB7A4
:106130009EB70A960FB6F8949EBF0FBE8DBFB6CF1E
:10614000892BA9F0AF92BF927F936F938CE698E171
:106150009F938F93CF93DF930F94D76CEDB7FEB7D8
:1061600038960FB6F894FEBF0FBEEDBF9FCFAF922B
:10617000BF9288E698E19F938F93CF93DF930F941C
:10618000D76C0F900F900F900F900F900F908ECFB5
:106190008F929F92AF92BF92CF92DF92EF92FF9237
:1061A0000F931F93CF93DF931092550510925405D0
:1061B0002FE320934F0510924E0510924D0510923B
:1061C0004C051092500510925105109252051092F4
:1061D00053059C01F90190812F5F3F4F9032D1F31D
:1061E0009E34C9F4818190ED980F9A3020F08D3261
:1061F00011F08B3281F432969F012F5F3F4F8081E7
:1062000080538A3008F47BC09F012F5F3F4F80810D
:10621000803209F476C0F093C608E093C5088F0178
:106220000F5F1F4FC0816AE270E0C8010F94807752
:10623000009731F0FC01319780818032E1F31182C7
:10624000CD3429F0C43519F0C73409F04BC0F8013A
:1062500080810F5F1F4F8032D1F380538A3008F066
:1062600041C0C0934F0530E020E04AE0DF011196C5
:10627000429FC001439F900D11249C01205331097E
:106280008081280F311D87FD3A95818190ED980F0F
:106290009A30C8F130934E0520934D058E3261F44B
:1062A000329690E04AE0DF0131968C9150ED580F24
:1062B0005A3058F190934C05CD01DC0101964C9178
:1062C0004032D9F3CD3489F52E31310539F018F546
:1062D0002731310519F02C31310539F5B0935505C9
:1062E000A0935405DF91CF911F910F91FF90EF90F4
:1062F000DF90CF90BF90AF909F908F900895F9015D
:106300007BCFF90181CFFD01B1CF949F800D112486
:1063100090ED980FC8CF2537310538F02737310574
:10632000E8F2203A83E03807C9F2D091C50840E08E
:1063300050E0BA0110E000E0C12CD12C7601C394EA
:10634000FD0131968C91882309F47FC08132E1F4FC
:10635000CD34D1F420323105B9F440935005509337
:1063600051056093520570935305F0935505E093E2
:10637000540563E270E0CF010F948077009709F431
:10638000B1CFFC011082AECF81548A3108F058C0E1
:10639000DF019D91903291F0A0EDA90FAA30E8F0B5
:1063A0009E3271F4918190539A30B8F00115110525
:1063B00019F48F010150110990E013C0FD01E8CFDD
:1063C0009D3211F09B3291F79181A0EDA90FAA3077
:1063D00020F09E3259F79281E6CF9E2F9D1B309779
:1063E00059F3A82FB0E04601570104C0880C991C4E
:1063F000AA1CBB1C8A95D2F7482959296A297B29EE
:10640000AE5CBA4F9C9380818154DF018A3108F4DD
:1064100097CFDF018191882309F492CF90ED980FF7
:106420009A30B8F393ED980F923098F38B3289F34A
:10643000CD010196EC91E03209F082CFDC01F8CF7A
:106440000115110501F78D01DECF1093550500935D
:106450005405409350055093510560935205709335
:10646000530540CFFC0165917591859194910895F4
:106470008091B908882319F080E00F945E1C80E0B9
:1064800008954F925F926F927F928F929F92AF92F8
:10649000BF92CF92DF92EF92FF92CF93DF9300D023
:1064A00000D01F921F92CDB7DEB75C01DB01CD900B
:1064B000DD90ED90FC90E091E316F091E416FE8300
:1064C000ED8384819581A681B78189839A83AB838B
:1064D000BC839C01AD01C701B6010F9431742B013F
:1064E0003C01F50180809180A280B380AD81BE81A6
:1064F0008D919D910D90BC91A02D8D839E83AF8336
:10650000B88727E137EB41ED58EBC301B2010F9497
:10651000927687FDD0C027E030E040E753E4C30126
:10652000B2010F94406D18160CF4C5C02D813E8148
:106530004F815885C501B4010F9431742B013C0182
:1065400027E137EB41ED58EB0F94927687FDB3C00E
:1065500027E030E040E753E4C301B2010F94406DFF
:1065600018160CF4A8C020E030E0A9016D817E81EE
:106570008F8198850F9432742B013C0120E030E02C
:1065800040E450E40F94406D87FF05C0412C512C2E
:1065900030E4632E762C27E137EB41ED58E3C3015D
:1065A000B2010F9431749B01AC01C501B4010F9489
:1065B000927687FD80C020E030E040E753E46D81B3
:1065C0007E818F8198850F9432742B013C0120E0ED
:1065D00030E043E653E40F949276181634F4412CDD
:1065E000512C23E6622E23E4722E27E137EB41ED96
:1065F00058E3C301B2010F9432749B01AC01C50191
:10660000B4010F94406D18160CF455C020E030E032
:10661000A90169817A818B819C810F9432744B012D
:106620005C0120E030E040E951E40F94406D87FFC9
:1066300006C0812C912C90E9A92E91E4B92E27E176
:1066400037EB41ED58E3C501B4010F9431749B0160
:10665000AC01C701B6010F94927687FD2CC020E0F3
:1066600030E040E753E469817A818B819C810F940B
:1066700032744B015C0120E030E044E553E40F94B8
:106680009276181634F4812C912C84E5A82E83E49C
:10669000B82E27E137EB41ED58E3C501B4010F9463
:1066A00032749B01AC01B1E0B983C701B6010F940C
:1066B000406D18160CF41982898128960FB6F8944B
:1066C000DEBF0FBECDBFDF91CF91FF90EF90DF9087
:1066D000CF90BF90AF909F908F907F906F905F9082
:1066E0004F9008958F929F92AF92BF92CF92DF9278
:1066F000EF92FF92CF93DF93EC018090DE089090B1
:10670000DF08A090E008B090E10820E030E0A901A7
:10671000C501B4010F94406D882309F452C0C880AC
:10672000D980EA80FB80A7019601C501B4010F94CE
:10673000406D18160CF04AC020911E0530911F05BF
:106740004091200550912105C701B6010F94406D7D
:10675000882321F1C0921E05D0921F05E0922005EA
:10676000F092210520911A0530911B0540911C05DE
:1067700050911D05C701B6010F94A66D9B01AC0198
:1067800060E070E080E89FE30F943174609317023B
:10679000709318028093190290931A026091170265
:1067A000709118028091190290911A02DF91CF9195
:1067B000FF90EF90DF90CF90BF90AF909F908F9021
:1067C000089560E070E080E89FE3F0CF60E070E063
:1067D000CB01ECCF9B01AC01485F5F4FBC016C5F0C
:1067E0007F4F0C94E5280F931F93CF93DF9300D036
:1067F00000D01F921F92CDB7DEB7FC018B0183A59D
:10680000811112C081E083A784819581A681B7811F
:10681000B05889839A83AB83BC83BE016F5F7F4F7F
:1068200088EA98E00E94EA331D821E821F82188641
:1068300020E030E040E05FE36091DB097091DC092B
:106840008091DD099091DE090F94327469837A8317
:106850008B839C839E012B5F3F4FAE014F5F5F4F49
:1068600067ED79E083ED99E00E94E5281D821E82A4
:106870001F82188620E030E040E05FE3F801608589
:106880007185828593850F94327469837A838B83B3
:106890009C83B8016C5F7F4F9E012B5F3F4FAE0121
:1068A0004F5F5F4FC8010E94E52828960FB6F89405
:1068B000DEBF0FBECDBFDF91CF911F910F91089525
:1068C0002F923F924F925F926F927F928F929F9200
:1068D000AF92BF92CF92DF92EF92FF920F931F93EE
:1068E000CF93DF93CDB7DEB7A2970FB6F894DEBF94
:1068F0000FBECDBF8C011B015E834D834090D30939
:106900005090D4096090D5097090D6098090D7092D
:106910009090D809A090D909B090DA09DB018D9147
:106920009D910D90BC91A02D8F87988BA98BBA8BD0
:106930009C01AD01C301B2010F9431746B017C0164
:10694000D10114968D919D910D90BC91A02D8B8BB2
:106950009C8BAD8BBE8B9C01AD01C501B4010F9426
:1069600031746F8B788F898F9A8FAD81BE818D91B5
:106970009D910D90BC91A02D8F839887A987BA8790
:106980009C01AD01C301B2010F9431746B8F7C8FF8
:106990008D8F9E8FAD81BE8114968D919D910D90AE
:1069A000BC91A02D8B879C87AD87BE879C01AD01D4
:1069B000C501B4010F9431746F8F78A389A39AA392
:1069C000A7019601C701B6010F94A66D6B017C016A
:1069D0002F89388D498D5A8DCA01B9010F94A66D42
:1069E0009B01AC01C701B6010F9432744B015C01ED
:1069F0002F85388949895A896F81788589859A8553
:106A00000F9431742B013C012B893C894D895E899F
:106A10006B857C858D859E850F9431746B017C011F
:106A2000A3019201C301B2010F94A66D2B013C0199
:106A3000A7019601C701B6010F94A66D9B01AC0199
:106A4000C301B2010F9432740F94E0766B017C01A4
:106A50002B8D3C8D4D8D5E8DCA01B9010F94A66DB5
:106A60002B013C012F8D38A149A15AA1CA01B901BE
:106A70000F94A66D9B01AC01C301B2010F94327457
:106A80009B01AC01C501B4010F9492761816B4F5C0
:106A900020E030E0A901C701B6010F94927687FF8C
:106AA0002AC0C701B601905820E030E040EA50E427
:106AB0000F949276181614F5A1016D817E81C8019C
:106AC0000E946034A2960FB6F894DEBF0FBECDBF11
:106AD000DF91CF911F910F91FF90EF90DF90CF90BA
:106AE000BF90AF909F908F907F906F905F904F90EE
:106AF0003F902F900895C701B601D6CF20E030E037
:106B000040E050E4C501B4010F949276181624F4C5
:106B1000B101C8010E94F33319821A821B821C82C0
:106B2000BE016F5F7F4FC1010E94EA332DEC3CEC48
:106B30004CEC5CE3C701B6010F94A66D9B01AC0160
:106B4000F80160817181828193810F94A66D6983C0
:106B50007A838B839C83C8010F94E04ABE016F5FE8
:106B60007F4F8D819E810E94EA33ACCF3F924F923E
:106B70005F926F927F928F929F92AF92BF92CF92CD
:106B8000DF92EF92FF920F931F93CF93DF93CDB7D6
:106B9000DEB76C970FB6F894DEBF0FBECDBFDB013A
:106BA0000C91142F100F153008F067C11196DC906E
:106BB000C22ECD0CB4E0BC1508F45FC1ED2DF0E0A1
:106BC000EF5EFA4F8080912CB12CA12C002E04C0D6
:106BD000B694A794979487940A94D2F780FE4DC1F7
:106BE000EC2DF0E0EF5EFA4F8080912CB12CA12CBF
:106BF000012E04C0B694A794979487940A94D2F770
:106C000080FE3BC1322E642F7C0140908106509063
:106C10008206609083067090840680918906909128
:106C20008A06A0918B06B0918C06898F9A8FAB8FC4
:106C3000BC8F660F770B072E000C880B990B0F94F7
:106C4000476D4B015C01602F000F770B880B990B90
:106C50000F94476D298D3A8D4B8D5C8D0F94A66DE9
:106C6000A30192010F943274A50194010F94327420
:106C70006D877E878F87988B612F110F770B880B1D
:106C8000990B0F94476D298D3A8D4B8D5C8D0F9428
:106C9000A66DA30192010F943274A50194010F9483
:106CA000317469837A838B839C83409085065090EE
:106CB0008606609087067090880680918D06909178
:106CC0008E06A0918F06B0919006898F9A8FAB8F18
:106CD000BC8F632D660F770B072E000C880B990B6A
:106CE0000F94476D4B015C016D2DDD0C770B880B0C
:106CF000990B0F94476D298D3A8D4B8D5C8D0F94B8
:106D0000A66DA30192010F943274A50194010F9412
:106D10003274698B7A8B8B8B9C8B6C2DCC0C770BA4
:106D2000880B990B0F94476D298D3A8D4B8D5C8D97
:106D30000F94A66DA30192010F943274A5019401E2
:106D40000F9431746D837E838F839887F7018085DC
:106D50009185A285B38589879A87AB87BC878D8B00
:106D60009E8BAF8BB88F4FEE50E061E070E0CE01AC
:106D700041960E9467F44FEE50E061E070E0CE0172
:106D800005960E9467F44FEE50E061E070E0CE019E
:106D90000D960E9467F44FEE50E061E070E0CE0186
:106DA00001960E9467F489889A88AB88BC8827E19D
:106DB00037EB41ED58EBC501B4010F94927687FD96
:106DC0005CC027E030E040E753E4C501B4010F9414
:106DD000406D18160CF451C08D849E84AF84B88821
:106DE00027E137EB41ED58EBC501B4010F949276E2
:106DF00087FD43C027E030E040E753E4C501B4011C
:106E00000F94406D1816CCF18D809E80AF80B884B1
:106E100027E137EB41ED58EBC501B4010F949276B1
:106E200087FD2BC027E030E040E753E4C501B40103
:106E30000F94406D18160CF189809A80AB80BC804D
:106E400027E137EB41ED58EBC501B4010F94927681
:106E500087FD13C027E030E040E753E4C501B401EB
:106E60000F94406D18164CF0AE014F5F5F4FBE019E
:106E7000635F7F4FC7010E9460346C960FB6F89431
:106E8000DEBF0FBECDBFDF91CF911F910F91FF905D
:106E9000EF90DF90CF90BF90AF909F908F907F90BA
:106EA0006F905F904F903F9008958C38910514F04B
:106EB0008CE890E09093EA088093E9080C94CEDC8B
:106EC0000E94452ACB0108950F931F93CF93809181
:106ED0002205909123050097E9F0FC018F01C191F3
:106EE0002C2F2F7D81F0C53411F0C536B9F7F8018C
:106EF000108270E060E00F94CF68F801C083CF91FA
:106F00001F910F91089570E060E0CF911F910F9154
:106F10000D94CF6860E070E0CB01F1CF2FEB280F2C
:106F20002A3108F047C0E22FF0E08091500590919F
:106F30005105A0915205B091530504C0B695A7958F
:106F4000979587952A95D2F780FD02C081700895A4
:106F5000EE5CFA4FE081EE2341F18091C5089091FB
:106F6000C608E80FF92FF11D808190ED980F9A3037
:106F700030F08E3251F4818180538A3098F4F0934E
:106F80002305E093220581E008958D3211F08B32C4
:106F900049F4818190ED980F9A3088F38E3211F484
:106FA0008281EACFF0E0E0E0EACF10922305109270
:106FB0002205E9CF80E008950E948E37882341F0B2
:106FC00081E02091220530912305232B09F480E0F4
:106FD0000895CF93DF93EB010E94DC37882319F0EB
:106FE0000E94452AEB01CE01DF91CF91089583E500
:106FF0000E94DC378823E9F00F945F526093BA084F
:107000007093BB088093BC089093BD080E946437BE
:1070100020E030E04AE754E40F94A66D0F94A57584
:1070200060931B0270931C0280931D0290931E02BA
:1070300008958091500584FD0AC08091520587FD16
:1070400006C080915305837011F40C943DFB0E949F
:107050002CFB88E50E948E37882331F05F9A80915F
:10706000B8088E7F8093B80889E50E948E37882300
:1070700031F08A9A8091B8088D7F8093B8088AE5AC
:107080000E948E37882359F0809108018095817085
:10709000809306018091B8088B7F8093B80885E4BF
:1070A0000E948E3781110C946A260895CF93C62FC3
:1070B0000E94DC37882319F0CF910C94552A8C2F2D
:1070C000CF910895CF92DF92EF92FF926A017B01F8
:1070D0000E94DC37882331F0FF90EF90DF90CF9053
:1070E0000C946437C701B601FF90EF90DF90CF900A
:1070F00008954F925F926F927F928F929F92AF927C
:10710000BF92CF92DF92EF92FF921F93CF93DF93C4
:1071100000D01F92CDB7DEB719821A821B821C8263
:10712000CE0101964C0183EDC82E89E0D82E98EA55
:10713000E92E98E0F92E27ECA22E29E0B22E10E0DD
:1071400088E5810F0E94DC37F40181934F01882389
:1071500041F00E9464372B013C018091DA108823B2
:1071600059F0F60180819181A281B381F70180837A
:107170009183A283B38314C0812F0E947F2488232C
:1071800009F4D0C0F6012081318142815381C301CD
:10719000B2010F943274F701608371838283938309
:1071A0001F5FF4E0CF0ED11C84E0E80EF11C94E0E8
:1071B000A90EB11C133021F685E40E94DC378C83C4
:1071C000882309F4B9C00E9464376B017C0183E015
:1071D0000E947F24882371F02091DF093091E0091B
:1071E0004091E1095091E209C701B6010F94327450
:1071F0006B017C01C092B408D092B508E092B60849
:10720000F092B70880911C06882359F180916A1783
:1072100082FF27C08C81882321F18981811103C0DD
:107220008A818823F1F02DEC3CEC4CE45DE3609125
:107230001E0970911F0980912009909121090F94D6
:1072400032749B01AC016091DB097091DC09809183
:10725000DD099091DE090F949276181614F40F94BC
:10726000335D40E050E0BA0186E40E94623820E0DD
:1072700030E0A9010F949276181684F40E946437C6
:1072800020E030E040E752E40F942C7560938502D3
:107290007093860280938702909388028091DB101E
:1072A00083FD2CC08091DA10811128C080911B08C9
:1072B000882321F12091DF093091E0094091E10913
:1072C0005091E2096091B4087091B5088091B608B8
:1072D0009091B7080F9431742091280830912908B3
:1072E00040912A0850912B080F943274609328081B
:1072F0007093290880932A0890932B080F900F9081
:107300000F900F90DF91CF911F91FF90EF90DF9042
:10731000CF90BF90AF909F908F907F906F905F9035
:107320004F900895F5012081318142815381C3013D
:10733000B2010F9431742FCF8091DF099091E00951
:10734000A091E109B091E2098093B4089093B50847
:10735000A093B608B093B70855CFCF93DF93EB0156
:107360000E94DC37882321F0DF91CF910C946037A5
:10737000CE01DF91CF910895CF93DF93C82FD62F01
:107380000E94DC37882321F0DF91CF910C94692A89
:107390008C2F0E948E37811101C08D2FDF91CF91EC
:1073A0000895E5E1F9E082EBDF011D928A95E9F7A6
:1073B000089580911C06811104C00E94D1390D945A
:1073C000015E80916A1782FD0D94335D089580916E
:1073D0001509882361F09091C609891308C080912E
:1073E0006A1783FF04C083E599E00D94405C80E058
:1073F0000895FC01238121110C9440E90895CF9256
:10740000DF92EF92FF920F931F93CF9390913002F0
:10741000913009F461C0662351F01092000510927A
:10742000FC041092FD041092FE041092FF04C82F79
:107430000F945F52C090FC04D090FD04E090FE04D5
:10744000F090FF049B01AC012C193D094E095F0926
:1074500069017A01F7FC40C020910005C7FD15C005
:107460004C2F0C2E000C550B4C5F5F4FE22F022E61
:10747000000CFF0B4E175F077CF144EFC42EDD2498
:10748000D394E12CF12C2C1734F438EEC32E33E0D6
:10749000D32EE12CF12CC60ED71EE81EF91EC09289
:1074A000FC04D092FD04E092FE04F092FF04022F4F
:1074B000017010E084E2809FB001819F700D701B0D
:1074C000112460597C4F82E390E00E945395809193
:1074D00000058F5F80930005CF911F910F91FF9062
:1074E000EF90DF90CF9008950F931F9301E010E08D
:1074F00020E030E0082E04C0000F111F221F331FB0
:107500000A94D2F740915F05509160056091610542
:1075100070916205402B512B622B732B40935F05BA
:1075200050936005609361057093620590912F02FE
:10753000891303C081E08093DA101F910F910895A1
:107540004F925F926F927F928F929F92AF92BF9273
:10755000CF92DF92EF92FF920F931F93CF93DF931F
:10756000EC01209181063091820640918306509172
:107570008406688179818A819B810F9431746B01C3
:107580007C012091850630918606409187065091B6
:1075900088066C817D818E819F810F9431744B01AF
:1075A0005C01A701960160910B0270910C02809121
:1075B0000D0290910E020F94406D882309F450C083
:1075C000C0920B02D0920C02E0920D02F0920E02D9
:1075D0002091F4043091F5044091F6045091F704A1
:1075E000C701B6010F94A66D2B013C010F94D47511
:1075F0006B017C0120E030E0A9010F94406D87FD14
:1076000070C020E030E040E450E4C701B6010F94C0
:10761000927618162CF4C12CD12CC0E4EC2EFE2C42
:10762000A7019601C301B2010F9431746093EC0479
:107630007093ED048093EE049093EF04C701B601BC
:107640000F949E756093EA04062E000C770B6F5F13
:107650007F4F6430710514F064E070E06093E804DB
:10766000D09109021091EA04A501940160910F02E2
:107670007091100280911102909112020F94406D4E
:10768000811133C0D11381C02091D0043091D10435
:107690004091D2045091D3046091EC047091ED04B8
:1076A0008091EE049091EF040F94A66D2091D40484
:1076B0003091D5044091D6045091D7040F94327480
:1076C000DF91CF911F910F91FF90EF90DF90CF90BE
:1076D000BF90AF909F908F907F906F905F904F90F2
:1076E0000895C12CD12C76019BCF80920F029092ED
:1076F0001002A0921102B09212022091F80430916F
:10770000F9044091FA045091FB04C501B4010F94AF
:10771000A66D4B015C010F94D4756B017C0120E0D8
:1077200030E0A9010F94406D87FDF3C020E030E008
:1077300040E450E4C701B6010F94927618162CF479
:10774000C12CD12CB0E4EB2EFE2CA7019601C50173
:10775000B4010F9431746093F0047093F10480933A
:10776000F2049093F304C701B6010F949E756093E1
:10777000EB04062E000C770B6F5F7F4F64307105B2
:1077800014F064E070E06093E904C091EB04D1135D
:1077900005C080910A028C1709F470C08091EA0438
:1077A0009091EB0490930A02809309020C2E000C36
:1077B000DD0B25E01203C0011124FC01EC0FFD1FBD
:1077C000EE0FFF1FEE0FFF1FE35EF94F20813181A7
:1077D000428153812093E4043093E5044093E6040E
:1077E0005093E7040091E904002E000C110BFC01FA
:1077F000E00FF11FEE0FFF1FEE0FFF1FE35EF94FCB
:1078000060817181828193810F9431746093E0046F
:107810007093E1048093E2049093E3042091E804E0
:1078200035E02303F0011124CE0FDF1FCC0FDD1F45
:10783000CC0FDD1FC35ED94F288139814A815B811E
:107840002093DC043093DD044093DE045093DF0486
:10785000E00FF11FEE0FFF1FEE0FFF1FE35EF94F6A
:1078600060817181828193810F9431746093D80417
:107870007093D9048093DA049093DB048090F00431
:107880009090F104A090F204B090F3042091E004F1
:107890003091E1044091E2045091E304C501B40148
:1078A0000F94A66D2091E4043091E5044091E60424
:1078B0005091E7040F9432746B017C01C092D404A0
:1078C000D092D504E092D604F092D7042091D80447
:1078D0003091D9044091DA045091DB04C501B40120
:1078E0000F94A66D2091DC043091DD044091DE04FC
:1078F0005091DF040F943274A70196010F943174F4
:107900006093D0047093D1048093D2049093D304F5
:10791000BBCEC12CD12C760118CF1F93CF93DF9310
:10792000CDB7DEB72C970FB6F894DEBF0FBECDBF34
:10793000182F882379F020E030E0A90160918906B2
:1079400070918A0680918B0690918C060F94406D01
:107950008823F9F08091E2088117D9F00E942CFB6E
:107960008CE0E4E9F2E0DE01119601900D928A9537
:10797000E1F7CE0101960E94A03A8091E2088823A7
:1079800091F083ED99E00E944FFB1092E2080F9472
:107990000A122C960FB6F894DEBF0FBECDBFDF9152
:1079A000CF911F91089581E08093E20883ED99E0E3
:1079B0000E947CFAECCF80E00E948D3C10928506FC
:1079C0001092860610928706109288061092810601
:1079D00010928206109283061092840610928D06F1
:1079E00010928E0610928F061092900610928906C1
:1079F00010928A0610928B0610928C06EDE1F6E04A
:107A000021E836E080E090E0A0ECBFE7808391833E
:107A1000A283B38384839583A683B783808791876A
:107A2000A287B38784879587A687B787808B918B3A
:107A3000A28BB38B74962E173F0741F708954F9290
:107A40005F926F927F928F929F92AF92BF92CF92EE
:107A5000DF92EF92FF921F93CF93DF93EC01162FEB
:107A60002091DE083091DF084091E0085091E10854
:107A7000688179818A819B810F94406D882309F404
:107A8000AEC0B090E20880E00E948D3CC880D980F2
:107A9000EA80FB8020E030E0A901C701B6010F9425
:107AA000927618161CF0C12CD12C7601C092DE08FB
:107AB000D092DF08E092E008F092E1082DEB37E386
:107AC00046E855EBC701B6010F94927687FD0BC0CF
:107AD0002DEB37E346E855E3C701B6010F94406D3F
:107AE00018160CF078C0A701960160E070E080E8FD
:107AF0009FE30F942C7560931A0570931B05809378
:107B00001C0590931D0580EF9FEFA9E7B4EC8093CF
:107B10001E0590931F05A0932005B0932105BB205F
:107B200009F45DC04090D3095090D4096090D50904
:107B30007090D6098090D7099090D809A090D90963
:107B4000B090DA09C090DB09D090DC09E090DD0943
:107B5000F090DE0981E00E948D3C112309F43FC0C2
:107B60002091D3093091D4094091D5095091D6097B
:107B7000C301B2010F94406D81111CC02091D7093F
:107B80003091D8094091D9095091DA09C501B40161
:107B90000F94406D81110EC02091DB093091DC09FA
:107BA0004091DD095091DE09C701B6010F94406D87
:107BB0008823A9F0DF91CF911F91FF90EF90DF9084
:107BC000CF90BF90AF909F908F907F906F905F907D
:107BD0004F900D948B1960E070E0CB018CCFDF915A
:107BE000CF911F91FF90EF90DF90CF90BF90AF901B
:107BF0009F908F907F906F905F904F9008958F929D
:107C00009F92AF92BF92CF92DF92EF92FF92C0907D
:107C10008906D0908A06E0908B06F0908C0620E0D2
:107C200030E0A901C701B6010F94406D8823E1F14E
:107C3000A701960160E070E080E89FE30F942C7547
:107C40006B017C0180908D0690908E06A0908F062F
:107C5000B090900620E030E0A901C501B4010F9476
:107C6000406D882329F1A501940160E070E080E86F
:107C70009FE30F942C75C092F404D092F504E09227
:107C8000F604F092F7046093F8047093F90480937B
:107C9000FA049093FB04FF90EF90DF90CF90BF9099
:107CA000AF909F908F900895C12CD12C7601CACFB0
:107CB00060E070E0CB01DFCFEFE6F0E08081826032
:107CC000808308958091BE089091BF08892B79F434
:107CD0008091BE089091BF08892B49F42091BE087D
:107CE0003091BF0881E0232B19F480E0089581E0F2
:107CF0000895CF92DF92EF92FF926B017C0183E3B4
:107D0000C816D104E104F10470F082E3C81AD10866
:107D1000E108F10862E370E080E090E00F942C52FB
:107D20000F940C12ECCFC701B6010F942C52FF90A8
:107D3000EF90DF90CF900D940C128091A8068111E6
:107D40000AC08091DC08813041F080916A1782FB83
:107D5000882780F9089580E0089581E008955F9A6A
:107D60008091B8088E7F8093B8088A9A8091B8086D
:107D70008D7F8093B80880910801809581708093F1
:107D800006018091B8088B7F8093B8080C946A260E
:107D900090916A1793FB882780F993FF06C081E0D2
:107DA0009091D218911101C080E008958091A806A9
:107DB000811110C08091DC08823061F00E94C83EC1
:107DC000882349F080916A1782FB882780F991E027
:107DD0008927089581E008950E94D63E81110DC043
:107DE00010925F0510926005109261051092620575
:107DF000109263058FEF0E946C280D947C2081E027
:107E00000D94EC1FE5E1FAE010821182089581E003
:107E10000895DC01EC918E2F90E0FC01EE0FFF1F26
:107E2000E80FF91FE557F94E80818F778083089519
:107E30008F929F92AF92BF92CF92DF92EF92FF927A
:107E40000F93CF93DF931F92CDB7DEB75C017B0119
:107E500049016B01C40ED51EF501808191810F94FB
:107E60005E738983002311F0F7018083BE016F5F89
:107E70007F4FC4010F947330F50180819181019689
:107E800091838083FFEFEF1AFF0AEC14FD0421F7C2
:107E900080E00F90DF91CF910F91FF90EF90DF90F6
:107EA000CF90BF90AF909F908F900895009781F4EE
:107EB0001092900082E080939100109295001092B1
:107EC0009400C19A8091710082608093710008953E
:107ED000019761F41092A00082E08093A1001092BB
:107EE000A5001092A40089BB8093720008957F9230
:107EF0008F929F92AF92BF92CF92DF92EF92FF92BA
:107F00000F931F93CF93DF93EC017B01888188311E
:107F100008F0C3C090E0FC01EE0FFF1FE80FF91F4F
:107F2000E557F94E80818F770F94313219821A828A
:107F300088812CE0622F0F94E773829FB001112497
:107F400030E020E0AB01420F531FFA01EE0FFF1F9C
:107F5000E40FF51FE557F94E908197FD08C02F5F9C
:107F60003F4F2C30310571F790E00E94563F7880EA
:107F7000072D10E06801CC0CDD1CF601E00FF11FAD
:107F8000E557F94E80818068808377FC86C080E267
:107F9000E81682E0F8060CF03FC08A8128E532E05E
:107FA000281B310987FD3395220F331F220F331F02
:107FB000032E000C440B550B898178E8872E912CF9
:107FC000881A910887FD9394880C991C880C991C39
:107FD000092C000CAA08BB0860E070E0CB01F7FC9C
:107FE0000AC0B701653B710514F064EB70E0072E21
:107FF000000C880B990B281939094A095B090F9461
:10800000747324EB30E040E050E00F94A673820ECE
:10801000931EA41EB51E740187E18715D8F029812F
:1080200088E890E0821B910927FD9395880F991F9E
:10803000880F991FE816F90604F502972FB7F894F0
:10804000E601C00FD11FC557D94E880F991F9A83DB
:1080500089832FBF62E370E080E090E0DF91CF91F1
:108060001F910F91FF90EF90DF90CF90BF90AF9056
:108070009F908F907F900C94793E2A8188E592E0C2
:10808000821B910927FD9395880F991F880F991FCF
:10809000E816F90694F6C701D0CFDF91CF911F9172
:1080A0000F91FF90EF90DF90CF90BF90AF909F9097
:1080B0008F907F900895CF93DF93EB01682F70E04E
:1080C00084ED96E10E94773F688179818A819B8166
:1080D000643F21E072078105910520F464EF71E0AF
:1080E00080E090E00E94793E89B183FB882780F987
:1080F000DF91CF910895CF93DF9300D01F92CDB73A
:10810000DEB78EEE92E0A0E0B0E089839A83AB8385
:10811000BC83BE016F5F7F4F8AE50E945B400F907A
:108120000F900F900F90DF91CF910895CF93DF9331
:1081300000D01F92CDB7DEB78EEE92E0A0E0B0E0A7
:1081400089839A83AB83BC83BE016F5F7F4F8AE0D4
:108150000E945B400F900F900F900F90DF91CF9196
:108160000895CF93DF9300D01F92CDB7DEB784EF91
:1081700091E0A0E0B0E089839A83AB83BC83BE0129
:108180006F5F7F4F8CE30E945B400F900F900F90CA
:108190000F90DF91CF910895CF93DF9300D01F927E
:1081A000CDB7DEB784EF91E0A0E0B0E089839A8399
:1081B000AB83BC83BE016F5F7F4F80EA0E945B4050
:1081C0000F900F900F900F90DF91CF9108951F9215
:1081D0000F920FB60F9211240BB60F922F933F936D
:1081E0004F935F936F937F938F939F93AF93BF93BF
:1081F000EF93FF9348EA50E064EA70E081E090E09A
:108200000E94792AFF91EF91BF91AF919F918F9139
:108210007F916F915F914F913F912F910F900BBE86
:108220000F900FBE0F901F9018951F920F920FB6D0
:108230000F9211240BB60F922F933F934F935F939E
:108240006F937F938F939F93AF93BF93EF93FF931E
:1082500048E950E064E970E090E080E00E94792A0B
:10826000FF91EF91BF91AF919F918F917F916F910E
:108270005F914F913F912F910F900BBE0F900FBECA
:108280000F901F9018959091C00095FFFCCF8093A0
:10829000C6000895CF93DF93EC018991882319F0EC
:1082A0000E944341FACF8DE00E9443418AE0DF9172
:1082B000CF910C944341CF92DF92EF92FF92CF93F4
:1082C0006B017C01C42F4A3069F4F7FE0BC0F094B7
:1082D000E094D094C094C11CD11CE11CF11C8DE22F
:1082E0000E9443414C2FC701B601CF91FF90EF9000
:1082F000DF90CF900D94775CCF93DF93EC01FE017C
:1083000084912196882319F00E944341F8CFDF9190
:10831000CF9108950F931F93CF938C01C62F81E5C2
:1083200095E10E947C41C8010E947C418AE30E9441
:10833000434180E38C0F0E9443418AE0CF911F911B
:108340000F910C94434184ED96E10E947C4160E0E2
:1083500084EC96E10E948A4160E08FEA96E10E94F7
:108360008A4161E088EA96E10E948A4161E08DE9F4
:1083700096E10E948A4161E08DE896E10E948A417F
:1083800060E084E896E10E948A4161E08AE796E134
:108390000E948A4161E080E796E10E948A4160E0A4
:1083A00089E696E10E948A4161E081E696E10E94B9
:1083B0008A4161E083E596E10E948A4161E085E4BB
:1083C00096E10E948A4160E086E396E10E948A413C
:1083D00060E088E296E10E948A4160E082E196E1F5
:1083E0000E948A4161E081E096E10E948A4161E059
:1083F00082EF95E10E948A4161E08BEE95E10E9457
:108400008A4160E084EE95E10E948A4161E08BED53
:1084100095E10E948A4161E086EC95E10E948A41E3
:1084200061E088EB95E10E948A4161E085EA95E18F
:108430000E948A4160E088E995E10E948A4161E0FA
:1084400083E995E10E948A4161E086E895E10E9416
:108450008A4160E082E795E10E948A4160E08FE511
:1084600095E10E948A4160E08EE697E10E947C24BB
:10847000682F617086E595E10C948A4180915005E2
:10848000827149F4809152058C7829F480915305CA
:10849000837009F475C082E40E948E37882351F0FE
:1084A0000E94242A6093EC107093ED108093EE10DC
:1084B0009093EF1083E50E948E37882351F00E943D
:1084C000643760931C1170931D1180931E1190935B
:1084D0001F1184E50E948E37882351F00E94643773
:1084E0006093201170932111809322119093231196
:1084F00088E50E948E37882351F00E94643760938C
:10850000FD097093FE098093FF099093000A89E5A5
:108510000E948E37882351F00E9464376093010ACD
:108520007093020A8093030A9093040A8AE50E94DA
:108530008E378823B1F00E9464376093050A7093E8
:10854000060A8093070A9093080A2DEC3CEC4CEC49
:108550005DE30F94406D181624F08FEF9FE00E94AA
:108560007C4185E40E948E37882351F00E94643755
:108570006093090A70930A0A80930B0A90930C0A7D
:108580000895AF92BF92CF92DF92EF920F931F9315
:10859000CF93DF935B01EA016901882309F463C08B
:1085A00085EE9FE00E947C41F501608171818281AE
:1085B000938146E00E943AEFE1100BC08CED9FE002
:1085C0000E947C41688179818A819B8146E00E947A
:1085D0003AEF85ED9FE00E947C41F6016081718158
:1085E0008281938143E00E943AEF8EEC9FE00E94EB
:1085F0007C41F801608171818281938143E00E9416
:108600003AEF85EC9FE00E947C41F60120813181A8
:1086100042815381F80160817181828193810F943D
:10862000317443E00E943AEFEE20F9F08AE00E94B4
:10863000434180EB9FE00E947C41688179818A817F
:108640009B8146E00E943AEF8AE00E9443418AE023
:10865000DF91CF911F910F91EF90DF90CF90BF905E
:10866000AF900C944341E110E4CFDF91CF911F9183
:108670000F91EF90DF90CF90BF90AF9008950F9340
:108680001F93CF938C01C62F88E59AE00E947C410E
:10869000C8010E947C41CC2331F08AE0CF911F9128
:1086A0000F910C944341CF911F910F91089560E079
:1086B00086EF95E40E943F4388E69AE00E947C4161
:1086C0008AE00C944341EF92FF920F931F93CF9354
:1086D0007C018B01C42F60E086EF95E40E943F434C
:1086E000C7010E947C4180E20E944341C8010E9470
:1086F0007C41CC2319F08C2F0E9443418AE0CF911A
:108700001F910F91FF90EF900C944341DF92EF92F5
:10871000FF920F931F93CF93DF93D82E7B018A0193
:10872000E9010E945743D092C00840E0B7018AE0B7
:1087300096E40E9463430115110531F040E0B80151
:1087400083E096E40E946343209731F040E0BE014D
:1087500083E096E40E94634360E086EF95E40E9424
:108760003F438EEF95E40E947C418AE0DF91CF91F8
:108770001F910F91FF90EF90DF900C94434161E0C7
:1087800082E69AE00C943F43AF92BF92CF92DF9281
:10879000EF92FF920F931F93CF93DF938FEA99E0AD
:1087A0000E947C41C0E0D7E0D15021F080E20E94DD
:1087B0004341FACF8C2F0F94DE5CCF5FC53099F721
:1087C0008AE00E9443410DE116E0C0E080E20E9491
:1087D00043418C2F0F94DE5C5801D5E080E20E946B
:1087E0004341F501C080D180E280F380A70196016A
:1087F000C701B6010F942477882369F180E20E94B3
:1088000043418DE30E9443418DE30E9443418DE348
:108810000E9443418DE30E9443418DE30E94434106
:10882000D150F4E1AF0EB11CD111D8CF8AE00E9433
:108830004341CF5F0C5F1F4FC53041F68AE0DF91A7
:10884000CF911F910F91FF90EF90DF90CF90BF904D
:10885000AF900C94434120E030E0A901C701B6017C
:108860000F94927687FD03C08BE20E94434143E060
:10887000C701B6010E943AEFD3CFCF93DF93EB014C
:108880000E947C41CE01DF91CF910D94E55CCF93A6
:10889000C62F0E947C418C2FCF910D94DE5CCF922D
:1088A000DF92EF92FF926A017B010E947C4142E0DD
:1088B000C701B601FF90EF90DF90CF900C943AEF94
:1088C0008091510587FD2BC0809152058E7039F53E
:1088D000409110115091111160911211709113116A
:1088E0008FEE9FE00E944F4440911411509115115A
:1088F00060911611709117118CEE9FE00E944F4409
:10890000409118115091191160911A1170911B1119
:1089100083E092E30E944F448AE00C94434183E554
:108920000E94DC37882391F00E9464376093101115
:108930007093111180931211909313116093181179
:108940007093191180931A1190931B1180E50E9466
:10895000DC37882351F00E946437609310117093C4
:108960001111809312119093131182E50E94DC374C
:10897000882351F00E94643760931411709315118D
:10898000809316119093171184E50E94DC37882399
:1089900051F00E94643760931811709319118093FD
:1089A0001A1190931B110895CF92DF92EF92FF92CC
:1089B0006A017B010E947C414AE0C701B601FF9039
:1089C000EF90DF90CF900C945B412F923F924F92AB
:1089D0005F926F927F928F929F92AF92BF92CF924F
:1089E000DF92EF92FF920F931F93CF93DF93CDB758
:1089F000DEB7C654D1090FB6F894DEBF0FBECDBFA7
:108A000070E060E085E40E94AD39182F8F3F09F4D3
:108A100083C08823E9F08EE09AE1CA5BDF4F0FB68E
:108A2000F894DEBF0FBECDBFDF91CF911F910F91A4
:108A3000FF90EF90DF90CF90BF90AF909F908F907E
:108A40007F906F905F904F903F902F900C947C415F
:108A500024EB30E03A83298383E50E94DC378823C6
:108A600021F00E9460379A83898365E070E083E497
:108A70000E94AD398AA760E085E50E94BC39259641
:108A80008FAF259760E081E09AE10E942CCAA9810E
:108A9000BA81BD01BB0F880B990B0F94476D6D8395
:108AA0007E838F8327969FAF27970F945F52688BA3
:108AB000798B8A8B9B8B1F3F09F045C420E030E007
:108AC0004CE053E46D817E818F8127969FAD27977F
:108AD0000F94927618160CF0AAC186ED99E10E94C7
:108AE0007C41CA5BDF4F0FB6F894DEBF0FBECDBF2F
:108AF000DF91CF911F910F91FF90EF90DF90CF907A
:108B0000BF90AF909F908F907F906F905F904F90AD
:108B10003F902F900D94774746E450E05A83498365
:108B20009BCF1FAEAFC12496EEADFFAD24978083DF
:108B300083C2FBEE4F2E512C612C712C04C384E1B7
:108B400090E0A0E0B0E08C8B9D8BAE8BBF8BE4E11E
:108B50004E2E512C612C712C04C34C8A5D8A6E8A76
:108B60007F8AFFC22496EEADFFAD24978083D4C3E5
:108B700089819A81AB81BC8129A93AA94BA95CA9B9
:108B8000821B930BA40BB50BB7FD59C08FAD0E9490
:108B9000DEEF8AE00E94434189819A81AB81BC81EA
:108BA0008053984FAF4FBF4F89AB9AABABABBCABC9
:108BB0009DA9911177C02EA93FA948AD59ADB1012A
:108BC000802F26969FAD26970F94927618160CF05C
:108BD00053C020E030E040E050E4B101802F269601
:108BE0009FAD26970F9432746EAB7FAB88AF99AF71
:108BF0002CA53DA54EA55FA589819A81AB81BC813D
:108C0000280F391F4A1F5B1F2AAF3BAF4CAF5DAF28
:108C100020E030E040EC50E46D817E818F8127962A
:108C20009FAD27970F9431749101402F26965FAD29
:108C300026970F94406D881F8827881F8DAB8889E1
:108C40009989AA89BB89C816D906EA06FB0610F4D9
:108C5000D701C60129813A814B815C81281B390BE0
:108C60004A0B5B0BDA01C90181389F44A241B1056F
:108C7000A8F182E299E10EC289819A81AB81BC811F
:108C80002AAD3BAD4CAD5DAD821B930BA40BB50B78
:108C900042EA5BE361EB7BE3B7FDD1CF812F0E941A
:108CA000A9F4CDCF20E030E040EF51E46D817E812A
:108CB0008F8127969FAD27970F9431749B01AC014C
:108CC000B101802F26969FAD26970F94406D87FFA8
:108CD000B6CF4EE45CE36EE57CE3E0CF4AA55BA54E
:108CE000888D998D481759070CF09EC003970CF496
:108CF0009BC085EC98E10E947C411F3F09F076C043
:108D0000A5EBB8E1BA83A98384EA98E10E947C418B
:108D100089819A810E947C41488559856A857B8535
:108D200081EC98E10E944F448AE00E94434184EA2A
:108D300098E10E947C4189819A810E947C4149A1ED
:108D40005AA16BA17CA18DEB98E10E944F448AE06F
:108D50000E94434184EA98E10E947C4189819A8182
:108D60000E947C41B501A40189EB98E10E944F4427
:108D70008AE00E9443412596FFAD2597FF2391F19C
:108D80002CEA35EC47E25EE369A17AA18BA19CA1B4
:108D90000F94A66D6B017C012CEA35EC47E25EE393
:108DA000C501B4010F942C75288539854A855B85EA
:108DB0001F3F09F52093EC083093ED084093EE082F
:108DC0005093EF08C092F008D092F108E092F208B8
:108DD000F092F3086093F4087093F5088093F60816
:108DE0009093F70881E080936A027BCEE4E3F5E498
:108DF000FA83E98389CF20934F163093501640931E
:108E0000511650935216C0925316D0925416E092B7
:108E10005516F09256166093571670935816809315
:108E2000591690935A16DECF0E9467CE80C082EC0E
:108E300099E10E947C410E949CF38FE78093EB08AC
:108E400024EB30E0A8EEB3E00F94D8736CA77DA7B5
:108E50008EA79FA7288939894A895B89260F371FE2
:108E6000481F591F2AAF3BAF4CAF5DAF10926A024B
:108E700081E08093790232E0310F3EAF323008F466
:108E800050CE1FAFC888D988EA88FB88C9AADAAA59
:108E9000EBAAFCAA812C912C540189A29AA2ABA224
:108EA000BCA288869986AA86BB868FE790E0A0E060
:108EB000B0E08C8B9D8BAE8BBF8B1C8690E49A8F21
:108EC000ACE1AB8FB6E4BC8F1D8E1E8E1F8E18A238
:108ED0003FE7432E512C612C712C1DAA8EAA9FAA0C
:108EE000A8AEB9AE1EA21FA218A619A6E1E0EDA376
:108EF000198E188E212C312C00E026961FAE269755
:108F0000F5E11F02C00111249C012A5B394E229613
:108F10003FAF2EAF2297285F3F4F24963FAF2EAF33
:108F200024974AA5042E000C550B5BA74AA78091F5
:108F30007902882309F4B0C00F945F5269837A8361
:108F40008B839C835091A60658AB552309F48BC0A4
:108F50000E944FF46091E7087091E8081F3F39F0D4
:108F60002296AEADBFAD229714966D917C91072EDF
:108F7000000C880B990B0F94476D1B01082F269648
:108F80009FAF26972D8D3E8D4F8D58A126969FAD74
:108F900026970F94927618163CF42D8E3E8E0F8FE6
:108FA0002696BFAD2697B8A32C853A8D4B8D5C8D48
:108FB000B101802F26969FAD26970F94406D87FFB5
:108FC00007C02C863A8E0B8F2696EFAD2697EC8F36
:108FD000FDA19101402F26965FAD26976D817E8180
:108FE0008F8127969FAD2797FF2309F45AC00F94CE
:108FF000406D87FF38C049815A816B817C814C1953
:109000005D096E097F09DB01CA0188589341A109F6
:10901000B109B7FD28C08C899D89AE89BF898419A3
:109020009509A609B709B595A795979587951F3F07
:1090300009F079CD8093EB084EA35FA368A779A7C9
:10904000FD81FD8F2E812E8F3F813F8F27964FAD63
:10905000279748A389819A81AB81BC81888B998BA2
:10906000AA8BBB8B1DA220E030E040EF51E46D8164
:109070007E818F8127969FAD27970F94327491013F
:10908000402F26965FAD26970F94406D87FF70CDD9
:1090900080E499E10E947C41109279020E949CF345
:1090A000A1CE0F9492761816F4F689819A81AB813D
:1090B000BC81288939894A895B89821B930BA40B5F
:1090C000B50BAC01BD01485853416109710977FDE9
:1090D000CACF488D598D452B09F40DC1CEA0DFA014
:1090E000E8A4F9A4C80ED91EEA1EFB1E2EA13FA1BA
:1090F00048A559A5281B390B4A0B5B0BC301B201CC
:109100000F947473A70196010F94A6734C885D8821
:109110006E887F88420E531E641E751E54E14516EC
:109120005104610471040CF40ACD8CEE481651040C
:10913000610471040CF0FDCC90E8491651046104FF
:1091400071040CF40ACD4C8A5D8A6E8A7F8A2EEFF8
:1091500030E040E050E0241935094609570929015B
:109160003A014C895D896E897F898AEB99E10E9479
:10917000D444B301A20185EB99E10E94D4444C850B
:109180005A8D6B8D7C8D8EEA99E10E944F444D8DF6
:109190005E8D6F8D78A187EA99E10E944F44A88D7A
:1091A000B98D13970CF4A7C0C301B2010F94476D9A
:1091B00020E030E040E850E40F94A66D4B015C01E4
:1091C0002C853A8D4B8D5C8D6D8D7E8D8F8D98A10C
:1091D0000F9431742BED3FE049E450E40F94A66DF9
:1091E00020E030E040E05FE30F94A66D9B01AC010E
:1091F000C501B4010F942C756C877D878E879F877E
:10920000C701B6010F94476D2FE632E143E85AE3F8
:109210000F94A66D6B017C011E3F59F02AE939E9D4
:1092200049E15FE3812C912CA12C6EE3B62E1F3F08
:1092300059F42DEC3CEC4CE45EE37BEA872E7AEAB1
:10924000972EA92C7EE3B72E6C857D858E859F8514
:109250000F94A66D688779878A879B879B01AC01ED
:109260000F943274A70196010F942C7569A37AA309
:109270008BA39CA3288539854A855B85C701B601E8
:109280000F94A66DA50194010F94A66D4B015C018E
:109290004C855D856E857F8581EA99E10E944F440A
:1092A000B701A6018BE999E10E944F448AE00E9430
:1092B0004341BEAD8CE899E1B23010F08DE799E101
:1092C0000E947C41488559856A857B8587E799E1BD
:1092D0000E944F4449A15AA16BA17CA181E799E169
:1092E0000E944F44B501A4018BE699E10E944F44CE
:1092F0008AE00E9443418C899D89AE89BF89840D93
:10930000951DA61DB71DB595A795979587951F3FE8
:1093100009F028CC8093EB08288D398D2F5F3F4FC3
:10932000398F288F3D813C874E814A8F5F815B8FCB
:1093300027968FAD27978C8FC980DA80EB80FC80D1
:1093400098A99DA390CEE12E012E000CFF08F701F5
:1093500083E0EE0FFF1F8A95E1F7EF58FD4F66811E
:1093600077816F507109072E000C880B990B0F94B1
:10937000476D9B01AC016D817E818F8127969FADEA
:1093800027970F94927618160CF4A7CB82EC99E1EC
:109390000E947C410E949CF385E18E9DF0018F9D8F
:1093A000F00D1124EA5BF94E8FE7808722E330E06D
:1093B00049CDCF93DF93EB010E947C41CE01DF9139
:1093C000CF910D942A323F924F925F926F927F928B
:1093D0008F929F92AF92BF92CF92DF92EF92FF92C5
:1093E0000F931F93CF93DF938091520587FD38C071
:1093F000809153058370A1F5C091E316D091E416D6
:10940000488159816A817B8185E498E10E944F44BB
:109410004C815D816E817F818AEA96E40E944F448F
:109420004091DF165091E0166091E1167091E216BE
:1094300087EA96E40E944F448AE0DF91CF911F9122
:109440000F91FF90EF90DF90CF90BF90AF909F90E3
:109450008F907F906F905F904F903F900C9443411E
:109460006090D7167090D8168090D9169090DA1622
:10947000A090DB16B090DC160091DD161091DE1680
:10948000C090DF16D090E016E090E116F090E21662
:1094900088E50E94DC37C82F882309F49AC00E940F
:1094A0006437362E472E582ED92F20E030E046E67E
:1094B00053EC0F94927687FD0DC020E030E046E635
:1094C00053E4632D742D852D9D2F0F94406D181638
:1094D0000CF081C066EE70E082E398E10E94D94909
:1094E00066EE70E08DE298E10E94D9498AE298E147
:1094F0000E947C41C0E089E50E94DC37882361F14D
:109500000E946437362E472E582ED92F20E030E0A7
:1095100046E653EC0F94927687FD0DC020E030E0D4
:1095200046E653E4632D742D852D9D2F0F94406DD9
:1095300018160CF055C066EE70E087E198E10E94C5
:10954000D94966EE70E082E198E10E94D9498FE046
:1095500098E10E947C41C0E08AE50E94DC378823C4
:1095600009F443C00E9464376B017C0120E030E0C5
:1095700040E151EC0F94927687FD0AC020E030E084
:1095800040E151E4C701B6010F94406D18166CF527
:1095900067EF7FEF8DEF97E10E94D94969E070E0B6
:1095A00088EF97E10E94D94985EF97E1DF91CF914C
:1095B0001F910F91FF90EF90DF90CF90BF90AF90F1
:1095C0009F908F907F906F905F904F903F900C9402
:1095D0007C41C1E090CF632C742C852C9D2E8BCFC9
:1095E000A32CB42C052D1D2FB7CFCC23E1F0C30144
:1095F000D4018093D7169093D816A093D916B09320
:10960000DA16C501D8018093DB169093DC16A0937F
:10961000DD16B093DE16C092DF16D092E016E0920F
:10962000E116F092E216DF91CF911F910F91FF901A
:10963000EF90DF90CF90BF90AF909F908F907F90F2
:109640006F905F904F903F9008952F923F924F926E
:109650005F926F927F928F929F92AF92BF92CF92C2
:10966000DF92EF92FF920F931F93CF93DF93CDB7CB
:10967000DEB7CB54D1090FB6F894DEBF0FBECDBF15
:109680002DB73EB739AF28AF87E00F947F2E8111F9
:109690000BC061E086E50E9456388DA3853060F0EE
:1096A0008BE89FE00E947C41A8ADB9AD0FB6F8945D
:1096B000BEBF0FBEADBF40C33DA1332321F08BE63B
:1096C0009FE00E947C416AE080E50E945638182F96
:1096D0008CEF810F8F3218F087E49FE0E3CF60E0DA
:1096E00085E40E94BC39882309F448C081E08FAB2F
:1096F000E090E316F090E416D7012D913D914D9145
:109700005C916091D3097091D4098091D5099091B1
:10971000D6090F943274AB01BC0188E50E9462380F
:1097200069877A878B879C87F701248135814681F9
:1097300057816091D7097091D8098091D90990918A
:10974000DA090F943274AB01BC0189E50E946238DA
:109750006D877E878F87988BBE01635F7F4FCE01B9
:1097600009960E944132382E81110BC063E683E3D3
:109770009FE00E942CCA8BE19FE094CF92E09FABC8
:10978000B7CF8CE40E948E37082F882309F431C1AB
:109790000E94552A8EA3803118F084EF9EE082CF7C
:1097A000FEA1F13009F427C160E083E50E94BC39D5
:1097B0008AAF882321F0011102C037E03EA38DA1BA
:1097C000833020F08AED9EE00E947C419091E20877
:1097D0009DAF80E00E948D3C0F94CE0F1D8A1E8AA3
:1097E0001F8A188E198E1A8E1B8E1C8E83EF9FE493
:1097F000A3ECB7E48D8F9E8FAF8FB8A383EF9FE468
:10980000A3ECB7EC89A39AA3ABA3BCA3A12FB0E0B0
:10981000BCA7ABA7EDB7FEB724E0129FE019F10992
:1098200011240FB6F894FEBF0FBEEDBF8DB79EB7E3
:1098300001969CAF8BAF2DA14FA9BE01635F7F4FF7
:10984000CE0109960F94F3489B01AC010F94247745
:10985000811162C20F945F526115710581059105F6
:1098600011F00F94C668212C1BAA1CAA1DAA1EAABF
:10987000AEA1A150BB0B2C96BFAFAEAF2C97E22D83
:10988000F0E0F8A7EFA32BA53CA5E217F3070CF037
:1098900074C23196FEA7EDA73F932F93FF93EF93EA
:1098A00086EC9EE09F938F9380ED9EE09F938F9335
:1098B0001F920E9411CA8DB79EB709960FB6F894F1
:1098C0009EBF0FBE8DBF9EA1992309F458C10F946E
:1098D00077682AE030E040E050E00F94A6730F94E0
:1098E000476D20E030E040EA50E40F9492760FEFAD
:1098F0001FEF181614F001E010E00F94776828E6C7
:1099000031E040E050E00F94A6730F94476D2B01B7
:109910003C010F94776827E130E040E050E00F947D
:10992000A6736B5F7F4F8F4F9F4F0F94476D4B0117
:109930005C01ADA1A430D1F4BC01A40188EB9EE090
:109940000E944F44B301A20180EB9EE00E944F446D
:109950008AEA9EE00E947C410130110519F483E4FB
:109960000E94434186EA9EE00E947C41312CC8015E
:10997000110FAA0BBB0B2A968CAF9DAFAEAFBFAF3A
:109980002A972C96AEADBFAD2C973A161B060CF05D
:10999000F6C02A966CAD7DAD8EAD9FAD2A970F9423
:1099A000476D6B017C01BAADBB2341F1AC019B015A
:1099B0000F94327420E030E040E952E40F94A66D39
:1099C0009B01AC01C301B2010F9432742B013C0125
:1099D00020E030E044EB53E40F9492761816FCF448
:1099E00020E030E044EB53E4C301B2010F94317442
:1099F000EDCF1EA2D9CE22E02EA3D6CE0F9477684B
:109A000024E130E040E050E00F94A673675E7F4FA2
:109A10008F4F9F4F0F94476DA7019601CFCF20E046
:109A200030E0A901C301B2010F94406D87FF0BC064
:109A300020E030E044EB53E4C301B2010F943274F0
:109A40002B013C01ECCF0091E3161091E416F801D4
:109A500024813581468157816D857E858F859889E2
:109A60000F94317422966CAF7DAF8EAF9FAF22976B
:109A70002BED3FE049E450E4C301B2010F94A66D21
:109A800020E030E044E353E40F942C756B017C013B
:109A90000F9427756FA778AB89AB9AABD8012D913E
:109AA0003D914D915C9169857A858B859C850F945C
:109AB000317426966CAF7DAF8EAF9FAF2697A50110
:109AC00094016FA578A989A99AA90F94A66D9B0105
:109AD000AC0126966CAD7DAD8EAD9FAD26970F94F3
:109AE000327469837A838B839C83C701B6010F9498
:109AF000D276A50194010F94A66D22962CAD3DADB2
:109B00004EAD5FAD22970F9432746D837E838F8349
:109B1000988740EF50E070E060E0CE0101960E942F
:109B200067F440EF50E070E060E0CE0105960E94DF
:109B300067F4BDA1B43099F449815A816B817C816D
:109B40008AE99EE00E944F444D815E816F81788555
:109B50008AEA96E40E944F448AE00E944341198AAF
:109B60001A8A1B8A1C8AAE014F5E5F4FBE016B5F73
:109B70007F4FCE0101960F94C410339402CF20E0A2
:109B80004FA9BE01635F7F4FCE0109960F94F34842
:109B90004B015C01312CAC019B010F9424778111A6
:109BA00002C033243394A5019401C501B4010F947C
:109BB00024778111E2C0EFA1F8A5EE0FFF1FEE0F91
:109BC000FF1F2BAD3CADE20FF31F80829182A2827A
:109BD000B382A50194016D8D7E8D8F8D98A10F9418
:109BE0009276181624F48D8E9E8EAF8EB8A2A501A3
:109BF000940169A17AA18BA19CA10F94406D87FF6C
:109C000004C089A29AA2ABA2BCA2A50194016BA92F
:109C10007CA98DA99EA90F9432746BAB7CAB8DABE4
:109C20009EABADA5BEA5BD01BB0F880B990B0F94D4
:109C3000476D6FA378A789A79AA79B01AC016BA971
:109C40007CA98DA99EA90F942C752B013C014D8AEE
:109C50005E8A6F8A788EEBADFCADF8ABEFA710E0B3
:109C6000C12CD12C7601AFA5B8A96D917D918D91B4
:109C70009D91B8ABAFA7A30192010F9431749B01E2
:109C8000AC010F94A66D9B01AC01C701B6010F9406
:109C900032746B017C011F5F211628F72FA138A5B4
:109CA00049A55AA50F942C750F94E076698F7A8F89
:109CB0008B8F9C8FBDA1B23068F18DA59EA50F94AE
:109CC0002A326BA57CA585E99EE00E94D9498FE8E0
:109CD0009EE00E947C4143E0C501B4010E943AEF3E
:109CE00080E20E94434181E0EDA1E3300CF480E08A
:109CF000E12C8E010F5D1F4F9E01235E3F4FAE0191
:109D0000475E5F4FBE016B5E7F4F0E94C1428AE09B
:109D10000E9443412394B3CD0E9438320F94B50F73
:109D20008DAD0E948D3C0F948B1988AD99AD0FB607
:109D3000F8949EBF0FBE8DBFE8ADF9AD0FB6F89495
:109D4000FEBF0FBEEDBFC55BDF4F0FB6F894DEBFA1
:109D50000FBECDBFDF91CF911F910F91FF90EF907C
:109D6000DF90CF90BF90AF909F908F907F906F903B
:109D70005F904F903F902F9008950E94383233208B
:109D800069F284E89EE00E947C4181E0FDA11F16FB
:109D90000CF080E0EE24E3948E010F5D1F4F9E01D6
:109DA000235E3F4FAE01475E5F4FBE016B5E7F4F4C
:109DB0000E94C142698D7A8D8B8D9C8D0052110954
:109DC00026E042E00F940D689F938F9383E79EE017
:109DD0009F938F938DE79EE09F938F931F920E9496
:109DE00011CA2DB73EB7295F3F4F0FB6F8943EBF5B
:109DF0000FBE2DBF93CF2F923F924F925F926F92E3
:109E00007F928F929F92AF92BF92CF92DF92EF920A
:109E1000FF920F931F93CF93DF93CDB7DEB7CC584C
:109E2000D1090FB6F894DEBF0FBECDBF84E69DE02A
:109E30000E947C4187E00F947F2E81118FC084E5C2
:109E40000E94DC37882329F00E94603781110E942C
:109E500028EF80E090E0A0E8BFE389839A83AB839A
:109E6000BC838D839E83AF83B8878DEC9CECACE480
:109E7000BEE389879A87AB87BC8780E090E0A0E249
:109E8000B1E48D879E87AF87B88B8CE390E09A8B87
:109E9000898B8DEC90E09C8B8B8B8DEC9CECACECEF
:109EA000BEE38D8B9E8BAF8BB88F80E090E0A0EEF1
:109EB000BFE3898F9A8FAB8FBC8F1BA61CA64AE984
:109EC00059E969E97EE38FE40E9462386D8F7E8FE5
:109ED0008F8F98A360E083E40E94BC3989A360E07F
:109EE0008BE40E94BC398AA389E40E94DC3710E02D
:109EF000F12CE12C8823C1F00E94552A90E018161D
:109F0000190614F481E090E011E0180F212F215080
:109F1000330BC90126E0289FF001299FF00D112481
:109F2000EC58F74FE280F38082E40E94DC3788230C
:109F300019F00E9460377C01E114F10459F1C70166
:109F400088978536910520F16CE870E086E39DE006
:109F50000E94D94981E39DE00E947C41C457DF4FB4
:109F60000FB6F894DEBF0FBECDBFDF91CF911F912A
:109F70000F91FF90EF90DF90CF90BF90AF909F90A8
:109F80008F907F906F905F904F903F902F900895AB
:109F9000FA8AE98A8CE40E94DC378823E1F00E9487
:109FA00064376B017C01C986DA86EB86FC8620E08B
:109FB00030E0A9010F94927687FD0AC020E030E0DE
:109FC00040E050E4C701B6010F94406D18161CF430
:109FD00089E09DE0C1CF81E50E948E37882331F171
:109FE0008091220590912305892BE9F00E94643726
:109FF0006B017C01CD82DE82EF82F8862DEC3CEC99
:10A000004CE45DE30F94927687FD0AC020E030E0D7
:10A0100040E751E4C701B6010F94406D181634F4BF
:10A0200088ED9CE099CF8DEA9CE096CF83E50E9475
:10A03000DC378823E9F00E9464376B017C01CD8A0C
:10A04000DE8AEF8AF88E2DEC3CEC4CEC5DE30F944D
:10A05000927687FD0AC020E030E040E050E4C7017E
:10A06000B6010F94406D18161CF486E89CE074CF7E
:10A0700080E50E948E37882341F0809122059091DF
:10A080002305892B29F58FEF8BA786E40E94DC3707
:10A09000882309F43DC00E9464376B017C01C98E9E
:10A0A000DA8EEB8EFC8E20E030E040E85FE30F9428
:10A0B000927687FD0AC020E030E040E850E4C70116
:10A0C000B6010F94406D18161CF585E39CE044CF53
:10A0D0008BA58F5F8BA70E9464376B017C01CD86B7
:10A0E000DE86EF86F88A20E030E0A9010F949276B0
:10A0F00087FD0BC020E030E048EC51E4C701B60119
:10A100000F94406D18160CF0C0CF8EE59CE024CF64
:10A11000C98CDA8CEB8CFC8C8D889E88AF88B88CCF
:10A12000A7019601C701B6010F94A66D9B01AC0172
:10A1300060E070E084E490E40F942C7529813A810A
:10A140004B815C810F94A66D2B013C01A50194010C
:10A15000C501B4010F94A66DA70196010F94A66DD9
:10A160002CEE31E548EB5DE30F942C759B01AC01BF
:10A17000C301B2010F94A66D69837A838B839C839C
:10A18000112309F1412F4150550B26E0249FF00186
:10A19000259FF00D1124EC58F74F0081118188E4C0
:10A1A0000E94DC37882319F00E9460378C0101156A
:10A1B000110571F0C801855A91098838910530F070
:10A1C00087E09CE0C9CE10E000E0E9CF1C8B0B8B50
:10A1D00085E50E948E378823C9F00F945F52611580
:10A1E00071058105910511F00F94C66880912205D3
:10A1F00090912305892BC9F00E946437609316055E
:10A200007093170580931805909319056AE170E023
:10A2100082E50E94AD39AD969FAF8EAFAD9718160F
:10A22000190644F083ED9BE097CE60E070E088E48F
:10A2300092E4E4CF89E50E94DC37882381F10E9413
:10A2400064372091CB093091CC094091CD095091D0
:10A25000CE090F9431746B017C0188E50E94DC37D4
:10A26000882331F10E9464372091C7093091C809D1
:10A270004091C9095091CA090F9431746BA37CA312
:10A280008DA39EA3CFA2D8A6E9A6FAA6CE01839657
:10A290000E949924811115C089EA9BE05DCEC0908F
:10A2A000D709D090D809E090D909F090DA09D5CF34
:10A2B0006091D3097091D4098091D5099091D60904
:10A2C000DDCF84E40E948E3711E081270E948D3C0F
:10A2D00080E090E0A0EAB0E48DA79EA7AFA7B8AB5E
:10A2E00060E0CE018D960F9405115091FC08CD577A
:10A2F000DF4F5883C358D0401092FC080E9436DCD0
:10A3000086E59BE00E947C4189899A894A970CF0F6
:10A3100091C063E683E39BE00E942CCA0F9498529D
:10A320008B899C890E94AEFA41E061E080E00E9446
:10A33000D6F1882309F491C00F9477470F9498526F
:10A340001092DF091092E0091092E1091092E209DF
:10A350008FED99E00F94CF0C1BA5112309F4E2C0F7
:10A3600020E030E040E751E460910C1170910D1154
:10A3700080910E1190910F110F942C7521966CAF56
:10A380007DAF8EAF9FAF21971F3F09F00DC581E0D4
:10A3900080935D0563E68BE89BE00E942CCA68E829
:10A3A00073E182E090E00E94539580E1E3EDF9E0F3
:10A3B000A8EAB8E001900D928A95E1F7CE010196E6
:10A3C0000F94E04AC12CD12C76018091E70982FDDF
:10A3D0009EC068E873E182E090E00E94539520E01F
:10A3E00030E040E85EE36091B4087091B508809178
:10A3F000B6089091B7080F9432746093B4087093C4
:10A40000B5088093B6089093B70820E030E040E8A4
:10A410005EE3C701B6010F9432746B017C0120E04A
:10A4200030E84BE354E40F94927687FD60C01092BD
:10A430005D0513C063E686E49BE00E942CCA0F947E
:10A44000985210935D0589899A890E94553761E079
:10A4500081E00E9451F081115CCF6FEF8DE99BE0AC
:10A460000E942CCA8CA5811112C081E08CA78D811D
:10A470009E81AF81B885B0588DA79EA7AFA7B8AB16
:10A48000BE01635D7F4F88EA98E00E94EA3380E076
:10A4900090E0A0EAB0E48093B0089093B108A09354
:10A4A000B208B093B3081DA61EA61FA618AABE0127
:10A4B000635D7F4F88EA98E00E94EA33CD57DF4F13
:10A4C0005881C358D0405093FC080E9436DC10924B
:10A4D0005D058AA1811142CD1092EA081092E90827
:10A4E0000E94CEDC90E080E00E94AEFA37CDCE0133
:10A4F000CD960F94FB1880E1E3EDF9E0A8EAB8E00F
:10A5000001900D928A95E1F70E942CFB5ECF0E948C
:10A5100026D163E68EE79BE00E942CCA0F949852E6
:10A5200010925D05E1E1F5E085E0DF011D928A957D
:10A53000E9F780E1E3EDF9E0A8EAB8E001900D92D7
:10A540008A95E1F789859A85AB85BC858093B008AB
:10A550009093B108A093B208B093B3081DA61EA6AD
:10A560001FA618AABE01635D7F4F88EA98E00E948B
:10A57000EA33BE01635E7F4F88EA98E00E94EA33C7
:10A5800081E080935D0589A1882309F463C420914B
:10A59000D3093091D4094091D5095091D609E59657
:10A5A0002CAF3DAF4EAF5FAFE5978091D70990914B
:10A5B000D809A091D909B091DA09E1968CAF9DAF85
:10A5C000AEAFBFAFE197312C212C9FEFA4969FAF88
:10A5D000A497AFEFA896AFAFA897BFEFC158DF4FD2
:10A5E000B883CF57D040EFE4C058DF4FE883C0585E
:10A5F000D040F3ECCF57DF4FF883C158D04027E469
:10A60000CE57DF4F2883C258D04081E090E0A0E0D1
:10A61000B0E0022C04C0880F991FAA1FBB1F0A9428
:10A62000D2F7CC57DF4F88839983AA83BB83C45862
:10A63000D040A1E1B5E0E796BFAFAEAFE79710E03D
:10A6400000E09101032C000C440B550BC857DF4F61
:10A65000288339834A835B83C858D040C457DF4F6F
:10A660002882CC58D040E796AEADBFADE7978D912C
:10A67000E796BFAFAEAFE79790E0B0E0A0E0CC5771
:10A68000DF4F288139814A815B81C458D0408223C1
:10A690009323A423B523892B8A2B8B2B09F024C168
:10A6A000C857DF4F688179818A819B81C858D04023
:10A6B0000F94476D2091890630918A0640918B0650
:10A6C00050918C060F94A66D2091810630918206E0
:10A6D00040918306509184060F943274EB966CAFD0
:10A6E0007DAF8EAF9FAFEB97B801012E000C880BAA
:10A6F000990B0F94476D20918D0630918E064091F5
:10A700008F06509190060F94A66D2091850630918A
:10A71000860640918706509188060F9432746B012B
:10A720007C01EB962CAD3DAD4EAD5FADEB97E59664
:10A730006CAD7DAD8EAD9FADE5970F9431742B015F
:10A740003C01A7019601E1966CAD7DAD8EAD9FAD4C
:10A75000E1970F9431744B015C01A3019201C30195
:10A76000B2010F94A66D2B013C01A5019401C50116
:10A77000B4010F94A66D9B01AC01C301B2010F940B
:10A7800032740F94E0764B015C01EB962CAD3DAD3D
:10A790004EAD5FADEB976BA17CA18DA19EA10F94F7
:10A7A00031742B013C01A70196016FA178A589A501
:10A7B0009AA50F9431746B017C01A3019201C3012E
:10A7C000B2010F94A66D2B013C01A7019601C701B0
:10A7D000B6010F94A66D9B01AC01C301B2010F94A9
:10A7E00032740F94E07620E030E040E751E40F94BB
:10A7F0002C75A50194010F9432746B017C0180903B
:10A80000160590901705A0901805B090190520E046
:10A8100030E040E85FE3C501B4010F94927618166A
:10A82000F4F4C501B4010F949E754B015C0160E026
:10A8300070E0CB01181419041A041B0434F40F94AB
:10A840007768A50194010F94A6730F94476D9B013F
:10A85000AC01B601C7010F9432746B017C01C15881
:10A86000DF4F2881CF57D040C058DF4F3881C058C4
:10A87000D040CF57DF4F4881C158D040CE57DF4F2F
:10A880005881C258D040B601C7010F94406D87FF70
:10A890002BC0A4960FAFA497C457DF4F3881CC5874
:10A8A000D040A8963FAFA897EC96CFAEEC97ED9628
:10A8B000DFAEED97EE96EFAEEE97EF96FFAEEF9729
:10A8C000C158DF4FC882CF57D040C058DF4FD88221
:10A8D000C058D040CF57DF4FE882C158D040CE5744
:10A8E000DF4FF882C258D0400F5F1F4F053011056F
:10A8F00009F0B9CE4FEF241A340A55E02516310479
:10A9000009F083CEA4968FADA497E82FF0E0EF5E18
:10A91000FA4F208181E090E0A0E0B0E0A8960FAC73
:10A92000A89704C0880F991FAA1FBB1F0A94D2F7CB
:10A93000822B8083A8969FADA8976A969FAF6A974F
:10A94000A496AFADA4976B96AFAF6B97EC968FAD17
:10A95000EC97ED969FADED97EE96AFADEE97EF9637
:10A96000BFADEF976F968CAF9DAFAEAFBFAF6F9798
:10A97000A896BFADA897BF3F09F4FAC1A496EFAD62
:10A98000A497EF3F09F4F4C16B2FBB0F770B880B33
:10A99000990B0F94476D2091890630918A0640915A
:10A9A0008B0650918C060F94A66D209181063091F4
:10A9B000820640918306509184060F943274162FBC
:10A9C000072F382E292E862F902FA32DB22D659676
:10A9D0008CAF9DAFAEAFBFAF6597A496FFADA49708
:10A9E0006F2FFF0F770B880B990B0F94476D2091FA
:10A9F0008D0630918E0640918F06509190060F94EF
:10AA0000A66D20918506309186064091870650916B
:10AA100088060F9432746B017C016996CCAEDDAE72
:10AA2000EEAEFFAE6997CE018F5A9F4F0E949924D8
:10AA3000882309F4A1C120E030E040EA50E4612F0E
:10AA4000702F832D922D0F9432744B015C01CB013A
:10AA5000D50121968CAF9DAFAEAFBFAF21972596A4
:10AA6000CCAEDDAEEEAEFFAE2597A8962FADA89783
:10AA700021112AC2A4963FADA4973111FAC120E05A
:10AA800030E040EA50E4C701B6010F9432746B0124
:10AA90007C01A4964FADA497442309F40CC2A4965C
:10AAA0008FADA49784300CF006C222ED422E23E530
:10AAB000522E2BE7622E21E4722E21968CAC9DAC97
:10AAC000AEACBFAC219725968CAD9DADAEADBFAD04
:10AAD0002597A7968CAF9DAFAEAFBFAFA7979C0150
:10AAE000AD0169966CAD7DAD8EAD9FAD69970F944C
:10AAF0003174AB966CAF7DAF8EAF9FAFAB97A501B6
:10AB0000940165966CAD7DAD8EAD9FAD65970F944C
:10AB100031742D966CAF7DAF8EAF9FAF2D97AB96F6
:10AB20002CAD3DAD4EAD5FADAB9761962CAF3DAF5B
:10AB30004EAF5FAF6197A50194016091D309709109
:10AB4000D4098091D5099091D6090F9431744B01A5
:10AB50005C01A7962CAD3DAD4EAD5FADA797609162
:10AB6000D7097091D8098091D9099091DA090F9489
:10AB70003174A7966CAF7DAF8EAF9FAFA797812F33
:10AB8000902FA32DB22D8DA79EA7AFA7B8ABC9AAB2
:10AB9000DAAAEBAAFCAAC984DA84EB84FC84CDAAE5
:10ABA000DEAAEFAAF8AE2DEC3CEC4CEC5CE3C30162
:10ABB000B2010F94A66D29813A814B815C810F947B
:10ABC000A66D2091DF093091E0094091E109509193
:10ABD000E2090F94327469AF7AAF8BAF9CAFA501D5
:10ABE0009401C501B4010F94A66D4B015C01A796B9
:10ABF0002CAD3DAD4EAD5FADA797CA01B9010F9425
:10AC0000A66D9B01AC01C501B4010F94327420E024
:10AC100030E040E050E40F9492761816ACF420E057
:10AC200030E040E05FE3C701B6010F94327429962B
:10AC30006CAF7DAF8EAF9FAF2997BE01635C7F4F36
:10AC4000CE0101960E94F33389859A85AB85BC8538
:10AC500029968CAF9DAFAEAFBFAF2997A3961CAE20
:10AC60001DAE1EAE1FAEA397BE01615A7F4FCE012F
:10AC7000CD960E94EA33CE0101960F94E04AE0900F
:10AC80000411F09005110091061110910711A09088
:10AC90000011B0900111C0900211D09003119501E4
:10ACA000A601B701C8010F949276181614F4750125
:10ACB00086018090850290908602A0908702B090D5
:10ACC00088022DEC3CEC4CEC5DE3B701C8010F941D
:10ACD000A66D60938502709386028093870290939D
:10ACE000880240E0BE01675B7F4FCE018D960F94D6
:10ACF000595380E1E3EDF9E0A8EAB8E001900D9244
:10AD00008A95E1F78092850290928602A09287024E
:10AD1000B09288020E94342A81119FCB20E04FEF2D
:10AD2000BE01675A7F4FCE0101960E94B63520E0E2
:10AD300041E0BE01675A7F4FCE0101960E94B635B1
:10AD40002FEF40E0BE01675A7F4FCE0101960E946F
:10AD5000B63521E040E0BE01675A7F4FCE01019633
:10AD60000E94B6350E942CFB0E94342A811175CBBB
:10AD70008091241180932511AD964EAD5FADAD97B6
:10AD800041505109AD965FAF4EAFAD97452B09F4D9
:10AD900064CB6A968FAD6A9787FD5FCB6B968FAD5C
:10ADA0006B9787FFF0CB59CB63E68BE69BE00E9465
:10ADB0002CCA0F94985280E1E3EDF9E0A8EAB8E0DC
:10ADC00001900D928A95E1F72D853E854F85588932
:10ADD0006091B4087091B5088091B6089091B70859
:10ADE0000F9432746093B4087093B5088093B608DA
:10ADF0009093B708CE01CD960F94FB182D853E8514
:10AE00004F8558896091B4087091B5088091B60853
:10AE10009091B7080F9431746093B4087093B5089B
:10AE20008093B6089093B7088CA581117BCB81E005
:10AE30008CA78D819E81AF81B885B0588DA79EA7C4
:10AE4000AFA7B8ABBE01635D7F4F88EA98E00E9470
:10AE5000EA3368CB2BA13CA14DA15EA1E5962CAFB6
:10AE60003DAF4EAF5FAFE5978FA198A5A9A5BAA555
:10AE7000A4CB812F902FA32DB22D21968CAF9DAF07
:10AE8000AEAFBFAF219720E030E040EA50E4C70109
:10AE9000B6010F94317425966CAF7DAF8EAF9FAF26
:10AEA0002597A4965FADA49754300CF4E8CD182DE7
:10AEB000092D3A2C2B2C92ED492E93E5592E9BEF20
:10AEC000692E90E4792EF9CDA8969FADA89794307D
:10AED0000CF452C0A496AFADA497A4300CF120E0BE
:10AEE00030E040EA50E4612F702F832D922D0F94B3
:10AEF000317421966CAF7DAF8EAF9FAF219720E06C
:10AF000030E040EA50E4C701B6010F9431746B01A0
:10AF10007C01A496EFADA497E4300CF4C6CDCBCF62
:10AF2000812F902FA32DB22D21968CAF9DAFAEAF68
:10AF3000BFAF219720E030E040EA50E4C701B601FE
:10AF40000F94327425966CAF7DAF8EAF9FAF25976F
:10AF5000A496BFADA497B111D2CF20E030E040EA73
:10AF600050E4612F702F832D922D0F943174162F82
:10AF7000072F382E292E9FCFA496FFADA497F1114D
:10AF80000DC020E030E040E251E4B401C5010F946F
:10AF90003174162F072F382E292E87CDA4962FAD6A
:10AFA000A49724309CF020E030E040E251E4B4016A
:10AFB000C5010F94317421966CAF7DAF8EAF9FAFFA
:10AFC0002197182D092D3A2C2B2C6FCD182D092DDA
:10AFD0003A2C2B2C82ED482E83E5582E8BEF682ED1
:10AFE00081E4782E6ACD88EA99E00C947C4182EA6B
:10AFF00099E00C947C41CF92DF92EF92FF928AE528
:10B000000E94DC37882309F45AC00E94643720E08C
:10B0100030E040E050EC0F94406DC12CD12CE12C7D
:10B0200090ECF92E87FD0FC00E94643720E030E0DD
:10B0300040E050E40F94927618160CF462C00E941F
:10B0400064376B017C012091F8103091F910409128
:10B05000FA105091FB10C701B6010F94A66D0F9422
:10B060009E75CB010F94135380E50E948E3781119A
:10B070004EC0A70196016091DF167091E016809195
:10B08000E1169091E2160F9432746093DF1670937C
:10B09000E0168093E1169093E2160E94F7574091D4
:10B0A000DF165091E0166091E1167091E21686EE7F
:10B0B00097E10E944F448AE00E94434105C083E526
:10B0C0000E94DC378111A1CF8091520587FD24C0F9
:10B0D00080915305837001F50E94F7574091DF1668
:10B0E0005091E0166091E1167091E21687ED97E1BC
:10B0F0000E944F448AE0FF90EF90DF90CF900C9435
:10B100004341C12CD12CE12C80E4F82E9CCF0E942D
:10B11000692A8111AECFD8CF82E50E948E37811186
:10B12000DBCFFF90EF90DF90CF900895CF9384E531
:10B130000E94DC37C0E08823D9F00E94552AC82F2E
:10B140001816B4F40E94F7578DE40E944341809191
:10B150004D0590914E050F94E55C6C2FCC0F770B4D
:10B1600082EF90E10E94D9498AE00E944341CFEFEB
:10B170008C2FCF9108954F925F926F927F928F9212
:10B180009F92AF92BF92CF92DF92EF92FF92CF93B6
:10B19000DF93CDB7DEB72C970FB6F894DEBF0FBEA6
:10B1A000CDBF4090C7095090C8096090C909709000
:10B1B000CA092091410230914202409143025091CC
:10B1C0004402C301B2010F94327469837A838B8382
:10B1D0009C838090CB099090CC09A090CD09B09031
:10B1E000CE0920914502309146024091470250918C
:10B1F0004802C501B4010F9432746D837E838F833E
:10B200009887C090CF09D090D009E090D109F090F4
:10B21000D2092091490230914A0240914B0250914B
:10B220004C02C701B6010F94327469877A878B8705
:10B230009C8720914D0230914E0240914F025091D7
:10B240005002C301B2010F9432742B013C012091D2
:10B250005102309152024091530250915402C50163
:10B26000B4010F9432744B015C012091550230916E
:10B2700056024091570250915802C701B6010F94EF
:10B2800032746B017C010E94F75783E490E10E94C5
:10B290007C4183E50E948E37882321F00E94692A31
:10B2A00080933F0280913F02811151C085E195E179
:10B2B0000E947C418BE390E10E947C4149815A814C
:10B2C0006B817C8184E791E30E944F444D815E81D4
:10B2D0006F8178858AEA96E40E944F4449855A85B1
:10B2E0006B857C8587EA96E40E944F4489E390E170
:10B2F0000E947C4181E390E10E947C41B301A20164
:10B3000084E791E30E944F44B501A4018AEA96E4E0
:10B310000E944F44B701A60187EA96E40E944F4479
:10B320008AE02C960FB6F894DEBF0FBECDBFDF913A
:10B33000CF91FF90EF90DF90CF90BF90AF909F9014
:10B340008F907F906F905F904F900C94434189E174
:10B3500095E1AECF2F923F924F925F926F927F9284
:10B360008F929F92AF92BF92CF92DF92EF92FF9215
:10B370000F931F93CF93DF93CDB7DEB76A970FB6C6
:10B38000F894DEBF0FBECDBF83E50E948E37182F25
:10B390003090E208882319F00E94692A382E4090E4
:10B3A000D3095090D4096090D5097090D609809146
:10B3B000D7099091D809A091D909B091DA098B8B5E
:10B3C0009C8BAD8BBE8B8091DB099091DC09A091A9
:10B3D000DD09B091DE098F8B988FA98FBA8F112369
:10B3E00029F0311003C080E00E948D3C86E50E9468
:10B3F0008E37888B20E030E0A9016091890670913A
:10B400008A0680918B0690918C060F94406D88235C
:10B4100009F4C5C083E40E948E37882309F498C0DC
:10B420000E9464376B017C01ADE1B6E0B987A88763
:10B43000BF83AE83F5E0FD831D861E8628EC2F8733
:10B4400002EC1A86212C88EC8B8792E49C87AE81D3
:10B45000BF81BA8BA98B15E0E989FA898190919017
:10B46000A190B190FA8BE98B2A85322D4B855C85B2
:10B47000C501B4010F94406D87FF04C08A86292C52
:10B48000AB86BC862D853E854F85502FC501B40106
:10B490000F949276181624F48D869E86AF860B2D17
:10B4A0001150D1F6FD81F150FD838E819F8144962C
:10B4B0009F838E83F111CBCF2D853E854F85502FF5
:10B4C0006A85722D8B859C850F94327420E030E064
:10B4D00040E05FE30F94A66DA70196010F943274CC
:10B4E0006B017C012DEB37E346E855EB0F94927628
:10B4F00087FD0AC02DEB37E346E855E3C701B601E7
:10B500000F94406D181624F580E00E948D3C15E0E4
:10B51000A884B98405E0D5016D917D918D919D91AF
:10B520005D014D01B4E08B1A9108A70196010F94BB
:10B530003174F4016083718382839383015059F7DE
:10B540001150888599854496998788871111E0CF95
:10B55000A889AA2381F020E030E0A9016091890642
:10B5600070918A0680918B0690918C060F94406DA5
:10B5700081110E94C4438AE50E948E37882359F0C6
:10B580000E94643769837A838B839C8360E0CE0159
:10B5900001960E941F3D832D0E948D3C0BC03110EF
:10B5A00003C09889992339F30E94F75784EB9DE0F3
:10B5B0000E947C41332051F08091E208811106C045
:10B5C0000E94F35785E99DE00E947C410E94F75755
:10B5D00087E89DE00E947C418091E208811172C061
:10B5E00085E195E10E947C418AE00E9443410E94EE
:10B5F000F7578AE79DE00E947C41C090DE08D0901A
:10B60000DF08E090E008F090E10820E030E0A901D8
:10B61000C701B6010F94927618160CF056C042E09E
:10B62000C701B6010E943AEF8DE00E9443418AE0D3
:10B630000E944341A30192016091D3097091D40902
:10B640008091D5099091D6090F94406D81111FC04A
:10B650002B893C894D895E896091D7097091D80901
:10B660008091D9099091DA090F94406D81110FC032
:10B670002F89388D498D5A8D6091DB097091DC09D5
:10B680008091DD099091DE090F94406D81110F9436
:10B690008B196A960FB6F894DEBF0FBECDBFDF914F
:10B6A000CF911F910F91FF90EF90DF90CF90BF90BF
:10B6B000AF909F908F907F906F905F904F903F9052
:10B6C0002F90089589E195E18DCF85E79DE00E9457
:10B6D0007C41B0CFCF93C82F82E0C11184E040E01D
:10B6E00060E00E94819B0E94F7578DE79AE0CC238F
:10B6F00011F082E99AE0CF910C947C410E949CF376
:10B700000E94FF3E80E00F9499478091730881303A
:10B71000A1F40E94F3578BE299E00E947C4160E023
:10B7200081E299E00E942CCA6EE571E080E090E031
:10B730000E94793E88E0809373080895CF92DF924B
:10B74000EF92FF921F93CF93DF9300D01F92CDB75C
:10B75000DEB78EEEC82E82E0D82EE12CF12CC98205
:10B76000DA82EB82FC82BE016F5F7F4F8AE50E9426
:10B770005B4081110EC010E0812F0F900F900F9051
:10B780000F90DF91CF911F91FF90EF90DF90CF90BE
:10B7900008950E94CC40C982DA82EB82FC82BE010D
:10B7A0006F5F7F4F8AE50E945B40182F882319F353
:10B7B0000E94F35785E09AE00E947C410E947E5BE4
:10B7C000DBCFCF92DF92EF92FF921F93CF93DF9365
:10B7D00000D01F92CDB7DEB78EEEC82E82E0D82EF5
:10B7E000E12CF12CC982DA82EB82FC82BE016F5F10
:10B7F0007F4F8AE00E945B4081110EC010E0812FD4
:10B800000F900F900F900F90DF91CF911F91FF90AD
:10B81000EF90DF90CF9008950E94CC400E947B4033
:10B820000E9496400E947B40C982DA82EB82FC82B1
:10B83000BE016F5F7F4F8AE00E945B40182F882314
:10B84000E9F20E94F35788EC99E00E947C410E9443
:10B850007E5BD5CFFF920F931F93CF93DF93EC01C5
:10B860008B01F42E0E949CF30E94F35781E099E033
:10B870000E947C410115110511F404E315E42097A1
:10B8800011F4C8EFD8E00E9419D11F930F93DF93F2
:10B89000CF9388EE98E09F938F9381E08F930E94DF
:10B8A00011CA0E94989AC0912517C695C69580E244
:10B8B00097E10E94372DDC2FDD0F1D2F1C0FEDB7F8
:10B8C000FEB737960FB6F894FEBF0FBEEDBF83E00C
:10B8D0000E941B2C4BED53E16C2F80E00E94E22F65
:10B8E00010925B17D0935C1789ED98E00E94C72DEA
:10B8F00010925B1710935C178CEC98E00E94C72D98
:10B9000084E297E10F94525A8111E1CF61E08FEE0A
:10B9100098E00E943F4389EE93E030E6019729F0DA
:10B92000232F2A950000E9F7F9CFF89489EE93E0E8
:10B9300038EE019729F0232F2A950000E9F7F9CF77
:10B940000E949CF3FF2041F00E94AF3E0E946C26B3
:10B95000909905C0A895FCCF0E946A26F7CF909BCE
:10B9600002C0A895FCCFF0E0E0E0DF91CF911F91FD
:10B970000F91FF9019945F926F927F928F929F9296
:10B98000AF92BF92CF92DF92EF92FF920F931F93ED
:10B99000CF93DF931F92CDB7DEB77C0139018B01C6
:10B9A0005B01A40EB51ED12CC12CA016B10609F462
:10B9B00050C0F70180809180F80151908F01598229
:10B9C000C4010F945E735816B9F1652DC4010F942C
:10B9D0006673FFEFCF1ADF0AC6018F779927892B8D
:10B9E00021F162E070E080E090E00F942C52C401FD
:10B9F0000F945E7399818917F9F00E94F7578BE6CF
:10BA000096E00E947C4181E00F90DF91CF911F91E1
:10BA10000F91FF90EF90DF90CF90BF90AF909F90ED
:10BA20008F907F906F905F90089562E070E080E06B
:10BA300090E00E94793EDBCFBE016F5F7F4FC30174
:10BA40000F947330F70180819181019691838083F7
:10BA5000ACCF80E0D9CF80912411909125112FEFA8
:10BA60003FEF981751F0E92FF0E0EC5DFE4E228198
:10BA700030E09F5F9F7790932511C90108951F9231
:10BA80000F920FB60F9211240F900FBE0F901F90C0
:10BA900018951F920F920FB60F9211240BB60F92AA
:10BAA0002F933F934F935F936F937F938F939F93C6
:10BAB000EF93FF939091C60050912511309124117E
:10BAC00041E0430F4F772091AD04213108F099C038
:10BAD000E22FF0E08827E059F24A8F4F0D94297445
:10BAE000815DAA5DB95DC85DCF5D015ED35D015E1C
:10BAF000D75DDB5D015EDF5DE35DE75DEE5D015E11
:10BB0000F95D903229F0F8F49A3011F09D3001F58A
:10BB1000541731F0E32FF0E0EC5DFE4E9283342FAA
:10BB200030932411FF91EF919F918F917F916F91AD
:10BB30005F914F913F912F910F900BBE0F900FBED1
:10BB40000F901F9018959D3481F081E09E3471F024
:10BB500080E10CC09A3338F49033D0F69032C1F2C1
:10BB60009D32B1F7D5CF9D3499F782E08093AD0433
:10BB7000CFCF913359F018F4903251F2E9CF88E0E9
:10BB80009433A1F38BE0983389F3E2CF83E0EECFD7
:10BB900084E0903359F386E0913341F3D9CF85E0C7
:10BBA0009833B1F6E3CF87E0923391F6DFCF89E0A7
:10BBB000913371F6DBCF8AE0903351F6D7CF8CE02A
:10BBC000973331F6D3CF8DE0963311F6CFCF903245
:10BBD00009F49ECF8EE0933549F2BACF80ED890FFC
:10BBE0008A3008F095CF2FE02093AD048093AC0409
:10BBF0008FCF9A3019F09D3009F08ACF1092AD04A2
:10BC000087CF9A3019F09D3009F082CF80915E176E
:10BC10008823A1F3273001F138F4253079F7109209
:10BC200079021092C208EACF2A30D1F02F3031F7D2
:10BC30002091AC048091C0081092C008823089F332
:10BC4000843091F08130D1F6222319F02130B1F601
:10BC500082E08093C108D2CF81E080939B06CECF53
:10BC600081E080939A06CACF60EC71E2709331084C
:10BC700060933008C3CF8EBD0DB407FEFDCF08958D
:10BC80008FEF8EBD0DB407FEFDCF8EB50895909158
:10BC900064009B7F90936400982F906A96959CBD5A
:10BCA00080FD03C091E0863009F490E09DBD0895C9
:10BCB000CF93DF93EB010E947C41CE01DF91CF91C6
:10BCC0000C943EE5AF92BF92CF92DF92EF92FF923B
:10BCD0000F931F93CF93DF93CDB7DEB7E6970FB6E1
:10BCE000F894DEBF0FBECDBF0091540510915505ED
:10BCF000F80101900020E9F731976F01C01AD10ACD
:10BD0000F801CF01801B910B8C159D053CF48191AE
:10BD10008F32B9F7DF0111971C92F3CF8BE1EBE87B
:10BD2000F7E1DE015C9601900D928A95E1F7F12C26
:10BD3000E12CEC14FD040CF05DC0F801EE0DFF1DCC
:10BD40008081811103C08FEFE81AF80A5801AE0C08
:10BD5000BF1CF5018081882309F44CC0FFEFEF1A66
:10BD6000FF0AF801EE0DFF1D7F01E01AF10A819133
:10BD70008111FACFCE014C960E94D1E98BE1FE01F0
:10BD80007C96DE01119601900D928A95E1F7B5013E
:10BD9000CE0101960E94DFE1CE0101960E94F939A1
:10BDA0008FE20E9443418091981381113BC08CE83F
:10BDB00093E00E943EE580916A1784FF1BC01982C0
:10BDC0001C8221E0A501BE01645E7F4FCE01019679
:10BDD0000E94A4EB811129C08AE00E9443410E9485
:10BDE000F757B50184E598E10E94585ECE010196AF
:10BDF0000E94F9398AE00E944341CE014C960E948C
:10BE0000F939E6960FB6F894DEBF0FBECDBFDF91CD
:10BE1000CF911F910F91FF90EF90DF90CF90BF9047
:10BE2000AF90089588E993E1C4CFCE014C960E946B
:10BE300040E98BE1FE013196DE015C9601900D92A6
:10BE40008A95E1F7CE0101960E94F93972CF2F92BF
:10BE50003F924F925F926F927F928F929F92AF929A
:10BE6000BF92CF92DF92EF92FF920F931F93CF93E7
:10BE7000DF9300D000D000D01F921F92CDB7DEB765
:10BE8000B82E80911112843008F0D1C10F945F5206
:10BE90006B017C0180911112811108C080912411E5
:10BEA00090912511891B8F7709F463C681E6A82E2E
:10BEB00013C08A3019F08D3009F0F6C010920C12C0
:10BEC0008091AA119091AB11FC01EA55FE4E1682A9
:10BED000892BF1F40F940C1280911112843008F028
:10BEE000ECC08091241190912511891B8F7709F462
:10BEF000E4C00E942B5D97FFDCCF0E94F35781EBDB
:10BF000097E00E947C418091241180932511E4CF19
:10BF10001092AB111092AA110CEA11E1F801819173
:10BF2000803209F446C08E3409F0A9C06CEA77E08B
:10BF3000C8010F94BD6C4C01892B41F06EE470E098
:10BF4000C80104960F948077009709F4C8014AE06D
:10BF500050E070E060E001960F942D6A2B013C01E7
:10BF60008091A6119091A711A091A811B091A9114B
:10BF70000196A11DB11D481659066A067B0629F0D7
:10BF800060E089E797E0892851F16AE270E0C80132
:10BF90000F94AF779C01009729F1982F901B912C5B
:10BFA000992349F09150F801E90FF11D80819826FD
:10BFB000F7CF8F01B3CF4AE050E070E060E0C901F5
:10BFC00001960F942D6A292D30E050E040E0621771
:10BFD00073078407950751F060E08AE597E00F94B6
:10BFE00075367ACF60E080E397E0F9CF4092A611F2
:10BFF0005092A7116092A8117092A91180917308B4
:10C000008130E1F067E470E0C8010F948077009719
:10C01000A9F04AE050E070E060E001960F942D6ACC
:10C02000643071058105910548F48FE896E00E941F
:10C030007C4160E085E896E00E942CCAC092C70867
:10C04000D092C808E092C908F092CA088091AC1159
:10C050008B3309F441CF80911112843008F03CCF2A
:10C06000809113128A9DC00111246CEA71E18C5EEB
:10C070009D4E0F948B7780E00F942F362DCF8091BB
:10C080006A1780FFBBCF67EB74E4C8010F94BD6CE7
:10C09000009731F0FC01838180538A3008F0AECFE5
:10C0A00060E086E097E09BCF2AEA31E14CEA51E17B
:10C0B0006CE072E10E9428240FCF80916A1782FF02
:10C0C000B6C01A82198271E6F72EE0E1EE2EF9E68B
:10C0D000DF2E80911112843008F0A9C00E946024E4
:10C0E0008111A5C041E050E0BE016B5F7F4F8FEC36
:10C0F00098E10E9493E70D8110E0019711F00FEF96
:10C100001FEF8091D7189091D818A091D918B091AD
:10C11000DA188093661790936717A0936817B09307
:10C1200069170E9460240F3F100749F4811107C06E
:10C130000E94F3578FEC97E00E947C41CACF409158
:10C140001312242F30E00A3061F00D3051F08823B3
:10C1500009F45FC089819A81009719F001969A834A
:10C1600089831092B00489819A81F29EF001F39E36
:10C17000F00D1124EF5EFD4EE80FF91F1382892B9D
:10C1800069F50F940C120E946024882309F4A1CF52
:10C190000E942CFB8FEC98E10E9440E9809161178E
:10C1A000882391F18150809361178D9DC0011124E6
:10C1B00062E08355994F0E944DEDE091611724E0B4
:10C1C000E29FF0011124E755F94F6081718182816E
:10C1D00093810E945E280E9448E17BCF1A821982D7
:10C1E00081E00F942F368091661790916717A09188
:10C1F0006817B091691780930D1290930E12A09357
:10C200000F12B0931012BFCF0E9449E9E092730859
:10C2100060CF4F9DA00111244C5E5D4E9E012F5FAB
:10C220003F4F60EB74E0802F0E94282452CF0F9480
:10C230005F526B017C01B11004C08091A806882375
:10C2400051F0C092BA08D092BB08E092BC08F092BC
:10C25000BD08BB24B39480912E0590912F05A09129
:10C260003005B09131050097A105B10551F140911C
:10C27000BA085091BB086091BC087091BD08840F4A
:10C28000951FA61FB71FA7019601281B390B4A0B44
:10C290005B0BDA01C901B7FD14C00E94F35760912E
:10C2A000C5087091C6088AE298E00E94585E8AE04C
:10C2B0000E94434140E070E060E090E080E00E9436
:10C2C0002A5C80911B0290911C02A0911D02B091EA
:10C2D0001E02892B8A2B8B2B79F09091E816809186
:10C2E000E916981709F4ACC1C092BA08D092BB08FD
:10C2F000E092BC08F092BD088091C1049091C20404
:10C300009099E0C101969093C2048093C1048091FA
:10C31000C1049091C2048E3E92406CF00E94F3578B
:10C3200087E098E00E947C4140E070E060E090E0AF
:10C3300080E00E942A5C0F945F524B015C01809167
:10C34000C208811108C02091E8169091E91681E099
:10C35000291301C080E020914A1630914B1691E0DC
:10C3600089272A3A31050CF480E091E04091B50428
:10C370005091B6046091B7047091B804452B462BD8
:10C38000472B09F490E0981789F0882309F4A0C19D
:10C39000D501C40180569444A24FBF4F8093B50489
:10C3A0009093B604A093B704B093B8044090DF090B
:10C3B0005090E0096090E1097090E2092091B10489
:10C3C0003091B2044091B3045091B404C301B2015E
:10C3D0000F94406D882319F18091B5049091B604B3
:10C3E000A091B704B091B8044092B1045092B20445
:10C3F0006092B3047092B404892B8A2B8B2B09F4BE
:10C4000049C0D501C40180569444A24FBF4F8093C8
:10C41000B5049093B604A093B704B093B804809188
:10C42000B5049091B604A091B704B091B8040097F8
:10C43000A105B10579F1881A990AAA0ABB0AB7FCC5
:10C4400029C01092B5041092B6041092B70410924D
:10C45000B80482EF97E00E947C4160E08EED97E0A7
:10C460000E942CCA80914C1690914D1618161906F0
:10C4700024F490E080E00E94AEFA8091E908909167
:10C48000EA081816190634F41092EA081092E9081E
:10C490000E94CEDC8091BD049091BE04A091BF04A7
:10C4A000B091C00446015701881A990AAA0ABB0A2A
:10C4B000D501C401B7FD9CC12091E8169091E91601
:10C4C0008091680240916902291306C19091150A72
:10C4D000899FC0011124880F892F881F990B91957E
:10C4E0008D838091160A489FC0011124880F892FDF
:10C4F000881F990B91958E830F945F5269837A837D
:10C500008B839C8340E0BE016F5F7F4FCE01059619
:10C510000E9485FB6D8170E089E00F94565141E0E7
:10C52000BE016F5F7F4FCE0105960E9485FB6E8135
:10C5300070E087E00F9456518091A706882309F494
:10C540004AC100913B0210913C02C8010297209120
:10C550004C1630914D16281739070CF43CC18090C9
:10C56000E9168F82188619861A861B868091E8162E
:10C570009F80891509F4CAC0892D90E03BE6A32E5F
:10C58000A89EF001A99EF00D1124E65DF54F4589A6
:10C5900056896789708D452B462B472B81F4418D39
:10C5A000528D638D748D452B462B472B41F4458D61
:10C5B000568D678D70A1452B462B472BE1F12BE65D
:10C5C000B22EB89E9001B99E300D1124A901465D8E
:10C5D000554F1A01FA0161817281838194810F9410
:10C5E000E0764B015C01F10161A172A183A194A1EC
:10C5F0000F94456D2B013C01F10165A176A187A146
:10C6000090A50F94456D9B01AC01C301B2010F943D
:10C610002C75A50194010F94A66D4B015C01288532
:10C6200039854A855B850F949276181624F488869E
:10C630009986AA86BB868F818F5F8F708F8396CFF6
:10C64000BB2019F01092C30457CE0F945F52009193
:10C65000BA081091BB082091BC083091BD088090A9
:10C660001B0290901C02A0901D02B0901E02080DAB
:10C67000191D2A1D3B1D601B710B820B930B97FD2F
:10C68000E1CF8091C304811137CE81E08093C30450
:10C690005F9A8091B8088E7F8093B8088A9A8091BB
:10C6A000B8088D7F8093B8088091080180958170CB
:10C6B000809306018091B8088B7F8093B8080E9410
:10C6C0006A261ACE181619060CF021CE01971BCE39
:10C6D00080E090E0DC0162CE2091E9165BE6259FC8
:10C6E00090011124265D354FF901EF59FF4F9081DC
:10C6F000899FC0011124880F892F881F990B91955C
:10C700008D832E593F4FF9018081EDCE2091350266
:10C710003091360240913702509138026885798510
:10C720008A859B850F94A66D4B015C01B801012E93
:10C73000000C880B990B0F94476D9B01AC01C50150
:10C74000B4010F94327469837A838B839C83409104
:10C75000390250913A02B801CE0101960E9467F465
:10C7600089809A80AB80BC804090B9045090BA0414
:10C770006090BB047090BC04A3019201C501B40198
:10C780000F94406D87FF16C028E431EE4AE75FE35F
:10C79000C301B2010F94A66D20E037ED43EA5CE3DC
:10C7A0000F943274A50194010F94A66D69837A8366
:10C7B0008B839C8369817A818B819C816093B9048E
:10C7C0007093BA048093BB049093BC040F949E753D
:10C7D000CB010E94AEFAF4E6CF0ED11CE11CF11C95
:10C7E000C092BD04D092BE04E092BF04F092C00497
:10C7F0000F940C1280917308882309F47AC19091E8
:10C800000901892F8095817010910802181709F489
:10C810005AC020916A17206220936A1780930802F9
:10C8200090FD10C064EF71E080E090E00E94793EDE
:10C830000E946BE980916A1783FDBEC1112309F440
:10C8400042C002C00E945AE9123008F46BC100E0F5
:10C850000E945D2C83E0809389020F945F526C5993
:10C860007F4F8F4F9F4F6093590570935A05809368
:10C870005B0590935C05002331F1123021F5809126
:10C880006A1783FF20C00F94ED5D882379F081E063
:10C890000F94095D42EB50E065E179E080E797E1B4
:10C8A0000E9493E780E797E10E9440E90E94E73900
:10C8B000811144C10E94D1390F94015E81E08093BF
:10C8C00060170F94495E0F945F526B017C011091C9
:10C8D0001F021123F1F08091C3088823D1F0409109
:10C8E000C4045091C5046091C6047091C704460108
:10C8F0005701841A950AA60AB70AB501A40177FD63
:10C900001AC0833009F430C10CF01FC181300CF023
:10C9100024C1212F30E0A8EEB3E00F94D873C60EE7
:10C92000D71EE81EF91EC092C404D092C504E0923E
:10C93000C604F092C7048091DC08813009F073C00E
:10C940000F945F526B017C018091CC049091CD04D7
:10C95000A091CE04B091CF04A7019601281B390BFA
:10C960004A0B5B0BDA01C901B7FD3AC0D701C6011A
:10C97000805F984DAF4FBF4F8093CC049093CD0410
:10C98000A093CE04B093CF0480901006909011062F
:10C99000A0901206B09013060F94BA1FAB01BC0111
:10C9A000409310065093110660931206709313067D
:10C9B0008091200890912108A0912208B09123082D
:10C9C00088199909AA09BB09840F951FA61FB71FCB
:10C9D0008093200890932108A0932208B093230805
:10C9E0008091C8049091C904A091CA04B091CB046D
:10C9F00046015701881A990AAA0ABB0AD501C4013F
:10CA0000B7FD11C020E8C20E2EEED21E26E3E21EB4
:10CA1000F11CC092C804D092C904E092CA04F092FA
:10CA2000CB040E942BFA0F947E230E9467CE809144
:10CA30002D05882379F10F945F526B017C01809161
:10CA4000290590912A05A0912B05B0912C0546014E
:10CA50005701881A990AAA0ABB0AD501C401B7FD71
:10CA600019C020912D0530E0A8EEB3E00F94D873E3
:10CA7000C60ED71EE81EF91EC0922905D0922A05BF
:10CA8000E0922B05F0922C0580E00E94DEEF8AE018
:10CA90000E94434180912805882359F10F945F52E9
:10CAA0006B017C018091240590912505A0912605BC
:10CAB000B0912705A7019601281B390B4A0B5B0B88
:10CAC000DA01C901B7FD15C02091280530E0A8EEB4
:10CAD000B3E00F94D873C60ED71EE81EF91EC0929D
:10CAE0002405D0922505E0922605F09227050E94A4
:10CAF00006E12B960FB6F894DEBF0FBECDBFDF91D7
:10CB0000CF911F910F91FF90EF90DF90CF90BF904A
:10CB1000AF909F908F907F906F905F904F903F90DD
:10CB20002F90089560E087E698E00E942CCA8091DB
:10CB3000660581118CCE0E94989A89CE84E898E08F
:10CB40009093310880933008BECE843009F0E1CE56
:10CB50000E94F7578BE898E004C00E94F7578AEBD1
:10CB600098E00E947C41D5CE0E94F75783EA98E076
:10CB7000F8CF8091C7089091C808A091C908B091DA
:10CB8000CA08A7019601281B390B4A0B5B0BDA0177
:10CB9000C901885E9340A109B109B7FD87C989EC35
:10CBA00097E00E947C41C092C708D092C808E092EA
:10CBB000C908F092CA087AC9123028F460E085E703
:10CBC00098E00E942CCA01E043CE2F923F924F92F0
:10CBD0005F926F927F928F929F92AF92BF92CF920D
:10CBE000DF92EF92FF920F931F93CF93DF93CDB716
:10CBF000DEB7EE970FB6F894DEBF0FBECDBF8091C3
:10CC0000E208888B87E50E948E37882309F41FC1CC
:10CC100020E030E0A9016091890670918A06809138
:10CC20008B0690918C060F94406D811108C00E9474
:10CC3000F35781E69EE00E947C4110E01BC18AE52B
:10CC40000E94DC37882339F10E9464372091CF0994
:10CC50003091D0094091D1095091D2090F9431748B
:10CC60006B017C0120E030E040E251ECC701B601ED
:10CC70000F94927687FD0AC020E030E040E251E454
:10CC8000C701B6010F94406D181674F40E94F35753
:10CC900084E59EE0D0CFC090DB09D090DC09E09025
:10CCA000DD09F090DE09DECF40E050E060EC7FE788
:10CCB00088E50E9462382091C7093091C8094091E7
:10CCC000C9095091CA090F9431742B013C0140E00D
:10CCD00050E060EC7FE789E50E9462382091CB0943
:10CCE0003091CC094091CD095091CE090F94317407
:10CCF0004B015C016FEF89E40E945638182F6FEFEB
:10CD00008AE40E945638082FA3019201C301B201A0
:10CD10000F94247781116EC0A5019401C501B4015F
:10CD20000F942477811166C08BA19CA1ADA1BEA1F7
:10CD30008BAB9CABADABBEAB209181063091820634
:10CD40004091830650918406C301B2010F9431745F
:10CD50002B013C0120E030E040E05FE36BA97CA9BF
:10CD60008DA99EA90F94A66D9B01AC01C301B201D0
:10CD70000F9432742BA93CA94DA95EA90F942C7570
:10CD80000F949E75162F4FA058A469A47AA42091E1
:10CD90008506309186064091870650918806C50128
:10CDA000B4010F9431744B015C0120E030E040E0AD
:10CDB0005FE3C301B2010F94A66D9B01AC01C501F5
:10CDC000B4010F943274A30192010F942C750F9447
:10CDD0009E75062F812F012E000C990B97FD2FC0F9
:10CDE00005977CF5802F002E000C990B97FD2BC02A
:10CDF00005975CF5153008F020CF053008F01DCF01
:10CE000080E00E948D3C95E01902F0011124E00FB2
:10CE1000F11D07FDFA95EE0FFF1FEE0FFF1FE35EFA
:10CE2000F94FC082D182E282F38288890E948D3CD0
:10CE30008889882309F401CF0F948B19FECE10E066
:10CE4000D1CF14E0CFCF00E0D5CF04E0D3CF8AE438
:10CE50000E948E37182F811127C070E060E086E5B0
:10CE60000E94AD399A838983059708F18FE29EE08D
:10CE70000E947C41812FEE960FB6F894DEBF0FBE64
:10CE8000CDBFDF91CF911F910F91FF90EF90DF9079
:10CE9000CF90BF90AF909F908F907F906F905F905A
:10CEA0004F903F902F9008950E94DB3CC6CE60E0EB
:10CEB00084E40E94BC398F8740E050E0BA018AE5E3
:10CEC0000E9462386BA77CA78DA79EA740E050E820
:10CED0006BE376E483E50E94623820E030E040E7CF
:10CEE00052E40F942C7560937D0270937E028093C0
:10CEF0007F0290938002E090E316F090E416D70151
:10CF00008D909D90AD90BC9020E030E0A901C501CE
:10CF1000B4010F9432746BAF7CAF8DAF9EAF20E045
:10CF200030E040E450E40F94406D87FF06C01BAE34
:10CF30001CAEB0E4BDAFE0E4EEAF20E030E040E78F
:10CF400053E4C501B4010F9432746BAB672E8FAB01
:10CF500098AF20E030E043E653E40F949276181641
:10CF600034F41BAA612CF3E6FFAB23E428AFD7010E
:10CF700014968D909D90AD90BC90179720E030E076
:10CF8000A901C501B4010F943274D62EE72EF82EF4
:10CF9000092F20E030E040E951E40F94406D87FF15
:10CFA00005C0D12CE12CF0E9FF2E01E420E030E0B7
:10CFB00040E753E4C501B4010F943274B62EC72E76
:10CFC00089AF9AAF20E030E044E553E40F949276C5
:10CFD000181634F4B12CC12CB4E5B9AFE3E4EAAFD0
:10CFE00088E40E948E37882309F415C20E946437B2
:10CFF0000F949E751B0177FF02C06F5F7F4F759581
:10D0000067957195619571096D587F4F072E000CDA
:10D01000880B990B0F94476D762E872E982EA92E8C
:10D020002D2D3E2D4F2D502F0F94927618161CF457
:10D03000D72C74010A2D2BAD3CAD4DAD5EAD672DE7
:10D04000782D892D9A2D0F949276181624F07BACAA
:10D050008CAC9DACAEAC872D982DA92DBA2D8B8BA9
:10D060009C8BAD8BBE8B8D2D9E2DAF2DB02F8F8BBE
:10D07000988FA98FBA8FB101330C880B990B0F943D
:10D08000476D1B012C01AC019B016D2D7E2D8F2D59
:10D09000902F0F943274D62EE72EF82E092F2B2DB9
:10D0A0003C2D49AD5AAD0F94406D87FF04C0BD2C97
:10D0B000CE2CF9AE0AAFA2019101672D782D892DF2
:10D0C0009A2D0F943274D62EE72EF82E092F2BA905
:10D0D000362D4FA958AD0F94406D87FF04C0DBAAD1
:10D0E0006E2CFFAA08AF8BA9962DAFA9B8AD8B8F78
:10D0F0009C8FAD8FBE8F8B2D9C2DA9ADBAAD8F8F20
:10D1000098A3A9A3BAA3BE01695E7F4FCE0143963F
:10D110000E944132882309F4AFC1BE01615E7F4F96
:10D12000CE014B960E944132E82E882309F4A4C117
:10D130002F89388D498D5A8D6F8D78A189A19AA13B
:10D140000F94317420E030E040E85EE30F94A66D68
:10D150004B015C012B893C894D895E896B8D7C8DEF
:10D160008D8D9E8D0F94317420E030E040E85EE3B9
:10D170000F94A66D6BA37CA38DA39EA38FA298A6EC
:10D18000A9A6BAA689819A811816190674F48DEF9A
:10D190009DE00E947C418F85882321F083EF9DE0F4
:10D1A0000E947C418AE00E9443410E942CFB0F9424
:10D1B000CE0F80E00E948D3C80E090E0A0E2B1E4E0
:10D1C0008FA798ABA9ABBAAB60E0CE018F960F9456
:10D1D00005112091890630918A0640918B06509165
:10D1E0008C066BA17CA18DA19EA10F94406D811135
:10D1F00030C020918D0630918E0640918F0650915F
:10D2000090066FA178A589A59AA50F94406D81110C
:10D2100020C0209181063091820640918306509172
:10D2200084066B897C898D899E890F94406D81115C
:10D2300010C0209185063091860640918706509156
:10D2400088066F89788D898D9A8D0F94406D88231B
:10D25000A9F00E94DB3C88E0FE01B396A9E8B6E0A5
:10D2600001900D928A95E1F788E0FE017396A1E89E
:10D27000B6E001900D928A95E1F7188A60E085E4A6
:10D280000E94BC3988248394811102C062E0862EFA
:10D290001B861C861D861E861A8A9E2C43ECC42E75
:10D2A0004DE0D42E51EDA52E5DE0B52E1A89153036
:10D2B0000CF0ECC06B857C858D859E859B01AC0157
:10D2C0000F9424778111E2C03324339435E0232E68
:10D2D000911005C033243A9422242A9484E091E0EA
:10D2E0009926F12EFF0CFF0CF10EF394898B19890E
:10D2F0006A89121509F4C6C0062E000C770B880B3C
:10D30000990B0F94476D2FA138A549A55AA50F94E5
:10D31000A66D2F89388D498D5A8D0F9432742B014B
:10D320003C01612F110F770B880B990B0F94476D00
:10D330002BA13CA14DA15EA10F94A66D2B893C8928
:10D340004D895E890F9432746B837C838D839E83B9
:10D350004F82588669867A8689819A81892B79F0ED
:10D360006F2D8FED9DE00E94474469E170E08DEDE7
:10D370009DE00E94D9498AED9DE00E947C411F9268
:10D38000F9E1FF931F92FF92DF92CF92BF92AF928B
:10D390001F920E9411CA2981482DBE01695F7F4FEB
:10D3A000CE0103960F94F3482B013C014B865C861B
:10D3B0006D867E860FB6F894DEBF0FBECDBFAC0182
:10D3C0009B010F94247781115AC009898A8925E02D
:10D3D000020380011124080F111D87FD1A95000F0B
:10D3E000111F000F111F035E194FA30192016BA5BE
:10D3F0007CA58DA59EA50F943274D8016D937D9365
:10D400008D939C931397188A81E00E94275FF39471
:10D410008989830D6BCF4D2D5E2D6F2D702F86E486
:10D420000E9462381B012C014BAD5CAD6DAD7EAD31
:10D430008CE40E9462386B8B7C8B8D8B9E8B2F8A49
:10D44000388E498E5A8E4B2D5C2D69AD7AAD82E4B3
:10D450000E9462386B017C014BA9562D6FA978ADF3
:10D4600082E50E9462386B8F7C8F8D8F9E8FCF8E6E
:10D47000D8A2E9A2FAA247CE83E19EE0F9CC88893E
:10D480000E948D3C8A898F5F8A8B10CF0F947747DB
:10D490000E943832882359F088890E948D3C80E0B0
:10D4A00090E0A0ECBFE78B879C87AD87BE876B853C
:10D4B0007C858D859E859B01AC010F94247781111D
:10D4C00059C08F85811126C082E0F82E02E094E0D9
:10D4D000C92E12E0DC2CD11A21E041E0612F802F0F
:10D4E0000E94DA2421E04FEF612F8F2D0E94DA2471
:10D4F0002FEF41E06D2D802F0E94DA242FEF4FEFA8
:10D500006D2D8F2D0E94DA24115020F70150F394D5
:10D510000F3FF9F60E94C4430E94FF3D8F858111A1
:10D5200024C08BED99E00E9472334B015C0183EDC6
:10D5300099E00E94A03A9B01AC01C501B4010F948F
:10D54000A66D9B01AC016091DB097091DC098091B3
:10D55000DD099091DE090F9431746093DB097093BB
:10D56000DC098093DD099093DE098F858111E888BD
:10D57000E092E2080F94B50F8091E20881110F94B8
:10D580000A120E940A2A0F948B196B857C858D855F
:10D590009E8511E09B01AC010F94247781116ACC28
:10D5A0004CCBCF93DF93C82FD62F8091DB1083FD18
:10D5B00014C08091270A811110C080918E02909131
:10D5C0008F02AC014150510920914C1630914D16FB
:10D5D0002417350714F40E94AEFA40E06D2F8BE05B
:10D5E0000E94819BCC2339F040E061E080E0DF9134
:10D5F000CF910C94D6F18091270A91E089278093EE
:10D60000790280917902882389F080914A1690915D
:10D610004B1620914C1630914D16821B930B97FFA1
:10D6200003C0919581959109029744F41092790273
:10D630008091DB1083FF06C0C1E01AC080E00E9429
:10D64000275FDFCFC091270AC11112C080918E02DF
:10D6500090918F02019720914C1630914D1628170A
:10D66000390754F70E94F7578CE69AE00E947C41F4
:10D670008C2FDF91CF910895AF92BF92CF92DF921E
:10D68000EF92FF920F931F93CF93DF93CDB7DEB747
:10D6900064970FB6F894DEBF0FBECDBF0E949658B8
:10D6A000D82E87FDB5C08AE50E94DC37882309F4AF
:10D6B000C0C040E050E0BA018AE50E9462387B01B8
:10D6C0008C014D2D63E085E00E94819B2091DB0958
:10D6D0003091DC094091DD095091DE0960E070E095
:10D6E0008AE793E40F9431745B016C019701A80100
:10D6F0000F949276181614F07501860120E030E040
:10D70000A901B701C8010F949276181624F4E12CF0
:10D71000F12C00E010E0B701C8010F949E75072EB0
:10D72000000C880B990B0F94476D6D837E838F835C
:10D73000988720E030E0A9010F94406D882321F004
:10D74000CE0105960E94AC2880E090E0A0EAB1E40A
:10D7500089879A87AB87BC871D861E861F86188A95
:10D760008CE40E948E37882309F468C00E946437D5
:10D770006B017C0120E030E0A901C701B6010F94E4
:10D78000927687FF04C0F7FAF094F7F8F094C98A0C
:10D79000DA8AEB8AFC8A20914C1630914D1624309F
:10D7A000310574F080914A1690914B16821B930BB1
:10D7B00097FF03C091958195910901E004970CF4BE
:10D7C00000E063E080E00E94D16A811140C083E004
:10D7D00080933002109265050E94989A6D817E8137
:10D7E0008F8198858B019C01305809831A832B8384
:10D7F0003C8320E030E0A9010F94406D882321F0A4
:10D80000CE0101960E94AC28109265050E94989A5C
:10D8100064960FB6F894DEBF0FBECDBFDF91CF91F7
:10D820001F910F91FF90EF90DF90CF90BF90AF903E
:10D830000895E12CF12C00E211E443CFC0901806CA
:10D84000D0901906E0901A06F0901B0693CF83E063
:10D85000E82E22E0AE01475F5F4FBE016F5E7F4F53
:10D86000CE010D960F94DF47B9CF6F927F928F92C2
:10D870009F92AF92BF92CF92DF92EF92FF920F935F
:10D880001F93CF93DF9300D000D01F921F92CDB78C
:10D89000DEB75C014B013A01F22E68010091A0064F
:10D8A00010929C0610929D0610929E0610929F0662
:10D8B0001092A0060F946B5280914C1690914D16C9
:10D8C0008C159D051CF4C6010E94AEFA60E080E054
:10D8D0000E94D16A811122C1109265050E94989A16
:10D8E0001C141D0444F4C6010E94AEFA40E060E03E
:10D8F00080E00E94D6F140E060E088E00E94819BD9
:10D9000060E081E00E94D16A80E090E0A0E7B2E4AC
:10D9100089839A83AB83BC8380E090E0A0E8B0EC7D
:10D920008D839E83AF83B887BE016F5F7F4FCE012B
:10D9300005960F94551187E00F94E70E811158C09A
:10D940008091DB099091DC09A091DD09B091DE099D
:10D9500040910505509106056091070570910805F5
:10D96000C0900105D0900205E0900305F0900405F9
:10D97000C092A808D092A908E092AA08F092AB0839
:10D980004093AC085093AD086093AE087093AF0815
:10D990008093B0089093B108A093B208B093B308F5
:10D9A00080E090E0A8E4B2E489839A83AB83BC83EF
:10D9B000CE0101960F94FB188091090590910A05FC
:10D9C000A0910B05B0910C058093B0089093B1081D
:10D9D000A093B208B093B30880E090E0A0EAB0E46E
:10D9E00089839A83AB83BC83CE0101960F94FB1885
:10D9F000C12CD12C80E7E82E82E4F82EC982DA828D
:10DA0000EB82FC8280E090E0A0E8B0E48D839E830E
:10DA1000AF83B887BE016F5F7F4FCE0105960F942D
:10DA2000551120E030E0A90160910D0570910E05BF
:10DA300080910F05909110050F94406D87FF0BC0EA
:10DA4000C982DA82EB82FC82BE016F5F7F4F8DE07C
:10DA500095E00F94551180910D0590910E05A091C0
:10DA60000F05B09110058093DF099093E009A09312
:10DA7000E109B093E2098093B4089093B508A093AC
:10DA8000B608B093B70884EB98E00F94CF0C809160
:10DA90001C0681110F94335D109265050E94989ABF
:10DAA00061E085E19BE00E943F438091A8068150A0
:10DAB0008093A80641E851E26DE17BE085E00F9498
:10DAC000EA488091A806882339F00E9448E18091B5
:10DAD000A80681508093A80680E00F949947809112
:10DAE000DC08823011F40F947C200F9477470E9459
:10DAF000989A28960FB6F894DEBF0FBECDBFDF917F
:10DB0000CF911F910F91FF90EF90DF90CF90BF903A
:10DB1000AF909F908F907F906F900895E12C2F2D64
:10DB2000A301B401C5010F94DF47DACE4F925F9293
:10DB30006F927F92AF92BF92CF92DF92EF92FF925D
:10DB40001F93CF93DF9300D000D01F921F92CDB7C9
:10DB5000DEB75C01E62EF42E642F80E00E94D16ACD
:10DB6000182F81111BC0EE2021F0109265050E9434
:10DB7000989A812F28960FB6F894DEBF0FBECDBFBE
:10DB8000DF91CF911F91FF90EF90DF90CF90BF90EA
:10DB9000AF907F906F905F904F900895EE2029F0A6
:10DBA00040E06F2D83E00E94819B80E090E0A0E741
:10DBB000B2E48D839E83AF83B88780E090E0A0E8D5
:10DBC000B0EC89839A83AB83BC83BE016B5F7F4FCC
:10DBD000CE0101960F94551168E873E180E090E062
:10DBE0000E94793EC12CD12C88ECE82E81E4F82EDD
:10DBF000CD82DE82EF82F88680E090E0A0E8B0E49B
:10DC000089839A83AB83BC83BE016B5F7F4FCE0158
:10DC100001960F9455114090141150901511609079
:10DC2000161170901711C0921411D0921511E09234
:10DC30001611F092171180E090E0A0E2B2E48D831B
:10DC40009E83AF83B887F50180819181A281B381E2
:10DC500089839A83AB83BC83BE016B5F7F4FCE0108
:10DC600001960F9455114092141150921511609223
:10DC7000161170921711129A64E670E080E090E03D
:10DC80000E94793E76CF8F929F92AF92BF92CF92B1
:10DC9000DF92EF92FF921F93CF93DF9300D000D0DB
:10DCA0001F921F92CDB7DEB70E949658182F87FD9E
:10DCB000ADC08AE50E94DC37812C912C90E2A92E20
:10DCC00091E4B92E882341F040E050E0BA018AE5A2
:10DCD0000E9462384B015C01412F64E083E00E94A6
:10DCE000819B20E030E0A901C501B4010F94927638
:10DCF00018167CF580E090E0A0EAB0E48D839E8366
:10DD0000AF83B8872091DB093091DC094091DD09B0
:10DD10005091DE09C501B4010F9432746B017C018E
:10DD200020E030E04AE753E40F94406D87FD06C0E1
:10DD3000C12CD12C8AE7E82E83E4F82EC982DA823E
:10DD4000EB82FC82BE016B5F7F4FCE0101960F9488
:10DD5000E61085E50E948E37882309F469C00E9489
:10DD600064376B017C0120E030E0A901C701B601F6
:10DD70000F94927687FF04C0F7FAF094F7F8F094C6
:10DD8000F7FAF094F7F8F094C982DA82EB82FC8219
:10DD900044E061E0CE0101960E94966D20E030E003
:10DDA000A901C501B4010F94927618165CF580E0C4
:10DDB00090E0A0EAB0E48D839E83AF83B887A5018D
:10DDC00094016091DB097091DC098091DD099091EB
:10DDD000DE090F9431746B017C0120E030E0A90171
:10DDE0000F94927618161CF0C12CD12C7601C982A2
:10DDF000DA82EB82FC82BE016B5F7F4FCE0101961F
:10DE00000F94E610109265050E94989A28960FB616
:10DE1000F894DEBF0FBECDBFDF91CF911F91FF9071
:10DE2000EF90DF90CF90BF90AF909F908F9008952C
:10DE300088E01802F0011124EC5EF94FC080D18017
:10DE4000E280F38090CFBF92CF92DF92EF92FF9269
:10DE50000F931F93CF93DF9300D01F92CDB7DEB700
:10DE60007C016B018A01B22E61E088E09BE00E9498
:10DE70003F4341E851E26FE07BE085E00F94EA48E0
:10DE80009091A80681E0890F8093A80680916A1777
:10DE900082FF06C08B7F80936A179E5F9093A806CF
:10DEA0000F94B42080E1E3EDF9E0A1E0B5E001904A
:10DEB0000D928A95E1F70E942CFB81E00F9499471F
:10DEC00020E030E0A901F7016081718182819381B6
:10DED0000F94406D8823F1F08091270A81110CC0C6
:10DEE00080918E0290918F02019720914A16309175
:10DEF0004B162817390774F080E090E0A0E7B2E4F1
:10DF000089839A83AB83BC83BE016F5F7F4FC70158
:10DF10000F94551187E00F94E70E811103C0B601ED
:10DF20000F94D22220E030E0A901F80160817181D4
:10DF3000828193810F94406D882329F042E06B2DFC
:10DF4000C8010E94966D129A64E670E080E090E04D
:10DF50000E94793E81E00F900F900F900F90DF911B
:10DF6000CF911F910F91FF90EF90DF90CF90BF90D6
:10DF70000895CF92DF92EF92FF92CF93DF936B01E0
:10DF80007C01D42FC091C30883E08093C30881E053
:10DF90008093C208C114D104E104F10431F00F945C
:10DFA0005F52C60ED71EE81EF91E8091C208882354
:10DFB00089F0C114D104E104F10421F48D2F0E94F1
:10DFC000275FF3CF0F945F526C197D098E099F096B
:10DFD00097FDF4CF1092C208C093C308DF91CF9190
:10DFE000FF90EF90DF90CF9008951F93CF93DF9332
:10DFF000D82FC62F0E946A5B61E08C2F0E94FF39E8
:10E000000F945F52685370458F4F9F4F60939C06EB
:10E0100070939D0680939E0690939F061092A00693
:10E020001091C30883E08093C30830E020E041E210
:10E0300056E46AEF7AE082E00E94864381E08093B2
:10E04000C2088091C208882309F463C060E08C2F65
:10E050000E94FF398091A006882309F456C040E051
:10E0600060E08AE00E94819B0E94F75780EE9AE070
:10E070000E947C4130E020E04AEC5AE061ED7AE019
:10E0800082E00E94864341E060E070E0CB010E94A4
:10E09000B96F30E020E050E040E06DEB7AE085E0E1
:10E0A0000E94864310929C0610929D0610929E0636
:10E0B00010929F061092A0060F946B5260E080E0D1
:10E0C0000E94D16A8D2F0E946A5B0F945F52685341
:10E0D00070458F4F9F4F60939C0670939D06809371
:10E0E0009E0690939F061092A00630E020E041E249
:10E0F00056E461EB7AE082E00E94864381E08093FF
:10E10000C20861E08C2F0E94FF3981E00E94275FE6
:10E1100098CF1093C308DF91CF911F910895CF92AC
:10E12000DF92EF92FF920F931F93CF93DF93CDB7C0
:10E13000DEB7A0970FB6F894DEBF0FBECDBF0E942A
:10E14000965887FDD1C0482F61E081E00E94819BF5
:10E1500085E40E948E37882309F4D5C00E94643775
:10E160006B017C0120E030E0A9010F94927687FFDB
:10E1700004C0F7FAF094F7F8F094F7FAF094F7F88F
:10E18000F094C98ADA8AEB8AFC8A8CE0E0EAF2E051
:10E19000DE01119601900D928A95E1F78AE50E94C1
:10E1A000DC37882351F040E050E0BA018AE50E9454
:10E1B000623869877A878B879C8788E50E94DC377D
:10E1C000882351F040E050E0BA0188E50E946238AF
:10E1D00069837A838B839C8389E50E94DC3788235B
:10E1E00051F040E050E0BA0189E50E9462386D8349
:10E1F0007E838F83988785E50E948E37882309F474
:10E2000089C00E9464376B017C0120E030E0A901E5
:10E21000C701B6010F94927687FF04C0F7FAF09415
:10E22000F7F8F094F7FAF094F7F8F094CD8ADE8AD4
:10E23000EF8AF88E198E1A8E1B8E1C8E8CE40E942B
:10E240008E37882309F46FC00E9464376B017C010C
:10E2500020E030E0A901C701B6010F94927687FF54
:10E2600004C0F7FAF094F7F8F094CD8EDE8EEF8EBE
:10E27000F8A262E070E082E40E94AD39F82E80914D
:10E28000A806811131C021E0AE014B5E5F4FBE0197
:10E290006F5F7F4FCE0141960E94236F882321F14B
:10E2A0006F2D81E00E94F56F82E50E94DC378823A4
:10E2B00009F442C00E94603740E050E060EA71E437
:10E2C0004D875E876F87788B2091A806222361F0A7
:10E2D0008C012F2DAE01435F5F4FBE01635E7F4F08
:10E2E000CE0149960E94356CA0960FB6F894DEBF19
:10E2F0000FBECDBFDF91CF911F910F91FF90EF9097
:10E30000DF90CF900895C12CD12C80E8E82E80E4D6
:10E31000F82E33CFC0901406D0901506E090160664
:10E32000F090170672CFC0901806D0901906E090B2
:10E330001A06F0901B068CCF90E080E0BDCFCF9204
:10E34000DF92EF92FF920F931F93CF93DF93CDB79E
:10E35000DEB76C970FB6F894DEBF0FBECDBF8CE46E
:10E360000E948E37882309F4C3C00E9464376B0172
:10E370007C0120E030E0A9010F94927687FF04C071
:10E38000F7FAF094F7F8F094F7FAF094F7F8F094BD
:10E39000C98EDA8EEB8EFC8E8CE0E0EAF2E0DE01D4
:10E3A000119601900D928A95E1F788E50E94DC377D
:10E3B0008823A1F040E050E0BA0188E50E9462386D
:10E3C0002091C7093091C8094091C9095091CA09E3
:10E3D0000F94317469837A838B839C8389E50E94CF
:10E3E000DC378823A1F040E050E0BA0189E50E94C3
:10E3F00062382091C7093091C8094091C9095091EC
:10E40000CA090F9431746D837E838F8398878AE560
:10E410000E94DC37882351F040E050E0BA018AE5E1
:10E420000E94623869877A878B879C87F0906A1789
:10E43000F2FAFF24F0F840E061E080E00E94819B66
:10E4400060E080E50E94BC39E82E1D861E861F868E
:10E45000188A8091A80681113CC02E2DAE01435F21
:10E460005F4FBE016F5F7F4FCE0149960E94236FC1
:10E47000882379F180911C0681110F94335DFF2070
:10E4800011F0EE2031F160E080E00E94F56F898D9F
:10E490009A8DAB8DBC8DB0588D8B9E8BAF8BB88F0A
:10E4A000198A1A8A1B8A1C8A1D861E861F86188A4C
:10E4B0008091A806882369F010E000E020E0AE011A
:10E4C0004B5E5F4FBE016F5E7F4FCE010D960E9487
:10E4D000356C6C960FB6F894DEBF0FBECDBFDF91E2
:10E4E000CF911F910F91FF90EF90DF90CF90089503
:10E4F000C12CD12C80E8E82E80E4F82E45CF2F9255
:10E500003F924F925F926F927F928F929F92AF92C3
:10E51000BF92CF92DF92EF92FF920F931F93CF9310
:10E52000DF93CDB7DEB7E5970FB6F894DEBF0FBE29
:10E53000CDBF8DAB2091C3082CAB81E08093C30885
:10E5400080914F058D3409F4C5C4843511F40C94C1
:10E55000AC86873409F091C180914D0590914E05AC
:10E560008B31910509F4D9C108F079C18430910546
:10E5700008F030C1209173088230910508F48EC1F3
:10E58000213009F091C111E0029709F010E00E94DA
:10E59000793819821A821B821C821D821E821F8278
:10E5A000188682E50E94DC37882309F48CC10E941A
:10E5B00064376B017C0120E030E0A9010F94406DCD
:10E5C000882309F4EAC04090D3095090D4096090A0
:10E5D000D5097090D6098091D7099091D809A0915A
:10E5E000D909B091DA098CA79DA7AEA7BFA78090E3
:10E5F000A8089090A908A090AA08B090AB088091B4
:10E60000AC089091AD08A091AE08B091AF0888AB6E
:10E6100099ABAAABBBABA5019401C301B2010F94A6
:10E62000406D81110DC028A939A94AA95BA96CA523
:10E630007DA58EA59FA50F94406D882309F4ADC0DC
:10E64000A3019201C501B4010F94317420E030E0C0
:10E6500040E05FE30F94A66D68A779A78AA79BA700
:10E660002CA53DA54EA55FA568A979A98AA99BA956
:10E670000F94317420E030E040E05FE30F94A66D2A
:10E680002B013C0120E030E0A901C701B6010F9445
:10E69000406D881F8827881F181709F40BC180E078
:10E6A00090E0A0E8BFEB8CA79DA7AEA7BFA728A5C9
:10E6B00039A54AA55BA5CA01B9010F94A66D4B0106
:10E6C0005C01A3019201C301B2010F94A66D9B01ED
:10E6D000AC01C501B4010F9432740F94E0764B0184
:10E6E0005C01AC019B01C701B6010F94317468ABAA
:10E6F00079AB8AAB9BABA5019401C701B6010F941E
:10E7000032749B01AC0168A979A98AA99BA90F94CD
:10E71000A66D6B017C0120E030E0A9010F94927698
:10E7200087FDCDC0C701B6010F94E0766B017C0177
:10E73000C301B2019058A50194010F942C752CA52A
:10E740003DA54EA55FA50F94A66DA70196010F9458
:10E75000A66D28A539A54AA55BA50F9432746983D7
:10E760007A838B839C83A501940168A579A58AA5EA
:10E770009BA50F942C752CA53DA54EA55FA50F94C8
:10E78000A66DA70196010F94A66DA30192010F94A7
:10E7900032746D837E838F83988720E030E0A901F7
:10E7A00069817A818B819C810F94406D81119FC01A
:10E7B00020E030E0A9016D817E818F8198850F94E2
:10E7C000406D811194C00E94F35785E091E10E9451
:10E7D0007C416AC08531910509F466C08A31910592
:10E7E00009F498C0049709F048C080E50E94DC371E
:10E7F000C12CD12C7601882321F00E94242A6B01A0
:10E800007C0183E50E94DC37882361F00E94643735
:10E8100020E030E04AE754E40F94A66D0F94A5750C
:10E820006B017C010E942CFB8091DB13811105C0E0
:10E8300060E08BE191E10E942CCA0F945F52C60EFA
:10E84000D71EE81EF91E0F945F526C197D098E09C0
:10E850009F0997FF29C080E00E94275FF4CF8A328A
:10E86000910509F4ACC160F48D31910509F4D4C06F
:10E8700008F46CC04E9709F428C10F94D14714C016
:10E880008B35910509F47EC28C35910509F47EC261
:10E890008A35910591F71092DD0806C0213021F4E8
:10E8A0000E9479380F944816FDA9F111ABC40F945A
:10E8B000C052A8C480E090E0A0E8BFE3F4CEC12C31
:10E8C000D12C760135CF89E40E94DC37882331F0E2
:10E8D0000E94643769837A838B839C838AE40E94D5
:10E8E000DC37882309F459CF0E94643752CF412F77
:10E8F000BE016F5F7F4F88EA98E00F9459530F94E1
:10E900005F526093BA087093BB088093BC089093E1
:10E91000BD08CACF0E94FB4EC7CF87E00F947F2E61
:10E920008111C2CF8CE0ECEAF2E0DE011196019099
:10E930000D928A95E1F770E060E080E50E94E9378A
:10E94000BE016F5F7F4F0F94D222AECF87E00F944E
:10E95000E70E811106C060E08FE40E94BC3981118E
:10E96000A3CF0E942CFB109240026091E2088CE43D
:10E970000E94BC39E82E80E00E948D3C0F945F52CB
:10E980006093BA087093BB088093BC089093BD084D
:10E990000F94CE0F81E080932D080F94B31A8AE56F
:10E9A0000E948E37F82E882369F081E00F94E70EDD
:10E9B000182F82E00F94E70E11110C945E8811E07D
:10E9C000811101C010E088E50E948E37082F811167
:10E9D0000C94C18611110C94D1860C94C486012F1D
:10E9E000182F0C94D18660E070E080E890E40C94DD
:10E9F000DA86A3019201C501B4010C94278760E077
:10EA000086E391E10E942CCA0E94F75784E291E1CB
:10EA10000E947C410C94FF8714E00F945F52609336
:10EA2000BA087093BB088093BC089093BD0880918E
:10EA3000E208811127C08EE40E948E37882321F0DE
:10EA400087E491E10E94908887E00F947F2E8111E6
:10EA50001FC00E94E5658823D9F0115001F130E014
:10EA600020E041E851E262E771E185E00E948643DF
:10EA700061E085E691E10E943F438DE491E10E94CF
:10EA80009088CBCF60E08FE40E94BC39882399F254
:10EA90000E94574380E192E10E94908805CF61E097
:10EAA00083E092E10E943F438EE891E10E949088CA
:10EAB00061E08CE691E20E943F4340E070E060E05C
:10EAC0008FE791E10E942A5CEFCE0091E31610914E
:10EAD000E416D8012D913D914D915C916091D3093F
:10EAE0007091D4098091D5099091D6090F94327410
:10EAF000AB01BC0188E50E94623869837A838B830D
:10EB00009C83F80124813581468157816091D70922
:10EB10007091D8098091D9099091DA090F943274D3
:10EB2000AB01BC0189E50E9462386D837E838F83CF
:10EB30009887BE016B5F7F4FCE0101960E944132E4
:10EB4000882309F4B1CE80E00E948D3C0F94CE0F53
:10EB500061E085E40E94BC39182F21E0482FBE01F6
:10EB60006B5F7F4FCE0101960F94F3486B017C01E0
:10EB7000AC019B010F942477811119C049815A81FE
:10EB80006B817C8182E392E10E944F444D815E81E2
:10EB90006F8178858DE292E10E944F44B701A60112
:10EBA00088E292E10E944F448AE00E9443410F9420
:10EBB000B50F11110E940A2A0F948B1975CE8091FE
:10EBC0007308813009F070CE89E40E94DC37082F89
:10EBD000F12C882319F00E946037F82E8AE40E94F5
:10EBE000DC37E82E882379F00E946037182F002345
:10EBF00009F4C0C0F4E0FF1508F0B9C08AE392E15F
:10EC00000E947C4151CE10E00111F4CF80E1E3ED90
:10EC1000F9E0A8EAB8E001900D928A95E1F70023A7
:10EC200019F16F2DFF0C770B880B990B0F94476D23
:10EC30002091890630918A0640918B0650918C066E
:10EC40000F94A66D20918106309182064091830633
:10EC5000509184060F9432746093A8087093A908A9
:10EC60008093AA089093AB08EE2019F1612F110F41
:10EC7000770B880B990B0F94476D20918D0630917F
:10EC80008E0640918F06509190060F94A66D2091AC
:10EC900085063091860640918706509188060F942C
:10ECA00032746093AC087093AD088093AE08909373
:10ECB000AF0860E080E50E94BC398823C1F10023E1
:10ECC000D1F0E091E316F091E41620813181428188
:10ECD00053816091A8087091A9088091AA08909129
:10ECE000AB080F9431746093A8087093A9088093BF
:10ECF000AA089093AB08EE20D1F0E091E316F091D2
:10ED0000E41624813581468157816091AC08709169
:10ED1000AD088091AE089091AF080F943174609364
:10ED2000AC087093AD088093AE089093AF0840E0B4
:10ED300050E0BA0186E40E9462386B017C0120E059
:10ED400030E0A9010F9492761816C4F420E030E068
:10ED500040E752E4C701B6010F942C7569837A83AA
:10ED60008B839C83CE0101960F94FB189DCDEE20E2
:10ED700009F44CCF153008F449CF40CF60E070E083
:10ED8000CB01ECCF8FE08093DD088ECD80914C05D8
:10ED9000882381F1893009F087CD68EBA62E62E0E7
:10EDA000B62E73EDC72E79E0D72EE12C00E010E0EF
:10EDB000D5018D915D010E94DC37F82E882361F02A
:10EDC000133011F4082FFE2C0E946437F601608383
:10EDD000718382839383EF2C1F5FF4E0CF0ED11CED
:10EDE000143031F7EE2009F457C00F940A120F9433
:10EDF0008B195ACD58EBC52E52E0D52EF12CE12CB3
:10EE000000E010E0D6018D916D010E94DC37382EB4
:10EE10008823D9F10E9464374B015C01133059F00B
:10EE2000F701E953F64F20813181428153810F94DC
:10EE300031744B015C01F701ED52F64F20813181B5
:10EE400042815381C501B4010F9431742B013C01FF
:10EE50002DEB37E346E855EB0F94927687FD0AC019
:10EE60002DEB37E346E855E3C301B2010F94406D43
:10EE700018165CF41330C1F48092DF099092E00917
:10EE8000A092E109B092E209032D1F5FB4E0EB0EFE
:10EE9000F11C143009F0B6CF002309F4A8CF8FED90
:10EEA00099E00F94CF0CA3CFF701E350F74F5F0128
:10EEB000A301920160817181828193810F943274E8
:10EEC000D5016D937D938D939C931397812F0F9410
:10EED000C70EDBCF80914D0590914E058D37910582
:10EEE00009F4FCC508F058C28E34910509F49BC69C
:10EEF00008F021C18B31910509F4F4C508F0B1C0C7
:10EF00008531910509F46BC508F07AC0813191050E
:10EF100009F424C508F044C0029708F0AECC80E59F
:10EF20000E94DC37C12CD12C7601882321F00E946D
:10EF3000242A6B017C0183E50E94DC37882361F081
:10EF40000E94643720E030E04AE754E40F94A66D55
:10EF50000F94A5756B017C010E942CFB80915405D8
:10EF600090915505009709F4F3C40F944D358091A5
:10EF70004D0590914E056BE572E1892B11F463E527
:10EF800072E130E020E041E256E482E00E948643F4
:10EF900040E0C701B6010E94B96F0F94774784CC57
:10EFA0008231910511F40C946380449709F065CC8B
:10EFB00080916A1783FF0BC58EE892E10E947C4125
:10EFC00080916A1783FF17C08BE897E10E94D1E90F
:10EFD0008BE1EBE8F7E1DE01119601900D928A9545
:10EFE000E1F770E060E0CE0101960E9441EECE01B3
:10EFF00001960E94F9398FE792E10E947C4154CC3E
:10F000008831910509F400C5B0F48631910509F401
:10F01000EAC4479709F031CC809154059091550589
:10F02000FC012191222309F4E8C42032D1F7DF0149
:10F0300011971C92F6CF8931910509F44FC54A9773
:10F0400009F01BCC80916A1783FF2ECC83E50E94C8
:10F05000DC37882309F428CC0E94452A0E945E28C8
:10F0600023CC8132910509F4AFC508F03EC08E3142
:10F07000910509F499C568F48C31910509F48CC5A2
:10F080004D9709F0FACB80916A178E7F80936A17AB
:10F090000BCC8F31910509F49BC5809709F0EDCB1E
:10F0A00080916A1782FD0E942CFB80916A1783FF72
:10F0B000FBCB60E080E50E94BC39182F682F80915F
:10F0C0005405909155050E944DED83E50E94DC3773
:10F0D000882321F00E94452A0E945E280E9448E170
:10F0E0001111E2CB0E94EC3EDFCB8B34910509F489
:10F0F00092C5B0F48033910509F489C5893491052E
:10F1000009F0BBCB80E50E948E37882309F4CCCB75
:10F110000E94552A853608F084E680935E05C4CBAC
:10F120008C34910509F47BC58D34910509F0A5CB8C
:10F130000E94FF3EB9CB8D36910509F435C608F023
:10F1400086C08C35910509F4C2C708F03FC08335ED
:10F15000910509F4B0C778F48135910509F48EC79B
:10F160008235910509F089CB8091DD088F7D806122
:10F170008093DD0899CB8435910509F4A4C78535C2
:10F18000910509F07ACB83E50E948E37882309F434
:10F190008BCB0F945F526093BA087093BB08809337
:10F1A000BC089093BD080E94643720E030E04AE735
:10F1B00054E40F94A66D0F94A57560932E0570937B
:10F1C0002F0580933005909331056ECB8A369105DB
:10F1D00009F448C698F58836910509F4B6C589360C
:10F1E000910509F04ACB0E949658182F87FD0AC056
:10F1F0008CE593E10E947C41812F0E94DEEF8AE042
:10F200000E9443412CA92093C308E5960FB6F894B9
:10F21000DEBF0FBECDBFDF91CF911F910F91FF9049
:10F22000EF90DF90CF90BF90AF909F908F907F90A6
:10F230006F905F904F903F902F9008958B3691057F
:10F2400009F44BC68C36910509F42ECB16CB8337C7
:10F25000910509F4DDC708F05DC08037910509F418
:10F2600023CB08F048C08E36910509F445C68F3689
:10F27000910509F002CB83E50E948E37882331F097
:10F2800060E083E50E9456388093DB100E94F757B8
:10F290008DE693E10E947C418091DB10882309F484
:10F2A0003EC610E000E020E08091DB1090E0B0E08E
:10F2B000A0E0002E04C0B695A795979587950A946F
:10F2C000D2F780FF12C0FF24F394F20E222319F02C
:10F2D0008CE20E944341F801EE0FFF1FED59FC4EF6
:10F2E000859194910E947C412F2D0F5F1F4F053017
:10F2F0001105D1F61EC48137910509F413C6823772
:10F30000910509F0BACA0F94D7468AEF96E10E9498
:10F3100069F6CACA8737910509F4A8C770F5853719
:10F32000910509F479C78637910509F0A6CA0091BD
:10F3300054051091550594E0F12C40E0915009F4EA
:10F3400084C7F8018081282F2B7F213409F076C7EC
:10F350002181213309F079C7813409F484C78534C8
:10F3600009F441E098012E5F3F4F89012F5F3F4F25
:10F37000F80180818032C9F3E1CF8837910509F423
:10F3800079C78937910509F078CA10922D08109233
:10F390002C080F94B31A88CA8239E1E09E0711F451
:10F3A0000C94CA8408F0EBC08C3D910511F40C94C8
:10F3B000508208F072C0893C910509F4D0C708F06A
:10F3C00051C08B39910509F432C6B8F48C389105D7
:10F3D00009F4C7C58139910509F04FCA70E060E0B2
:10F3E00083E50E94AD39823008F44DC70E94F3577F
:10F3F0008DEA93E10E947C4157CA8E3B910509F446
:10F40000D7C5883C910509F038CA0E949658182F34
:10F4100087FD4ACA0091FC0884E40E94DC37F82E7C
:10F420008823B9F00E9464374B015C0120E030E092
:10F43000A9010F94406D882309F48FC724E01202BC
:10F44000F0011124E850F74F80829182A282B382AA
:10F450000F2D602F83E50E94BC398093FC080E9429
:10F4600036DC22CA8D3C910509F4C6C758F48B3CA2
:10F47000910509F49EC78C3C910509F0FEC90E94D4
:10F48000604412CA8E3C910509F4BAC7833D9105C8
:10F4900009F0F3C90E94BB5807CA8D3221E09207D8
:10F4A00011F40C948A8308F044C08831A1E09A07D3
:10F4B00011F40C94EA82F0F48D3D910511F40C9452
:10F4C00093828A3F910509F0D8C983E40E948E3760
:10F4D000882321F00E9460370E942C2C60915902F1
:10F4E00070915A028DE294E10E94D9498AE00E940B
:10F4F0004341DAC98232E1E09E0711F40C9486831D
:10F500008C32914009F0B9C964E071E083E50E9452
:10F51000E9378C0168EE73E080E50E94E9378938AD
:10F5200023E1920710F088E893E1B8010E94539517
:10F53000BBC9803321E0920711F40C940C8468F469
:10F540008E32A1E09A0711F40C9480848F3291409E
:10F5500009F093C90E94E544A7C98039E1E09E07FC
:10F5600011F40C94C6848139914009F086C98091C8
:10F57000B90881113CCC81E00F945E1C38CC8C30F2
:10F5800022E0920711F40C94E48508F0FDC0863E59
:10F59000A1E09A0711F40C94608508F0C6C0843A83
:10F5A000E1E09E0711F40C94D284B8F48A3921E08A
:10F5B000920709F479C98D39914009F05EC983E554
:10F5C0000E948E37882311F40C9492860E94692A37
:10F5D00080931C060E94D93967C9853AA1E09A0731
:10F5E00011F40C94D6848C3A914009F046C987E016
:10F5F0000F947F2E811158C968E2C62E6DE2D62E77
:10F60000E3EDF9E0F9A7E8A79E012F5F3F4F19014D
:10F61000790110E000E0C6010E943232A8A5B9A528
:10F620008D909D90AD90BD90B9A7A8A7A50194011C
:10F630000F9431742B013C01F701408251826282A8
:10F64000738220E030E040EA51EC0F94927687FD1F
:10F650000AC020E030E040EA51E4C301B2010F9457
:10F66000406D181684F4F801E45BF24DE4911E1627
:10F6700054F4B7FAB094B7F8B094D7018D929D9234
:10F68000AD92BC921397F70181909190A190B190A7
:10F690007F0120E030E040EA51ECC501B4010F9455
:10F6A000927687FF02C00C944B8520E030E040EA60
:10F6B00051E4C501B4010F94406D181614F40C9474
:10F6C0004B850F5F1F4FF4E0CF0ED11C03301105A7
:10F6D00009F0A1CF59E0E52E59E0F52E10E0F10137
:10F6E00081919191A191B1911F01F7018193919322
:10F6F000A193B1937F01812F0F94C70E1F5F133029
:10F7000071F70F948B1960E084EA94E10E942CCA8F
:10F7100063E972E084E690E00E9453956AEB72E040
:10F7200084E690E00E945395BFC8863FE1E09E07C3
:10F7300011F40C94D68568F4843F21E0920711F40B
:10F740000C94D285853F914009F097C80F94692E9B
:10F75000ABC8873FA1E09A0711F40C94DA85883F83
:10F76000914009F08AC881E0809391060F945D2E44
:10F7700010929106882309F497C80E94F75780EEEB
:10F7800094E10E947C4190C88C36E3E09E0709F426
:10F790008BC808F08DC08D3B22E0920711F40C94C9
:10F7A0000F8608F076C08835A2E09A0711F40C9411
:10F7B000F5858B35924009F060C80E949658082F55
:10F7C00087FD72C885E50E948E37882369F10E9403
:10F7D00064374B015C01E02E002E000CFF0820E096
:10F7E00030E0A9010F94927687FF04C0B7FAB09475
:10F7F000B7F8B09420E030E84BE354E4C501B4011D
:10F800000F949276970143E0220F331F4A95E1F758
:10F810002C5E394F181614F40C94F985D9018D9289
:10F820009D92AD92BC9213978CE40E948E378823F0
:10F8300009F43AC80E9464376B017C01002E000C69
:10F84000110B20E030E0A9010F94927687FF04C0ED
:10F85000F7FAF094F7F8F09420E030E84BE354E442
:10F86000C701B6010F949276980193E0220F331FDF
:10F870009A95E1F72C5E394F181614F40C9404860F
:10F88000D9011496CD92DD92ED92FC9217970C94CB
:10F8900054748E3BE2E09E0711F40C94138683357A
:10F8A000934011F00C943D740E94E3490C945474FD
:10F8B000873E23E0920711F40C948286C8F48438C2
:10F8C000A3E09A0711F40C941786803A934011F044
:10F8D0000C943D74209154053091550590916A1710
:10F8E000926090936A17C9010E9404ED0C945474BD
:10F8F000883EE3E09E0711F40C94A886893E93406D
:10F9000011F00C943D740F94495E81110C94547461
:10F910000E94D1390F94015E0F94BA1F6D337105A7
:10F920008105910520F08DE495E10E94908889E49D
:10F9300095E10E94908884EE80935E0585E395E1D1
:10F940000E947C4181E395E10E9490880C9454745C
:10F9500060E083E692E10E942CCA09CB80915005B9
:10F9600084FD17C08091520587FD13C08091530517
:10F97000837079F460E086E792E10E942CCA5F9878
:10F980008A988091080181708093060112980C94E6
:10F99000547488E50E948E3781115F9889E50E9432
:10F9A0008E3781118A988AE50E948E37882329F044
:10F9B0008091080181708093060185E40E948E3752
:10F9C000882311F40C94547412980C9454740E946B
:10F9D000F7578FE992E10E947C410C9454740E9485
:10F9E0006BE90C94547480916A1782FF02C00C94E6
:10F9F00054740E945AE90C94547460E00E944DEDD6
:10FA000010925E050C94547483E50E94DC378823C1
:10FA100021F00E94452A0E945E2884E50E94DC377E
:10FA20008823A9F00E94452A6B017C010F94612074
:10FA3000C0920C06D0920D06E0920E06F0920F06D0
:10FA4000CD28CE28CF2819F081E08093DC08809162
:10FA5000A8068823F9F080E090E0A0EAB1E4898369
:10FA60009A83AB83BC831C8E1D8E1E8E1F8E18A2A4
:10FA700019A21AA21BA210E000E020E0AE014F5F25
:10FA80005F4FBE01645E7F4FCE0180960E94356C51
:10FA90000C9454740E94C83E882381F00E9448E16F
:10FAA0000E94EC3E83E599E00E94F9E810920D1265
:10FAB00010920E1210920F121092101261E089EB48
:10FAC00091E20E943F4341E851E269EA72E185E038
:10FAD0000F94EA480F9477470C9454740E949F71D6
:10FAE0000C94547483E40E948E37882361F18FEB69
:10FAF00092E10E947C418091D2188823F9F0BE01E6
:10FB00006F5F7F4F8FEC98E10E948CE8CE010196E9
:10FB10000E943EE5CE0101960F941B5E80919813E2
:10FB2000882339F080E20E94434188E993E10E94F2
:10FB30003EE58AE00E9443410C94547485EB92E1C7
:10FB40000E947C41F6CF83E50E94DC37882301F1D7
:10FB50000E94552A182F8C3308F08CE380932805D7
:10FB60000F945F526B017C01212F30E0A8EEB3E0CF
:10FB70000F94D873C60ED71EE81EF91EC092240536
:10FB8000D0922505E0922605F09227050C94547436
:10FB90000E9406E10C94547480915405909155058F
:10FBA0000E9404ED0C94547480916A1783FD02C086
:10FBB0000C9454740F94B747809154059091550557
:10FBC0000E949CEC0C9454740E94625E0C945474D9
:10FBD0000F94BA1F6C8F7D8F8E8F9F8FBE016F5FCA
:10FBE0007F4FCE014C960E94E92FCE0101960F94D3
:10FBF0004D350E94F757BE016F5F7F4F8EEC92E14B
:10FC00000E94585E8AE00E9443410C9454740E9402
:10FC1000254B0C9454740E94EC3E0C9454740F9435
:10FC2000B4200C94547470E060E083E50E94AD3918
:10FC30008E34910531F40E944DFA0F9477470C945D
:10FC4000547489E393E10E947C4160911C08709197
:10FC50001D0880E393E10E943D4460911E0870916D
:10FC60001F0883E293E10E943D4460911C0870915B
:10FC70001D0880911E0890911F08681B790B8091C8
:10FC8000DC08815021E030E0823010F030E020E0EC
:10FC9000621B730B88E193E10E943D448AE00E945D
:10FCA000434180E193E10E947C4180912008909142
:10FCB0002108A0912208B09123088C8F9D8FAE8FD0
:10FCC000BF8FBE016F5F7F4FCE014C960E94E92F20
:10FCD000BE016F5F7F4F83E093E10E94585E809189
:10FCE000240890912508A0912608B09127088C8FB0
:10FCF0009D8FAE8FBF8FBE016F5F7F4FCE014C9641
:10FD00000E94E92FBE016F5F7F4F83EF92E10E9457
:10FD1000585E20E030E04AE754E460912808709192
:10FD2000290880912A0890912B080F942C75AB011B
:10FD3000BC018BED92E10E944F448DE60E9443414D
:10FD40008AE00E9443410C9454748091DB1083FF3D
:10FD500002C00C9454740E94965887FF02C00C9401
:10FD6000547489E40E94DC37882311F40C941188C0
:10FD70000E94552A90E01816190614F481E090E0CC
:10FD800026E0289FF001299FF00D1124EC58F74F31
:10FD9000808191810E94AEFA61E080E00F94C6609C
:10FDA0000F94DF600C9454748091DB1083FF02C0C9
:10FDB0000C9454740E949658F82E87FF02C00C943D
:10FDC000547489E40E94DC37882311F40C941C8855
:10FDD0000E94552A90E01816190614F481E090E06C
:10FDE00026E0289FF001299FF00D1124EC58F74FD1
:10FDF0008081918110E00E94AEFA61E081E00F9471
:10FE0000C66020914C1630914D1680914A16909103
:10FE10004B1682179307F4F48CE493E19F938F932E
:10FE200087E593E19F938F931F920E9411CA0F90D1
:10FE30000F900F900F900F9001E00F94DF60002360
:10FE400011F40C94547440E0612F8F2D0E94D6F170
:10FE50000C94547481E493E1112301F3012FEDCF4D
:10FE600010E0EBCF60E080E50E945638F82E31E0DC
:10FE7000381710F40C94547481E40E948E3760910A
:10FE8000150A062F10E0811102C00FEF10E089E47F
:10FE90000E94DC37882311F40C942E880E94552A86
:10FEA00090E01816190614F481E090E026E0289FEF
:10FEB000F001299FF00D1124EC58F74F04811581B2
:10FEC000EF2DF0E0EB5EF54F0F3F110519F010F04C
:10FED0000FEF10E000830C94547460E080E50E9402
:10FEE0005638823010F00C945474E82FF0E0EB5E3A
:10FEF000F54F10820C9454748EE40E94DC378823F2
:10FF000011F40C9454740E94452A6093A6117093C6
:10FF1000A7118093A8119093A9110C9454748FE5A4
:10FF200093E10ECE83E50E94DC37882369F00E94BE
:10FF3000552A8D3320F480931F020C9454748CE363
:10FF400080931F020C9454740E94F75760911F0213
:10FF500084E793E10E9447448AE00E9443410C9465
:10FF600054748091DB1083FF02C00C94547489E4B4
:10FF70000E94DC37882311F40C943A880E94552A99
:10FF800090E01816190614F481E090E026E0289F0E
:10FF9000F001299FF00D1124EC58F74F82819381D5
:10FFA0000E94553761E080E00F94C6600C94547451
:10FFB0008091DB1083FF02C00C94547489E40E948A
:10FFC000DC37882311F40C9445880E94552A90E070
:10FFD0001816190614F481E090E026E0289FF0013D
:10FFE000299FF00D1124EC58F74F8281938110E086
:10FFF0000E94553760E081E00F94C6602091E908C7
:020000021000EC
:100000003091EA088091E7089091E80882179307F9
:100010001CF48AE893E102C08BE793E160E00E9460
:100020002CCA60E0812F0E9451F00C94547483E537
:100030000E94DC37882311F40C9454740E94552AD2
:10004000182F8C3308F08CE380932D050F945F52AA
:100050006B017C01212F30E0A8EEB3E00F94D87340
:10006000C60ED71EE81EF91EC0922905D0922A0599
:10007000E0922B05F0922C050C9454740E949CF392
:100080000E943DFB0E94FF3E0E94023F1092CE085C
:100090001092CD081092CC0868EE73E080E090E0FA
:1000A0000E94793E0E946C2660E089E993E10E94FB
:1000B0002CCA0C9454748091DD088F7E80628093EA
:1000C000DD080C9454740E94F7370C9454740E9409
:1000D000965887FF02C00C9454748091500584FD9B
:1000E00009C08091520587FD05C08091530583703A
:1000F00009F489C028EBC22E22E0D22E3CEDE32E7B
:1001000030E1F32E10E0D6018D916D010E94DC37B5
:10011000882309F465C0133009F06DC00E9464376C
:100120004B015C0120E030E040EA51E40F94406D67
:1001300087FF4EC0A50194016091FC107091FD10E5
:100140008091FE109091FF100F942C752B013C01B3
:10015000AC019B016091090A70910A0A80910B0A17
:1001600090910C0A0F94A66D6093090A70930A0A85
:1001700080930B0A90930C0AA301920160910C11D9
:1001800070910D1180910E1190910F110F94A66D29
:1001900060930C1170930D1180930E1190930F11B9
:1001A0006091F5097091F6098091F7099091F8092D
:1001B0000F94456DA30192010F94A66D0F94A57540
:1001C0006093F5097093F6098093F7099093F80905
:1001D0008092FC109092FD10A092FE10B092FF1041
:1001E0001F5FF4E0EF0EF11C143009F08CCF0E9479
:1001F00008FB0C9454740E946437F701648B758B70
:10020000868B978BEDCF81E00F943C470C94547410
:100210000E94A3410C94547480915405909155050B
:10022000009741F0DC012C91222321F00F944D35F1
:100230000C9454740F9477470C945474803529F4BB
:10024000818180538A3008F48DC841110E94F7578C
:10025000FF2021F08AEA93E10E947C41C8010E94BC
:100260004A410C945474FF24F3947CC80F946F1A81
:100270000C94547481E080932D0880932C080F9483
:10028000B31A0C9454748C01112788E40E94DC3753
:100290008823C1F00E9460378A3A91050CF44BC064
:1002A0000E9460378D3291400CF048C00E94603748
:1002B00026E0209FF001219FF00D1124EC58F74F0C
:1002C0009183808382E40E94DC378823A9F00E9416
:1002D00060370597B4F10E9460378D389105A4F519
:1002E0000E94603726E0209FF001219FF00D11242D
:1002F000EC58F74F9383828386E40E94DC3788238F
:1003000011F40C9454740E94603797FD20C00E9431
:1003100060378F3F910509F0ECF40E94603726E0CA
:10032000209FF001219FF00D1124EC58F74F958389
:1003300084830C9454748AEA90E0BACF8CE291E002
:10034000B7CF85E090E0CECF8CE890E0CBCF90E0C7
:1003500080E0E5CF8FEF90E0E2CF80E07EC80E94A2
:10036000965887FF02C00C94547408EB12E08CED91
:10037000E82E80E1F82E9CEBC92E92E0D92ED80110
:100380008D918D010E948E37882359F00E94643729
:100390000F94A575F70160837183828393830E9414
:1003A000BAFAF4E0EF0EF11CC016D10641F70C9436
:1003B00054740E94965887FF02C00C94547418EB32
:1003C000E12E12E0F12E10E000E0D7018D917D01C9
:1003D0000E948E37882349F00E946437F801E45266
:1003E000FF4E64A375A386A397A30C5F1F4F003134
:1003F000110559F70C9454740E943E420C945474A5
:10040000B9E0EB2EB9E0FB2E10E088E5810F0E94E9
:100410008E37882351F00E946437F701608371831F
:1004200082839383812F0F94C70E1F5FF4E0EF0E3A
:10043000F11C133051F78091520587FF02C00C94D4
:10044000F77680915305837011F00C94F776409104
:10045000090950910A0960910B0970910C098FEC00
:1004600093E10E944F4440910D0950910E09609113
:100470000F09709110098AEA96E40E944F44409156
:10048000110950911209609113097091140987EABA
:1004900096E40E944F448AE00E9443410C945474B5
:1004A00082E40E948E37882341F080917B029091F4
:1004B0007C02909321028093200282E50E948E3775
:1004C000882341F0809120029091210290937C0238
:1004D00080937B0283E50E94DC37882331F00E9401
:1004E000603790937C0280937B02809150059091BD
:1004F0005105A0915205B0915305892B8A2B8B2B66
:1005000011F00C94547460917B0270917C0286ED22
:1005100093E10E94D94985E20E9443418AE00E940A
:1005200043410C9454740E949658082F87FF02C0D0
:100530000C94547483E50E94DC37002E000C110BE0
:100540007801EE0CFF1C882359F10E946037F701F7
:10055000E35CFD4F91838083000F111F000F111F7B
:10056000980126573D4F7901BC01990F880B990BD3
:100570000F94476D2AE037ED43E25CE30F94A66DDC
:10058000085F194FD8012D913D914D915C910F94C9
:10059000A66DF70160837183828393830C945474F6
:1005A0000E94F75785E40E94434180E3800F0E9438
:1005B0004341F701E35CFD4F608171818AED93E176
:1005C0000E94D94985E20E9443418AE00E9443414A
:1005D0000C94547480E50E948E37882311F40C9497
:1005E00054740E9460378C01892B09F082C083E526
:1005F0000E948E37882391F00E9460378F3F9807C2
:1006000031F484ED96E10E94093F0C945474BC01CE
:1006100084ED96E10E94773F0C9454740E94F75742
:1006200070E060E085EE93E10E94D9498091D61692
:1006300058E5C52E52E0D52EC81AD10887FDD394AF
:10064000CC0CDD1CCC0CDD1C0D2C000CEE08FF08C6
:100650008091D51678E8872E912C881A910887FD0D
:100660009394880C991C880C991C092C000CAA08DE
:10067000BB088091D41690E08F3FC9F1FC01EE0FCA
:10068000FF1FE80FF91FE557F94E8181928133E092
:10069000880F991F3A95E1F7B0E0A0E044E0B595E6
:1006A000A795979587954A95D1F702969C012F5F5C
:1006B0003F4F032E000C440B550B281939094A09EA
:1006C0005B09A4EBB0E00F94C573A701960128194C
:1006D00039094A095B090F94A673B90182EE93E1C7
:1006E0000E94D9498AE00E9443410C94547480E0EE
:1006F000DDCF0E94F357B8018CEF93E10E94D949F6
:100700008DEE93E10E947C410C9454740E94FB573F
:100710000C94547460E085E40E945638811174C0D2
:1007200080E50E948E37882351F00E9464376093E1
:100730004F1670935016809351169093521689E479
:100740000E948E37882381F00E9464372CEA35ECB2
:1007500047E25EE30F94A66D6093531670935416B0
:10076000809355169093561684E40E948E37882302
:1007700081F00E9464372CEA35EC47E25EE30F9487
:100780002C75609357167093581680935916909352
:100790005A160E94F75740914F165091501660918B
:1007A0005116709152168BE094E10E944F442CEA4E
:1007B00035EC47E25EE360915316709154168091D8
:1007C0005516909156160F942C75AB01BC0187E01D
:1007D00094E10E944F442CEA35EC47E25EE36091DD
:1007E0005716709158168091591690915A160F9479
:1007F000A66DAB01BC0183E094E10E944F448AE006
:100800000E9443410C9454740E94F3578FE094E18A
:100810000E947C410C94547480E50E948E3788239A
:1008200051F00E9464376093EC087093ED08809358
:10083000EE089093EF0889E40E948E37882381F0B8
:100840000E9464372CEA35EC47E25EE30F94A66D14
:100850006093F0087093F1088093F2089093F30886
:1008600084E40E948E37882381F00E9464372CEA4A
:1008700035EC47E25EE30F942C756093F4087093B7
:10088000F5088093F6089093F7080E94F757409177
:10089000EC085091ED086091EE087091EF0889E244
:1008A00094E10E944F442CEA35EC47E25EE360910C
:1008B000F0087091F1088091F2089091F3080F947C
:1008C0002C75AB01BC0185E294E10E944F442CEAF7
:1008D00035EC47E25EE36091F4087091F508809191
:1008E000F6089091F7080F94A66DAB01BC0181E268
:1008F00094E10E944F448AE00E9443410C94547456
:1009000083E50E948E37182F882369F00E94603794
:100910009C0190938F0280938E0291E0232B09F02B
:1009200090E09093270A80E50E948E37882361F03B
:1009300020918E0230918F02232B11F00E94692AA0
:100940008093270A0C94547411110C9454740E94CF
:10095000F75788E594E10E947C418091270A88231B
:1009600091F080E494E10E947C4160918E0270914C
:100970008F0287E494E10E94D94983E494E10E94C4
:100980007C410C9454748CE394E1EDCF0E942CFBD9
:100990000C9454740E9438320E940A2A0F948B19C6
:1009A0000C9454740E94AA590C9454746FEF7FEF06
:1009B00089E40E94AD39082F6FEF7FEF8AE40E942F
:1009C000AD39182F8AE50E94DC37D12C811107C080
:1009D00081E50E94DC37D82E882309F467C3C02E36
:1009E00081E0800F863008F04EC0912E81E0810FAB
:1009F000863008F048C00E9464372B013C01F02E7D
:100A000007FDF12C07FF02C004E0C02E812E17FD68
:100A1000812C17FF02C014E0912EB5E03B2ECF14BD
:100A200010F40C945474E82C3F9C500111249E1433
:100A300040F10E2D10E020E030E0A901DD2069F04A
:100A4000F501E00FF11FEE0FFF1FEE0FFF1FE35E3A
:100A5000F94F20813181428153810A0D1B1D000F06
:100A6000111F000F111F035E194FC301B2010F9434
:100A70003274D8016D937D938D939C931397E39477
:100A8000D6CFF394CCCF0E94F3578BE894E10E9429
:100A90007C410C9454740E94F35782EC94E10E94C0
:100AA0007C4161E084EB94E10E942CCA0E94989AF8
:100AB00068E270E088EC90E00E9453950C945474C6
:100AC00084E50E948E378823A1F010925F05109272
:100AD00060051092610510926205109263058FEF18
:100AE0000E946C2861E070E084E50E94AD3980933B
:100AF000630583E50E948E37882321F00E946037CA
:100B00000E946C2883E40E948E37882331F0809104
:100B10002F02803210F40E94743A80E50E948E37D2
:100B2000882331F00E946037803210F40E94743ABA
:100B300085E50E948E37882311F40C9454740E942A
:100B40006037803210F00C94547441E050E060E063
:100B500070E0082E04C0440F551F661F771F0A94CB
:100B6000D2F7409550956095709500915F05109172
:100B70006005209161053091620540235123622375
:100B8000732340935F0550936005609361057093F4
:100B9000620590912F0289130C9454741092DA100C
:100BA0000C9454740E9413F70C9454740F94C21A4A
:100BB0000C94547461E083E50E94BC3991E089276C
:100BC0000F9416270C94547480916A1782FF05C005
:100BD000806480936A170C94547483FD02C00C9453
:100BE00054740F94B7470C9454740E948F700C94F3
:100BF000547480E090E8ABE3B4E4F901808391831E
:100C0000A283B3830C94147C80E090E8ABE3B4E45B
:100C1000F90184839583A683B7830C9454740E944E
:100C20003C6B0C9454740E94436E0C945474A090CA
:100C30000D0AB0900E0AC0900F0AD090100A8BE4F3
:100C40000E94DC37882339F10E9464377B018C01D4
:100C500020E030E0A9010F94927687FD0AC020E0E1
:100C600030E040E251E4B701C8010F94406D18161E
:100C7000A4F48FE30E9443418BE40E94434186EF3A
:100C800094E10E947C418EEE94E10E947C418BEEC7
:100C900094E10E947C41750186019701A801B5018C
:100CA000C6010F94406D882361F00E942CFBC701A0
:100CB000D80180930D0A90930E0AA0930F0AB09367
:100CC000100A8091500590915105A0915205B09164
:100CD0005305892B8A2B8B2B11F00C9454740E9492
:100CE000F75740910D0A50910E0A60910F0A7091CA
:100CF000100A8AE095E10E944F448AE00E94434135
:100D00000C94547481E0809373081092301460E066
:100D100083E50E94BC3981110C9454740F945836A9
:100D20000C9454740E94F7578CE195E10E947C4129
:100D300080911C06882349F089E195E10E947C415D
:100D40008AE00E9443410C94547485E195E1F6CF0A
:100D50000E9402890C94547410914D050F945F52B7
:100D60006093BA087093BB088093BC089093BD0849
:100D7000112311F40C945474812F0E9428EF0C94C9
:100D80005474111107C011E089E50E948E37811358
:100D90000C94EF74012FF11204C001E011E0FF2464
:100DA000F39482E50E94DC37882311F40C94F374E9
:100DB0000E9464376CA37DA38EA39FA320E030E044
:100DC000A9010F94406D882381F0011105C0111114
:100DD00003C0FF2009F413C160E0CE0184960F9494
:100DE00005110E94CC400E947B40002309F480C082
:100DF000112309F47AC01092D3091092D4091092E9
:100E0000D5091092D6091092D7091092D8091092DC
:100E1000D9091092DA090F940A1284E39DE20E9424
:100E200032324B015C0188E39DE20E9432322B0199
:100E30003C01AC019B01C501B4010F9492761816D8
:100E400014F00C94F974A5019401C301B2010F943C
:100E50002C759B01AC010F94A66D20E030E040E8BA
:100E60005FE30F9432740F94E07620E030E048E4C2
:100E700052E40F94A66D68A379A38AA39BA320E0F4
:100E800030E040EC5FE3C301B2010F94A66D9058CF
:100E900069837A838B839C8320E030E040EC5FE3BE
:100EA000C501B4010F94A66D90586C8F7D8F8E8F05
:100EB0009F8FAE01405E5F4FBE016F5F7F4FCE01DF
:100EC0004C960F94C4100F94E41C1092D309109206
:100ED000D4091092D5091092D6091092D709109210
:100EE000D8091092D9091092DA0980E00F94D91D1F
:100EF000112319F081E00F94D91DFF2009F47FC060
:100F000083E00F947F2E81117AC00F940A122091F2
:100F1000090930910A0940910B0950910C0960E0D0
:100F200070E086EE92E40F9431742B013C01209125
:100F30000D0930910E0940910F095091100960E0A0
:100F400070E086EE92E40F9431744B015C01809165
:100F5000DB099091DC09A091DD09B091DE09809355
:100F6000B0089093B108A093B208B093B308009171
:100F7000E3161091E416D8012D913D914D915C91AD
:100F8000C301B2010F9431746093A8087093A9084B
:100F90008093AA089093AB08F8012481358146819B
:100FA0005781C501B4010F9431746093AC087093FC
:100FB000AD088093AE089093AF0888EA98E00E944D
:100FC0009924882311F40C94FF741C8E1D8E1E8EA0
:100FD0001F8E88E0E8EAF8E0DE01119601900D929C
:100FE0008A95E1F7AE01445E5F4FBE016B5F7F4FB4
:100FF000CE0101960F94C41082E00F94D91D0F9476
:101000000A1280912C0880932D088E2D0E948D3C11
:101010000F94B50F83E0809389020F948B190C9481
:10102000547483E50E94DC37882311F40C94D07E3D
:101030000E9460370C94CA7E83E50E94DC37182F2B
:10104000811108C082E50E94DC37082F882311F443
:101050000C94307F0E9460370C94FB7E83E50E94E5
:10106000DC37882311F40C94607F0E94452A8B01A1
:101070000C94607F83E50E94DC37882311F40C9484
:1010800054740E9460370C94D07F83E50E94DC3753
:10109000182F811107C082E50E94DC37882311F4E4
:1010A0000C9454740E9460370C94F87F0E94F3579C
:1010B0008BE694E10E947C410C945474882309F4DB
:1010C00062CE6BCEDF92EF92FF920F931F93CF937E
:1010D000DF93EC01E090C508F090C6088AE0D82EB6
:1010E0006AE070E0CE010F9480778C01009711F0D8
:1010F000FC011082CE010E94C83081E00E947F7204
:101100000115110519F0E801D992EACFC701DF9165
:10111000CF911F910F91FF90EF90DF900C94C8300A
:101120004F925F926F927F928F929F92AF92BF92F7
:10113000CF92DF92EF92FF920F931F93CF93DF93A3
:10114000CDB7DEB77C014DB65EB66090C508709035
:10115000C6088DB69EB66AE070E0C7010F947B6C3E
:101160006C018C010E191F09892B21F4C7010F9402
:101170008D6C8C01C80101962DB73EB7281B390B29
:101180000FB6F8943EBF0FBE2DBF8DB79EB7019628
:101190005C01A801B7010F94AE6CF501E00FF11FDF
:1011A0001082C5010E94C83081E00E947F72C11484
:1011B000D10451F076019FEFE91AF90A0FB6F894BD
:1011C0009EBE0FBE8DBEC5CF0FB6F8949EBE0FBE9D
:1011D0008DBEC3010E94C8300FB6F8945EBE0FBE2C
:1011E0004DBEDF91CF911F910F91FF90EF90DF9057
:1011F000CF90BF90AF909F908F907F906F905F90B7
:101200004F9008954F925F926F927F928F929F922C
:10121000AF92BF92CF92DF92EF92FF920F931F9304
:10122000CF93DF93CDB7DEB7C059D1090FB6F8948D
:10123000DEBF0FBECDBF0E94E739882369F083E58A
:101240000E948E37882301F120E040E070E060E0EA
:1012500082EC9AE90E94FB97C057DF4F0FB6F894D3
:10126000DEBF0FBECDBFDF91CF911F910F91FF90D9
:10127000EF90DF90CF90BF90AF909F908F907F9036
:101280006F905F904F90089583E40E948E3788237B
:1012900019F00E94B79AE0CF8090BC099090BD09E8
:1012A000A090BE09B090BF098091C50980FF05C01C
:1012B0009091DB1098609093DB10869581708093FD
:1012C000270A87EE90E10E94908880914B099091C7
:1012D0004C099E012F5F3F4F7901009799F09F9332
:1012E0008F938EED90E19F938F933F932F930F9465
:1012F000D76CC7010E9462880F900F900F900F90DB
:101300000F900F908091490990914A09009799F0A8
:101310009F938F9385ED90E19F938F93FF92EF9230
:101320000F94D76CC7010E9462880F900F900F90A6
:101330000F900F900F906E0131E8C30ED11C609199
:1013400028097091290980912A0990912B09860119
:1013500023E041E00F940D689F938F9383EC90E11D
:101360009F938F93FF92EF920F94D76CC7010E94C7
:1013700062888BEB90E10E94908887E08093B808A8
:10138000809307060F900F900F900F900F900F9083
:10139000809144098823F9F06091450970914609CC
:1013A000809147099091480923E041E00F940D682E
:1013B0009F938F9382EB90E19F938F93FF92EF9295
:1013C0000F94D76CC7010E9462880F900F900F9006
:1013D0000F900F900F9080914D098823A1F01F92DC
:1013E0008F931F921F9285EA90E19F938F93FF92B4
:1013F000EF920F94D76CC7010E9462880FB6F894E1
:10140000DEBF0FBECDBF80914E098823A9F01F9289
:101410008F931F9281E08F9385EA90E19F938F9342
:10142000FF92EF920F94D76CC7010E9462880FB6AB
:10143000F894DEBF0FBECDBF40904F0950905009C9
:10144000609051097090520920E030E0A901C30179
:10145000B2010F94406D811104C08091C50982FFD3
:1014600020C0860121E041E0C301B2010F940D6864
:101470009F938F938091C50982FB882780F91F92E3
:101480008F9388E990E19F938F93FF92EF920F944F
:10149000D76CC7010E9462880FB6F894DEBF0FBEFA
:1014A000CDBF60911A0970911B0980911C09909120
:1014B0001D098E010F581F4F23E041E00F940D6866
:1014C000782E692E6091160970911709809118097C
:1014D00090911909860123E041E00F940D686F9205
:1014E0007F929F938F9387E890E19F938F93FF92D2
:1014F000EF920F94D76CC7010E94628860911E0919
:1015000070911F09809120099091210923E041E009
:101510000F940D688CE790E10E949088DF92CF9243
:1015200082E790E19F938F93FF92EF920F94D76C95
:10153000C7010E946288809127098F9380912609B4
:101540008F938BE690E19F938F93FF92EF920F948E
:10155000D76CC7010E9462886091220970912309AB
:10156000809124099091250923E041E00F940D68B2
:101570009F938F9381E690E19F938F93FF92EF92D9
:101580000F94D76CC7010E9462888CE0ECE2F9E00E
:10159000A9E0B9E001900D928A95E1F78CE0E8E3CB
:1015A000F9E0ADEFB8E001900D928A95E1F780E0A7
:1015B0000F94C70E81E00F94C70E82E00F94C70E00
:1015C0008091C4098093DD0881E080931C060E940D
:1015D000D93983E599E09F938F9385E49DE39F93A9
:1015E0008F93FF92EF920F94D76C0FB6F894DEBFF3
:1015F0000FBECDBFC7010E9462888091C3098F933F
:101600008091C2098F938091C1098F938091C00905
:101610008F93BF92AF929F928F9283E590E19F93B9
:101620008F93FF92EF920F94D76CC7010E9462884C
:101630000FB6F894DEBF0FBECDBF0ECECF93DF93B3
:10164000C0911212C093E80981E6C89FE0011124FD
:10165000CC5EDD4E8091DB1080FF05C00E94F75705
:10166000CE010E944A41CE010E94C83080E0DF9145
:10167000CF910C947F728F929F92AF92BF92CF9234
:10168000DF92EF92FF92CF936B017C0120E030E07C
:10169000A9010F94406D87FFA3C06DEB77E386E04F
:1016A00095EBA70196010F9432746B017C0120E049
:1016B00030E040E251E40F94A66D20E030E048ECC9
:1016C00052E40F94A66D4B015C0120E030E040E253
:1016D00051ECC701B6010F94406D181654F420E088
:1016E00030E048EC52E4C701B6010F94927687FDD2
:1016F0008BC020E030E0A901C701B6010F94406D16
:1017000087FF73C060E070E080EA90ECA50194016F
:101710000F94327420E030E040E251E40F942C75D5
:101720000F949E756B017C01F7FC64C020E137E2E9
:1017300040E050E00F94A673CA01B9012AE030E0FE
:1017400040E050E00F94A673605D60939608C70177
:10175000B60128EE33E040E050E00F94A6739AE023
:10176000892E912CA12CB12CCA01B901A50194019B
:101770000F94A673605D60939708C701B60124E6D5
:1017800030E040E050E00F94A673CA01B901A50112
:1017900094010F94A673605D609398088EE2809325
:1017A0009908C701B601A50194010F94A673C62F2D
:1017B000CA01B901A50194010F94A673605D6093FD
:1017C0009A08C05DC0939B0886E998E0CF91FF908E
:1017D000EF90DF90CF90BF90AF909F908F90089543
:1017E0006DEB77E386E095E35CCF60E070E080EA44
:1017F00090E48CCFF094E094D094C094C11CD11CA0
:10180000E11CF11C6DE2A1CF20E030E0A901C7018D
:10181000B6010F94406D87FF6AC060E070E080EA17
:1018200090ECA50194010F94327420E030E040E286
:1018300051E40F942C750F949E754B015C0120E0D0
:1018400030E0A901C701B6010F94927687FD0BC065
:1018500020E030E040E251E4C701B6010F94406D52
:1018600060E287FD13C0B7FC47C0C501B40128EE94
:1018700033E040E050E00F94A673CA01B9012AE0BA
:1018800030E040E050E00F94A673605D60939708ED
:10189000C501B40124E630E040E050E00F94A673A7
:1018A0008AE0C82ED12CE12CF12CCA01B901A70184
:1018B00096010F94A673605D609398088EE2809302
:1018C0009908C501B401A70196010F94A673C62F0C
:1018D000CA01B901A70196010F94A673605D6093D8
:1018E0009A08C05DC0939B0887E998E06FCF60E0DD
:1018F00070E080EA90E495CFB094A09490948094A6
:10190000811C911CA11CB11C6DE2C0CF60913D02F5
:1019100070913E02072E000C880B990B0F94476DB7
:101920002AE037ED43E25CE30F94A66D20910806B0
:101930003091090640910A0650910B060F94A66D4E
:1019400060938A0270938B0280938C0290938D0235
:101950000895E091A308E23030F4F0E0EB5EF54F3B
:10196000809191088083089580915F178823C1F04A
:10197000815080935F17EBE8F7E1882351F08150A5
:10198000990B2BE1289FF001299FF00D1124EF53B3
:10199000F84E8BE1A6EAB7E101900D928A95E1F746
:1019A00020915F17211105C080916A178062809392
:1019B0006A1781E090E0A0E0B0E0211103C080E070
:1019C00090E0DC018093890890938A08A0938B08AB
:1019D000B0938C0810928E0881E08093880883E091
:1019E000809389020895CF93DF93EC01CB01BA0174
:1019F0000F94476D29EC38EC48EC5EE30F942C759E
:101A000020E030E040E05FE30F9432740F94A5755E
:101A10006883DF91CF9108958091590290915A0285
:101A20000C942C2CE091A30886E0E802F00111242C
:101A3000EC58F74F8091910890E095838483089546
:101A40008F929F92AF92BF92CF92DF92EF92FF92CE
:101A5000CF936B017C0120E030E0A9010F94406D31
:101A600087FD9FC06DEB77E386E095E3A7019601C4
:101A70000F9432746B017C0120E030E040E251E4CD
:101A80000F94A66D20E030E048EC52E40F94A66D70
:101A90004B015C0120E030E0A901C701B6010F94C1
:101AA000406D20E030E040EA50E487FF04C020E0D1
:101AB00030E040EA50ECC501B4010F94327420E0EC
:101AC00030E040E251E40F942C750F949E756B0149
:101AD0007C018BE2F7FE09C0F094E094D094C094AE
:101AE000C11CD11CE11CF11C8DE280939508C7013B
:101AF000B60120E137E240E050E00F94A6738AE09F
:101B0000882E912CA12CB12CCA01B901A5019401F8
:101B10000F94A673605D60939608C701B60128EE26
:101B200033E040E050E00F94A673CA01B901A5016B
:101B300094010F94A673605D60939708C701B60186
:101B400024E630E040E050E00F94A673CA01B901EA
:101B5000A50194010F94A673605D609398088EE2CE
:101B600080939908C701B601A50194010F94A6734B
:101B7000C62FCA01B901A50194010F94A673605D37
:101B800060939A08C05DC0939B0885E998E0CF9167
:101B9000FF90EF90DF90CF90BF90AF909F908F908D
:101BA00008956DEB77E386E095EB60CF8F929F927F
:101BB000AF92BF92CF92DF92EF92FF926B017C01C6
:101BC00020E030E0A9010F94406D87FD6BC06DEB04
:101BD00077E386E095E3A70196010F9432746B01D9
:101BE0007C0120E030E040E251E40F94A66D20E05B
:101BF00030E040E251E40F94A66D4B015C0120E01F
:101C000030E0A901C701B6010F94406D20E030E03B
